:100000000C94C90F0C94FA0F0C94FA0F0C94FA0F7D
:100010000C94FA0F0C94FA0F0C94FA0F0C94FA0F3C
:100020000C94FA0F0C94FA0F0C94FA0F0C94FA0F2C
:100030000C94FA0F0C94FA0F0C94FA0F0C940B6DAD
:100040000C94FA0F0C94FA0F0C94FA0F0C94FA0F0C
:100050000C94FA0F0C94FA0F0C94FA0F0C940FB145
:100060000C94FA0F0C947DB30C9453B30C94FA0FC8
:100070000C94FA0F0C94FA0F0C94FA0F0C94FA0FDC
:100080000C94FA0F0C94FA0F0C94FA0F0C94FA0FCC
:100090000C94BBA10C942BA10C9472A10C94B83AB3
:1000A0000C94FA0F0C94FA0F0C94FA0F0C94FA0FAC
:1000B0000C94FA0F0C94FA0F0C94FA0F0C94FA0F9C
:1000C0000C94FA0F0C94FA0F0C94FA0F0C9429B3B9
:1000D0000C94FFB20C94FA0F0C94D5B20C94ABB202
:1000E0000C94FA0F9F139213F713F713F713F713E8
:1000F000F713F713F713F713F7132510CF12D212D4
:10010000DC12F2121C13EB12F713F713F713F713A9
:10011000F713BF13D113EC13F219E619E619F2190C
:10012000F219CD19DA19DA19F219F219811E811EA4
:10013000692169216921DD1EB81EB81EB81E991EED
:10014000991E19225222DE2156225622B1218121E6
:100150005622192219225A4E674E6B4E6B4E864E0E
:10016000864E754E6F4E7C4ED04FF64F2950325012
:1001700035502950065029504050435017504F5089
:100180005250F352595427534353595465535954B9
:100190009953B553D7530E542A54CE54DF54D154E7
:1001A000D154DF54D454DF54D754D754D754D754F0
:1001B000D754D154E45DD35DD65DDE5DDE5DD65DA2
:1001C000D35DDE5DDE5DDE5DD35DD35DD35DDE5D83
:1001D000DE5DDE5DDE5DDE5DDE5DDE5DDE5DDE5D47
:1001E000DE5DE45D52652765626662666266626630
:1001F000F265346662666266626662663B66556692
:10020000426661658065E065E06580656165E06521
:10021000E065E065B665AB65A165CC65C1657F66E7
:10022000826627656266626662666266F265346649
:100230006266626662666266626662664E66917158
:10024000ED7131728E72A372C4713D723D723D7256
:10025000B871A471C0725776577666763F763F764E
:1002600046765F765F765F763F763F7683768376F7
:100270009C767E767E768F768876887688767E7691
:100280007E769C8C9C8C9C8C8E8C078D078D078D2C
:10029000078D078D078DBB8CAA8CCB8CE78CDD8CF2
:1002A0007696EA95EA9585962297209776968F9688
:1002B0008F968F96769676963F9632961496FD9503
:1002C000FA9532964496669666961F961F96AC9659
:1002D000DB96EF96DB96DB969F96CB96CB96CB96EE
:1002E000B196BD9644977E9744973397339744973A
:1002F0004497D099D0994497449786A389A3A1A302
:10030000B8A302A415A435A458A55BA54AA54EA57B
:1003100054A592A55FA563A569A56DA571A577A54F
:100320007BA57FA592A585A589A58DA527A62CA629
:1003300031A63BA645A6BEA64FA657A65FA669A6B0
:1003400073A67DA68CA696A6BEA6A0A6AAA6B4A6AF
:100350000CBC0CBC0CBC0CBC09BC09BC10BC10BC5B
:1003600010BC10BC10BC10BC10BC10BC09BC09BC3B
:1003700010BC10BC10BC10BC10BC0EBC0CBC076385
:100380004236B79BD8A71A39685618AEBAAB558C07
:100390001D3CB7CC5763BD6DEDFD753EF617723150
:1003A000BF000000803F08000000BE922449123EBA
:1003B000ABAAAA2ABECDCCCC4C3E00000080BEAB7E
:1003C000AAAAAA3E00000000BF000000803F000073
:1003D000000000084178D3BB4387D1133D190E3C80
:1003E000C3BD4282AD2B3E68EC8276BED98FE1A9B7
:1003F0003E4C80EFFFBE01C4FF7F3F0000000000C5
:100400000C948D790C94C9330C9464570C9467C97F
:100410000C9469A60C9491710C9469A50C943BA65C
:100420000C9419B00C949A6B0C948FB40C94ED71DD
:100430000C9454A50C94F7130C94DE210C94D75310
:100440000C94F8240C94BDB40C9443500C9499BEB5
:100450000C940E540C94DE5D0C94D2780C94A1781C
:100460000C946C900C94E4700C94DA830C94AC961D
:100470000C94A1830C94078D0C94EB830C94AB2B00
:100480000C944EA50C94CC650C94C47D0C94BC7B50
:100490000C9452500C9435A40C9496A60C94D35DF5
:1004A0000C947CBD0C9442660C9478570C94077E97
:1004B0000C942A540C94B8710C94216B0C944FA694
:1004C0000C9483760C94B4830C940EBC0C949C9C7A
:1004D0000C94B47E0C94BE780C9461BD0C94877817
:1004E0000C947ABD0C94159D0C9485A50C94902BBE
:1004F0000C94DC850C94213A0C94F2190C9429503C
:100500000C9452B00C945A4E0C94CB960C94BB8C19
:100510000C94D0640C94A0B40C9406500C9489A351
:100520000C949BB60C9466960C9463A50C9468BDD1
:100530000C94A4710C94C5390C948F760C94A1651D
:100540000C94DD8C0C94E0650C941F960C945776FB
:100550000C940CBC0C94C9780C9444970C94869F12
:100560000C94EF960C94FE830C94D6830C945BA5AC
:100570000C949C8C0C9482660C9478BD0C94E45D75
:100580000C94A7B30C9457A60C94C2850C940B6BD7
:100590000C944F640C94912B0C9456220C94595447
:1005A0000C9409BC0C944E660C94BF2E0C94A57848
:1005B0000C9460B40C94B5780C94EDB00C94667601
:1005C0000C9434660C94A38D0C94C4710C94149602
:1005D0000C94B5560C948E8C0C9415A40C94F4B316
:1005E0000C94C0280C947D7D0C94D1780C94859645
:1005F0000C949F960C94FD950C94EB120C94D0994E
:100600000C94AA7C0C94AA8C0C9488760C94D754E5
:100610000C94A0A60C9462660C9465530C947E977F
:100620000C94959F0C9480650C9458A50C94DBBE9B
:100630000C9432960C94F6B10C9435500C94323ADA
:100640000C94A82B0C9446760C9420970C947696D8
:100650000C9443B00C947E760C944AA50C947C4E7A
:100660000C9427650C9475700C944F500C94B376D1
:100670000C94806B0C941C130C9493660C94B8A38C
:100680000C9425100C9473A60C94B4A60C9474B01E
:100690000C9410BC0C94E1280C9445A60C94D883BF
:1006A0000C94047C0C942CA60C94269A0C941AB5E9
:1006B0000C9459B40C947D7C0C94F2650C9492A526
:1006C0000C94BC840C94476C0C9427A60C94D21206
:1006D0000C943B660C94CF830C94779D0C945265DC
:1006E0000C948C890C947C6B0C94D4830C94B02B5C
:1006F0000C9499530C946B4E0C9481210C94EC1334
:100700000C94E0700C9440BF0C9468640C949EB000
:100710000C94B5530C94CD190C9402A40C945FA6C0
:100720000C94098A0C947F660C9499390C94AC56FD
:100730000C94AAA60C94DF540C94F64F0C94B59F1D
:100740000C94D1540C94A48D0C940A6B0C943D72AF
:100750000C944A280C94687F0C949F130C94B19BC2
:100760000C94AB650C94864E0C94247B0C94B38350
:100770000C948F960C94BF130C944C7E0C940FC069
:100780000C9417500C9489A50C94CF120C94E5701E
:100790000C94CDB40C94DC120C9466B00C940B8ABF
:1007A0000C94F2120C947F7A0C9443530C94C07204
:1007B0000C940E7D0C9467BD0C94D0870C94692129
:1007C0000C94E78C0C9456640C94CE540C94616594
:1007D0000C94D1130C9431B40C94F3520C94B19644
:1007E0000C94BEA60C941CC00C9431A60C943397A8
:1007F0000C94289B0C9440500C94DB960C94B6659A
:100800000C94991E0C94A0B00C942B6B0C94F924AE
:100810000C944C280C94DA190C94754E0C94A59CED
:100820000C94811E0C94A0830C9477A50C94449690
:100830000C946D690C949A390C94AA560C94E09C13
:100840000C9452220C945FA50C94E28E0C9455915A
:100850000C9431720C94BD960C9496830C94A483E2
:100860000C94BD390C94674E0C94717A0C943F76BD
:100870000C9455660C947FA50C948E720C94DB7BC3
:100880000C9486780C9462BD0C94FC240C94D45483
:100890000C94CC7D0C94D65D0C94A1A30C94E6B37F
:1008A0000C94B1210C943A9A0C949D780C94F08895
:1008B0000C943F960C9432500C94D04F0C94BC6B1B
:1008C0000C9498390C9475C60C94F2390C94B22B94
:1008D0000C941FB40C9401250C94C67D0C948F8944
:1008E0000C947BA50C945B640C9422970C949C76DE
:1008F0000C942D6B0C94CB8C0C94247E0C9486A3BE
:100900000C94596B0C945F760C9418790C94921398
:100910000C94D3C10C94EA950C946BBD0C9453BE0B
:100920000C9489890C94C1650C94DD1E0C949289F9
:100930000C94A3720C94A7320C9427530C94A939ED
:100940000C946F4E0C948CA60C94FA950C94E619AA
:100950000C948DA50C94C4B30C9471A50C94A67F33
:100960000C946DA50C94B81E0C9419220C947DA6C1
:100970006364696E6F70737578585B00476F74209D
:10098000495020616464726573733A00276970206E
:100990005B69705B2C646E735B2C67775B2C737583
:1009A000626E65745D5D5D5D27202D20736574202A
:1009B0007374617469632049500A004661696C650B
:1009C0006420746F20636F6E666967757265204579
:1009D000746865726E6574207573696E672044482B
:1009E00043502E20596F752063616E20736574200B
:1009F0006970206D616E75616C6C7921000A757388
:100A0000657320444843500A00204D41534B3A003F
:100A10002047573A0020444E533A004C6F616465BA
:100A2000642066726F6D20666C6173682049503A6D
:100A3000005374617274696E67206C616E00246E7D
:100A40006F6465730024666F726D61740024646165
:100A500074617479706500302D31303000696E74C6
:100A6000656765720068737600636F6C6F72004F24
:100A70004E2C4F46462C48414C542C524553542C36
:100A8000584F4E2C584F46462C544F47474C450024
:100A9000656E756D00666C6F617400332E302E319B
:100AA0000024686F6D696500757074696D652C66EA
:100AB0007265656865617000303437346330615F3A
:100AC000323032312D30342D3032004C6967687449
:100AD0004875622000246E616D65007265616479FD
:100AE000002074727920616761696E20696E20351B
:100AF000207365636F6E6473006661696C65642C56
:100B00002072633D004177616974696E6720666F8A
:100B1000722072657461696E656420746F706963B8
:100B20007300636F6E6E656374656420617320008B
:100B3000202E2E2E0020757365723A003A000A416D
:100B40007474656D7074696E67204D5154542063E0
:100B50006F6E6E656374696F6E20746F200024730E
:100B60007461746500646973636F6E6E6563746548
:100B700064005573696E67204D5154542070617341
:100B800073776F72642066726F6D20636F6E666933
:100B900067004E3A00446576696365204E616D6575
:100BA0003A00526562696E6420737563636573739E
:100BB0002E20495020616464726573733A00457257
:100BC000726F723A20726562696E64206661696C48
:100BD0000052656E65776564207375636365737332
:100BE0002E20495020616464726573733A00457227
:100BF000726F723A2072656E65776564206661690E
:100C00006C000A4E6F206C696E6B00416363657007
:100C100074696E6720636F6D6D616E64732E2E2E26
:100C20000A004452590046414E5F4F4E4C590058FD
:100C30004F4E0048414C54002054533A0020543A3F
:100C4000003D0050696E3A00447269766572205228
:100C500065733A00416C72656164792048616C7417
:100C600065640A00416C726561647920496E616354
:100C7000746976650A00416C72656164792041632C
:100C8000746976650A005475726E696E6720584FF4
:100C90004E0A00584F464620736B69707065642E8B
:100CA000205072657620636D643A005475726E65EB
:100CB00064206F66662066726F6D3A0052657374C9
:100CC0006F7265642066726F6D3A004E6F207374A8
:100CD0006F7265642076616C756573202D20646584
:100CE0006661756C743A200049676E6F7265642C9A
:100CF000206368616E6E656C20636D643D004F75A6
:100D0000744F664D656D6F7279210A003B2000209B
:100D1000436D643D00205375623D00204974656D4C
:100D20003D0052414D3D002064656C74613A002DD8
:100D30003E002F002056616C3A00496E3A004D6F1C
:100D4000746F722074696D656F757400556E6B6E8B
:100D50006F776E20636D6400466F72636564206513
:100D60007865637574696F6E00496E76616C69644D
:100D70002050494420706172616D20617272617906
:100D80002E002C002C002C002C005049443A2063EB
:100D90006F6E666967206661696C65643A005049E8
:100DA0004420636F6E666967206C6F6164656420C0
:100DB0000050494420636F6E666967206572726FE8
:100DC00072005049443A204F7574206F66206D655B
:100DD0006D6F72790053686F770020636D643D001A
:100DE0002D00312D7769726520636F756E743A201E
:100DF0000020416464723A00646576230020616CCF
:100E000069766500204E6F64653A005365617263D0
:100E100068696E6700312D776972652073686F723B
:100E2000746564005265747279696E672064696DD7
:100E30006D657220434D440A004D6F6462757320E6
:100E4000706F6C6C696E67206572726F723D002006
:100E500056616C3A20004D423A20004E6F74207368
:100E60007570706F72746564207265672074797034
:100E7000650A00496C6C6567616C20617267756D0D
:100E8000656E74730A005265747279696E672056D4
:100E90004320434D440A004D6F6462757320706FA8
:100EA0006C6C696E67206572726F723D002D002058
:100EB00050492056616C203A004D6F646275732072
:100EC000706F6C6C696E67206572726F723D002D79
:100ED0000020464D2056616C203A005265747279AC
:100EE000696E672056432074656D7020434D440A37
:100EF00000696E00735F6F7574006D79686F6D6562
:100F000000202D3E2000202D3E2000202D3E2000E0
:100F10000000000000000000004F4E000000000034
:100F200000004F46460000000000005245535400A8
:100F300000000000544F47474C4500000048414C1A
:100F4000540000000000584F4E0000000000005800
:100F50004F46460000000000494E4352454153456C
:100F60000044454352454153450048454154000023
:100F7000000000434F4F4C00000000004155544F0B
:100F8000000000000046414E5F4F4E4C5900445255
:100F90005900000000000053544F500000000000B2
:100FA0004849474800000000004D454449554D0060
:100FB00000004C4F570000000000005452554500FF
:100FC0000000000046414C534500000000454E41E2
:100FD000424C4544000044495341424C4544005270
:100FE0004742000000000000485356000000000087
:100FF0000054787432436D643A00693136000169F7
:10100000333200027531360003753332000469381B
:1010100068000569386C0006753868000775386C1B
:10102000000878313000094164642040533A2000C0
:101030003A002066726F6D20004D4220676F742069
:101040000000002100240027002A002D003000337A
:101050000001010000040107010A01010210202023
:1010600008081020401020408002010201080402FC
:101070000101020408102040808040201008040272
:1010800001800402018040201008040201080402CB
:1010900001010204081020408001020408102040D1
:1010A0008005050505070508080808020202020A6E
:1010B0000A080804040404010101010101010103FB
:1010C00003030303030303040707070C0C0C0C0CB6
:1010D0000C0C0C0202020206060606060606060BA9
:1010E0000B0B0B0B0B0B0B00002000230026002921
:1010F000002C002F0032000001000003010601094E
:10110000013D00494E3A002D3E002000230050656D
:101110006E646564207374617465207265747269AD
:10112000657665643A003E003C00543A00437572AF
:1011300072656E74204C414E20636F6E666967283D
:1011400069702C646E732C67772C7375626E65748E
:10115000293A000A55736520746865736520636FCA
:101160006D6D616E64733A202768656C7027202D61
:10117000207468697320746578740A276D61632030
:1011800064653A61643A62653A65663A66653A3022
:1011900030272073657420616E642073746F7265EC
:1011A000204D41432D6164647265737320696E2024
:1011B000454550524F4D0A276970205B69705B2C82
:1011C000646E735B2C67775B2C7375626E65745D00
:1011D0005D5D5D27202D20736574207374617469D3
:1011E000632049500A277361766527202D2073619B
:1011F000766520636F6E66696720696E204E565271
:10120000414D0A2767657427205B636F6E666967C7
:1012100020616464725D27202D2067657420636FF0
:101220006E6669672066726F6D207072652D636FE0
:101230006E666967757265642055524C20616E64F4
:101240002073746F726520616464720A276C6F6129
:101250006427202D206C6F616420636F6E66696760
:101260002066726F6D204E5652414D0A277077648A
:1012700027202D20646566696E65204D51545420E9
:1012800070617373776F72640A276B696C6C2720C7
:101290002D2074657374207761746368646F670AC6
:1012A00027636C65617227202D20636C6561722055
:1012B000454550524F4D0A277265626F6F74272063
:1012C0002D207265626F6F7420636F6E74726F6C25
:1012D0006C657200536F6674207265626F6F74691B
:1012E0006E672E2E2E00444D58696E20427566663C
:1012F000657220616C6C6F632065727200496E6963
:101300007420696E2063683A00444D584F75742EFE
:1013100020467265653A00094453323438322065FC
:1013200072726F720009526573657420646F6E6526
:101330000009436865636B696E6720666F722031D0
:101340002D5769726520646576696365732E2E2E4C
:10135000004453323438322D31303020707265738E
:10136000656E74004572726F7220312D7720696E40
:10137000697420233220467265653A007773746180
:10138000742E20467265653A005465726D2E2046B3
:101390007265653A004572726F7220312D7720694F
:1013A0006E697420233100467265653A00445332F9
:1013B0003438325F3130305F4932435F544F5F31F0
:1013C000575F42524944474520696E697400204185
:1013D0006464723A00646576230052414D3D000A10
:1013E000312D7769726520000A6D71747420000ACE
:1013F0006D6F64627573207632000A6D6F6462757A
:101400007320763120282B29000A696E7075747359
:1014100020000A6974656D7320000A436F6E666967
:1014200067757265643A003B003D0050696E3A0092
:101430003B003D4C4F5700546865726D6F3A004F4A
:101440006E6520776972652052656164790A00468D
:101450007265653A00444D58206F7574207374614D
:10146000727465642E204368616E6E656C733A20F9
:1014700000444D5820696E20737461727465642E47
:10148000204368616E6E656C733A00206163746915
:101490007665200020696E6163746976652000209E
:1014A00076616C7565206973200020756E6B6E6FB8
:1014B000776E0A00204772703A0020696E76616C80
:1014C0006964004D6F64627573206F702066616996
:1014D0006C65640A003D005643230020636D643D43
:1014E000003D0056435F6865617423005374617466
:1014F00075732064656666657265640A002D3E003A
:101500005075623A2000636D6400434F4F4C0048B1
:10151000454154004155544F002D3E005075623AEC
:101520002000736574002D3E005075623A20002D36
:101530003E005075623A2000556E6B6E6F776E20DC
:10154000636D64200A004F4646004F4E006363738C
:101550003831313A2064617461206E6F7420617695
:1015600061696C61626C6500636373383131206E50
:101570006F7420696E697469616C697A656400458D
:101580005252004C4F57004D454449554D00484973
:1015900047480046414E5F4F4E4C59004452590057
:1015A0004845415400434F4F4C004155544F007241
:1015B0006177007175656974007377696E67006C97
:1015C0006F636B00005EBCE2613FDD83C29C7E20E6
:1015D000A3FD1F419DC3217FFCA2401E5F01E3BD0F
:1015E0003E6082DC237D9FC1421CFEA0E1BF5D0303
:1015F00080DE3C62BEE0025CDF81633D7C22C09EF7
:101600001D43A1FF4618FAA427799BC584DA3866E2
:10161000E5BB5907DB856739BAE406581947A5FBCE
:101620007826C49A653BD987045AB8E6A7F91B45C2
:10163000C6987A24F8A6441A99C7257B3A6486D8B6
:101640005B05E7B98CD2306EEDB3510F4E10F2ACA2
:101650002F7193CD114FADF3702ECC92D38D6F318E
:10166000B2EC0E50AFF1134DCE90722C6D33D18F82
:101670000C52B0EE326C8ED0530DEFB1F0AE4C1276
:1016800091CF2D73CA947628ABF517490856B4EA62
:101690006937D58B5709EBB536688AD495CB29774E
:1016A000F4AA4816E9B7550B88D6346A2B7597C942
:1016B0004A14F6A8742AC896154BA9F7B6E80A5436
:1016C000D7896B35436F6E6E65637465642E004316
:1016D0006F6E6E2E2061626F727465640020002D43
:1016E0003E00436F6E76657274696E6720005361C9
:1016F0007665643A0020537566663A002041543A94
:1017000000206973200044656C6574696E6720630E
:101710006F6E662E2052414D207761733A005374EC
:101720006F707065640053746F7070696E672063CA
:1017300068616E6E656C73202E2E2E00556E6C6F78
:10174000636B696E6720636F6E666967202E2E2E4D
:1017500000536B697070696E672E2E004F75744F61
:10176000664D656D6F727921005D20000A5B003A5D
:10177000004D41433A004C6F61646564006C6F61D9
:1017800064206661696C6564004E6F2073746F72CB
:10179000656420636F6E666967004C6F6164696E93
:1017A0006720436F6E6669672066726F6D204545DE
:1017B00050524F4D000A72657175657374204D511A
:1017C000545420436F6E66696700536176656420E8
:1017D000746F20454550524F4D00536176696E67D6
:1017E00020636F6E66696720746F20454550524FC5
:1017F0004D2E2E0053617665640A00536574206493
:10180000796E616D69632049500A00454550524F19
:101810004D20636C65617265640A00506173737773
:101820006F726420757064617465640A00636F751B
:101830006C64206E6F742070617273653A2000557D
:101840007064617465640A002B002D004854545084
:101850002F312E312025690020485454502F312E2D
:10186000310D0A486F73743A2025730D0A41636382
:101870006570743A202A2F2A0D0A436F6E6E6563D5
:1018800074696F6E3A20636C6F73650D0A0025737F
:101890000020000D0A00474554006661696C6564CC
:1018A00020746F20636F6E6E6563740A0045525238
:1018B0004F523A2053657276657220726574757264
:1018C0006E65642000446F6E652E0A004170706C76
:1018D00079696E672E0A00436F6E666967207061D2
:1018E0007273696E67206661696C65640A00676F70
:1018F0007420436F6E6669670A00436F6E6669679E
:10190000205552493A20687474703A2F2F002044B1
:10191000656661756C7420636F6E666967207365B8
:101920007276657220757365643A20006C617A790D
:10193000686F6D652E727500205361766564000ACC
:10194000282D295359534C4F47000A282B29504919
:1019500044000A282D294D43503233303137000AD4
:10196000282D294152544E4554000A282D294F5400
:1019700041000A282B29535049204C4544000A288D
:101980002B294D4F544F5220435452000A282B29E3
:101990004143204841494552000A282B29434353DB
:1019A00038313120262048444331303830000A286D
:1019B0002D29524553544152545F4C414E5F4F4E76
:1019C0005F4D5154545F4552524F5253000A282DD7
:1019D000294841524452455345542C207573696E31
:1019E0006720736F6674000A282D29434F554E54A3
:1019F0004552000A282D29444854000A282B294F13
:101A000057495245000A282B294D4F44425553004F
:101A10000A282B294144414652554954204C4544FB
:101A2000000A282B29444D58000A282B2957697A87
:101A30006E657435313030000A282B294453323416
:101A400038322D313030000A282D29467265655212
:101A5000616D207072696E74696E670064653A61C9
:101A6000643A62653A65663A66653A3037000A4616
:101A700069726D77617265204D41432041646472E3
:101A800065737320006C617A79686F6D652E72756D
:101A9000000A436F6E666967207365727665723AF5
:101AA000000A282B295741544348444F47000A282D
:101AB0002B29434F4E54524F4C4C494E4F0032301D
:101AC000313130334C0020432B2B20766572736903
:101AD0006F6E3A00303437346330615F3230323108
:101AE0002D30342D3032000A4C617A79686F6D6583
:101AF0002E7275204C6967687448756220636F6E3A
:101B000074726F6C6C65722000444D582D4F757463
:101B100020496E697400444D582D4F7574207374BC
:101B20006F700041737369676E65643A00444D5885
:101B3000206374726C3A200044656661756C742091
:101B400073657269616C206D6F6465204E38312059
:101B50007573656400384531002600384E31000643
:101B600000384532002E00384E32000E00384F311A
:101B7000003600384F32003E003745310024003730
:101B80004E31000400374532002C00374E32000C35
:101B900000374F31003400374F32003C00203D3ECB
:101BA000004D6F646275732074656D706C6174654F
:101BB000206E6F7420666F756E643A2000496E76F1
:101BC000616C69642074656D706C6174652E002CA5
:101BD000002C002C002C004D4255533A20636F6EB0
:101BE000666967206661696C65643A004D6F64627E
:101BF000757320636F6E666967206572726F72001D
:101C00004D6F6462757320636F6E666967206C6FD9
:101C10006164656420004D4255533A204F7574202D
:101C20006F66206D656D6F7279004D4255533A2095
:101C3000506F6C6C696E67206572726F7220004E17
:101C40006F7420737570706F72746564207265674D
:101C500020747970650A00656E64506F6C6C2000AA
:101C60002D2D2D00506F6C6C2000556E6B6E6F77B4
:101C70006E207375666669782000556E6B6E6F779F
:101C80006E20636D642000466F7263656420657822
:101C900065637574696F6E003D004C45474143595B
:101CA00020494E3A0076616C0074656D7000736176
:101CB00074006875650066616E00524742004853C3
:101CC00056006D6F646500536574436D643A00534C
:101CD0006574466C61673A00436C72466C61673AA2
:101CE0000053746F726564204558543A00737566EA
:101CF000666978436F64653A00204F464600204F7E
:101D00004E00757074696D65006672656568656121
:101D10007000247374617473002045787069726573
:101D2000640A00202D746172676574207A6F6E6595
:101D30002D0020416C61726D204578706972656478
:101D40000A0020636D643A00204375723A00205304
:101D500065743A0063637338313120697320616CB4
:101D6000726561647920696E697469616C697A650C
:101D700064006864633130383020697320616C72AC
:101D80006561647920696E697469616C697A6564FA
:101D90000048444331303830206E6F7420696E69DA
:101DA0007469616C697A6564004E6F742073757034
:101DB000706F727465642072656720747970650A4B
:101DC00000293A0028543A003D3E002D3E0057724B
:101DD0006F6E672041737369676E6D656E74200066
:101DE000524742783A200020764C6576656C3A007E
:101DF00020436F6E76563A0020436F6E76533A005A
:101E000020486F743A00436F6C643A0020436F6E51
:101E100076657274656420563A00436F6E7665721B
:101E200074656420533A002D3E0057726F6E672030
:101E300041737369676E6D656E7420002D3E0057A7
:101E4000726F6E672041737369676E6D656E742083
:101E500000556E6B6E6F776E2073756666697820BD
:101E600000556E6B6E6F776E20636D642000636C3F
:101E7000724374723A20002F00496E3A20003E3EB1
:101E80002000496E76616C696420636F6D6D616ED0
:101E9000640000002200250028002B002E003100E5
:101EA000340002010000050108010B0100000A0BCB
:101EB00002090C0D0E0807030401000000000000D9
:101EC0000000000000000000000000000000000012
:101ED00000000000000000001211100000000000CF
:101EE00000000000000000000000000000000000F2
:101EF00000002C20002E003E3E3E004E6F204D4143
:101F00004320636F6E666967757265643A20736516
:101F100074206669726D776172652773204D414345
:101F20000A00556E6B6E6F776E2073756666697802
:101F30002000556E6B6E6F776E20636D64200053CA
:101F40006574706F696E743A00496E7075742076AE
:101F5000616C75653A0050574D2D4F757420496E70
:101F600069740050574D2D4F75742073746F700055
:101F70005247422050574D002050574D0052474283
:101F8000572050574D003D0050696E3A000075C60D
:101F900067C911241FBECFEFD1E2DEBFCDBF00E085
:101FA0000CBF1AE0A0E0B2E0EEEDF6EB01E00BBFF3
:101FB00002C007900D92A034B107D9F721E1A0E447
:101FC000BAE001C01D92AC3BB207E1F71FE0C8ECDC
:101FD000DFE000E006C021970109802FFE010E948A
:101FE000FBD6C73CD10780E00807A9F70E946DC95E
:101FF0000C945DDB0C9400004F925F926F927F9285
:102000008F929F92AF92BF92CF92DF92EF92FF9208
:102010000F931F93CF93DF93CDB7DEB7C25AD14052
:102020000FB6F894DEBF0FBECDBF20919410309153
:102030009510F9013B96EA31F10508F0D8C38827DD
:10204000EE58FF4F8F4F0C94FBD60AEE13E0CE569E
:10205000DE4F19830883C259D140CC56DE4F188217
:1020600019821A821B82C459D140CE57DE4F198380
:102070000883C258D140CC57DE4F188219821A8289
:102080001B82C458D140CE59DE4F19830883C256F3
:10209000D140CC59DE4F188219821A821B82C45655
:1020A000D140CE5BDE4F19830883C254D140CC5B54
:1020B000DE4F188219821A821B82C454D14061E318
:1020C0007AE08EE49EE00E9460B18EE49EE00E9481
:1020D00087B2BE016E567E4F86E090E00E94044DAE
:1020E000892B09F467C16BE17AE08EE49EE00E94DF
:1020F00060B11A830983CC56DE4F88819981AA8109
:10210000BB81C459D1408B839C83AD83BE83CE01F8
:1021100001960E94B8ACBE016E577E4F8AE090E0F7
:102120000E94044D892B09F42EC165E17AE08EE40A
:102130009EE00E9460B11A830983CC57DE4F8881EC
:102140009981AA81BB81C458D1408B839C83AD8384
:10215000BE83CE0101960E94B8ACBE016E597E4F7F
:102160008EE090E00E94044D892B09F4DFC060E10D
:102170007AE08EE49EE00E9460B11A830983CC5914
:10218000DE4F88819981AA81BB81C456D1408B835F
:102190009C83AD83BE83CE0101960E94B8ACBE0184
:1021A0006E5B7E4F82E190E00E94044D892B09F422
:1021B00077C069E07AE08EE49EE00E9460B11A8305
:1021C0000983CC5BDE4F88819981AA81BB81C4548D
:1021D000D1408B839C83AD83BE83CE0101960E9448
:1021E000B8AC1A830983CC5BDE4F88819981AA81C0
:1021F000BB81C454D1408B839C83AD83BE83CF57B6
:10220000DF4F19830883C158D040CC59DE4F8881F5
:102210009981AA81BB81C456D140CD57DF4F8883B5
:102220009983AA83BB83C358D040CE53DF4F198311
:102230000883C25CD040CC57DE4F88819981AA8147
:10224000BB81C458D140CC53DF4F88839983AA8384
:10225000BB83C45CD040CE5FDE4F19830883C2507D
:10226000D140CC56DE4F88819981AA81BB81C45967
:10227000D140CC5FDE4F88839983AA83BB83C4504F
:10228000D1409E012F5F3F4FAE014F575F4FBE01C0
:102290006E537F4FCE018E5F9E4F0E94E44B85C0F0
:1022A0001A830983CC59DE4F88819981AA81BB8129
:1022B000C456D1408B839C83AD83BE83CF57DF4F01
:1022C00019830883C158D040CC57DE4F888199814B
:1022D000AA81BB81C458D140CD57DF4F88839983F1
:1022E000AA83BB83C358D040CE53DF4F19830883E2
:1022F000C25CD040CC56DE4F88819981AA81BB81D7
:10230000C459D140CC53DF4F88839983AA83BB83C0
:10231000C45CD040AE014F5F5F4FBE016F577F4F2F
:10232000CE018E539F4F0E94304C3FC01A830983C9
:10233000CC57DE4F88819981AA81BB81C458D14096
:102340008B839C83AD83BE83CF57DF4F1983088374
:10235000C158D040CC56DE4F88819981AA81BB817B
:10236000C459D140CD57DF4F88839983AA83BB835B
:10237000C358D040BE016F5F7F4FCE018F579F4F34
:102380000E94824C12C01A830983CC56DE4F88818A
:102390009981AA81BB81C459D1408B839C83AD8331
:1023A000BE83CE0101960E94CD4C8EE49EE00E9439
:1023B00087B2F5C06DEF79E08EE49EE00E9460B1D7
:1023C0000FB6F894A89580916000886180936000B2
:1023D000109260000FBE80919F0A811107C084E8AF
:1023E0009AE00E94737981E080939F0A81E49AE0E9
:1023F0009093E10C8093E00C0E94464BCE01019635
:102400000E941DC689819A810E94B96B46E050E006
:1024100062E97BE089E090E00E9490B78AEE93E069
:102420009A8389831B821C821D821E82CE010396A1
:102430000E94A36B0E94B86B8091E00C9091E10C1C
:10244000DC0192961D921D921D921C929597FC01A3
:1024500016A217A210A611A69A961D921D921D9261
:102460001C929D9740EE5EE260E070E046AB57AB99
:1024700060AF71AF40EA5FE060E070E0DA964D93E4
:102480005D936D937C93DD973E9624E1DF011D9271
:102490002A95E9F726E0E2E9FBE0DC0118960190D5
:1024A0000D922A95E1F7FC01EE5BFF4F10820E942E
:1024B00064498C01019709F04AC0CE0101960E943F
:1024C0001DC689819A810E94B96B6091E00C709160
:1024D000E10C625F7F4FCE0101960E949FB2CE0158
:1024E00003960E94A36B6091E00C7091E10C6A5E10
:1024F0007F4FCE0101960E949FB2CE0103960E94AB
:10250000B16B6091E00C7091E10C6E5E7F4FCE017B
:1025100001960E949FB2CE0103960E94AA6B0E9470
:10252000B86B6091E00C7091E10C625E7F4FCE0160
:1025300001960E949FB28B819C81AD81BE81809368
:10254000DC0C9093DD0CA093DE0CB093DF0C99E2D1
:1025500088E10FB6F894A895809360000FBE909321
:102560006000A895012B69F46BEB79E086E59EE0AD
:102570000E9460B16CE879E086E59EE00E9460B15F
:1025800030C16CE779E08EE49EE00E9460B1CE013C
:1025900001960E940EADCE0101960E94B8AC82E079
:1025A00090E021C18091AB0A811103C081E080934A
:1025B000AB0A83E090E017C18091D70A811123C74D
:1025C0008091400A81110BC060E070E080E090E0F3
:1025D0000E946F8108C10E940AB8811108C184E07D
:1025E00090E001C1A895CE55DE4F1882C25AD14065
:1025F000FE01EE56FE4F119211928EE0DF011D9208
:102600008A95E9F70E940AB8882319F085E090E0DE
:10261000EAC00091CF0F1091D00F0115110509F4F8
:1026200044C2C8010E94C9B9E82EF12CB2E0EB16F1
:10263000F1040CF03DC239C20E9445A79B01AC01D8
:102640006091A70A7091A80A8091A90A9091AA0A9C
:10265000AA24AA94BA2C650118E8E12E13E1F12E00
:1026600000E010E00E941C3E882309F4C0C020E076
:1026700030E043E050E061E4CE0101960E94D23E9A
:1026800060E675E0CE0101960E9468DA00910E0DB9
:1026900010910F0DB801CE0101960E9449CE099606
:1026A0000817190790F10E940AB8882371F18091E8
:1026B000140D9091150D019611F481E090E0909326
:1026C000150D8093140DE0910C0DF0910D0D80917E
:1026D000150D8583E0910C0DF0910D0D8091140D79
:1026E000868360910C0D70910D0D47E050E0CE0196
:1026F00001960E9441B8AC014550510960910C0D02
:1027000070910D0D82EA0E9461B886E090E090938E
:102710009510809394106BE07CE08EE49EE00E9424
:1027200060B165C00E9445A76093A70A7093A80A8C
:102730008093A90A9093AA0A85EF9FEF54C00E9444
:1027400045A79B01AC016091A70A7091A80A8091EE
:10275000A90A9091AA0AAA24AA94BA2C650118E899
:10276000E12E13E1F12E00E010E00E941C3E8823D0
:1027700009F43DC0109295101092941038C00E9438
:102780000AB881110E943BAD0E9445A76093A70A39
:102790007093A80A8093A90A9093AA0A8DE090E00A
:1027A00022C00E9445A79B01AC016091A70A7091CD
:1027B000A80A8091A90A9091AA0AAA24AA94BA2CDC
:1027C000650110E1E12E17E2F12E00E010E00E9419
:1027D0001C3E811104CF0BC00E940681892B09F099
:1027E000FECE86EF9FEF90939510809394100FB6D6
:1027F000F894A895809160008861809360001092A1
:1028000060000FBE809194109091951002970CF487
:102810003DC10091E00C1091E10C0115110509F486
:1028200035C10E9445A74B015C017801FEE3EF0E24
:10283000F11CF70180819181A281B381A5019401EE
:10284000281B390B4A0B5B0BCA01B901683E33E008
:1028500073078105910508F446C028EE33E040E097
:1028600050E00E9484D6861A970AA80AB90AD701AE
:102870008D929D92AD92BC921397F80186A597A573
:10288000A0A9B1A969017A01CC0CDD1CEE1CFF1CCA
:102890008C159D05AE05BF0528F416A617A610AA2F
:1028A00011AA09C0821B930BA40BB50BF80186A7D4
:1028B00097A7A0ABB1ABF80182A993A9A4A9B5A928
:1028C0008C159D05AE05BF0528F412AA13AA14AAFB
:1028D00015AA09C0821B930BA40BB50BF80182ABA0
:1028E00093ABA4ABB5ABF80186A597A5A0A9B1A9F8
:1028F000892B8A2B8B2B69F4EE5BFF4F8081833011
:1029000041F484E08083C8010E94644901967C01FF
:1029100002C0E12CF12CF80182A993A9A4A9B5A9C0
:10292000892B8A2B8B2BA1F4EE5BFF4F80818330A8
:1029300011F081110DC01082F8013E9684E1DF0193
:102940001D928A95E9F7C8010E94644903967C01AB
:10295000B2E0EB16F10429F0E4E0EE16F10409F020
:102960004AC0CE0101960E941DC689819A810E94AB
:10297000B96B6091E00C7091E10C625F7F4FCE010A
:1029800001960E949FB2CE0103960E94A36B6091B4
:10299000E00C7091E10C6A5E7F4FCE0101960E94BF
:1029A0009FB2CE0103960E94B16B6091E00C7091D2
:1029B000E10C6E5E7F4FCE0101960E949FB2CE0168
:1029C00003960E94AA6B0E94B86B6091E00C709114
:1029D000E10C625E7F4FCE0101960E949FB28B8117
:1029E0009C81AD81BE818093DC0C9093DD0CA09323
:1029F000DE0CB093DF0CF3E0EF16F10461F15CF450
:102A000031E0E316F104D1F042E0E416F104F1F50F
:102A100061ED7BE02FC054E0E516F10449F185E05B
:102A2000E816F10499F562E07CE086E59EE00E94FC
:102A300060B186E59EE00E9487B206C06EEE7BE044
:102A400086E59EE00E9460B186EF9FEF909395101F
:102A5000809394101BC06EEB7BE086E59EE00E94A5
:102A600060B10E940AB8882379F30E943BADECCF95
:102A700062EA7BE08EE49EE00E9460B1CE010196A6
:102A80000E940EADCE0101960E94B8AC99E288E199
:102A90000FB6F894A895809360000FBE90936000E5
:102AA0002091941030919510AEC48EE090E09BCEB2
:102AB00060E070E0C8010E94E8708C019093D30A36
:102AC0008093D20A65E97BE08EE49EE00E9460B1CB
:102AD000B8018EE49EE00E949DB28EE49EE00E94CA
:102AE00087B262E97BE08BEF9EE00E9460B14AE032
:102AF00050E0B7018BEF9EE00E9480B28BEF9EE02A
:102B00000E9487B20091CF0F1091D00F61E070E06A
:102B1000C8010E94E8705C0192E0E916F10491F0AE
:102B200062E0C8010E9448B9FC01C184D284F3E08C
:102B3000EF16F10459F063E070E0C8010E94E870FC
:102B40008C0107C08BE5C82E87E0D82E8E010E556C
:102B50001E4F40E150E0BE016E567E4F86E390E08E
:102B60000E94C280892B51F425E0E216F1040CF09A
:102B70005FC3AE014E565E4F7A0104C0CE018E5641
:102B80009E4F7C01B092280DA092270DD0922A0D65
:102B9000C092290D83EB96E79093200D80931F0D33
:102BA00040E150E065E67BE0CE018E579E4F0E94EB
:102BB00036CE20E030E041E050E060E2CE018E59B8
:102BC0009E4F0E94D23E40E250E06EE57BE0CE0197
:102BD0008E599E4F0E9418CE6EE37BE08EE49EE0FD
:102BE0000E9460B1B5018EE49EE00E949DB26CE34C
:102BF0007BE08EE49EE00E9460B14AE050E0B601C6
:102C00008EE49EE00E9480B265E37BE08EE49EE06D
:102C10000E9460B1B8018EE49EE00E949DB260E324
:102C20007BE08EE49EE00E9460B1D8018C9181111E
:102C300004C0E12CF12C00E010E0A090D20AB0908A
:102C4000D30A0E940AB881117DC180910A0D90912A
:102C50000B0DDC01ED91FC910688F789E02D1995AB
:102C60008823A1F081E090E09093150D8093140DDE
:102C700087E0EAE3F2E0DE01119601900D928A9579
:102C8000E1F7FE01319685E090E037C06091270DB5
:102C90007091280D80910A0D90910B0D4091290D96
:102CA00050912A0DDC01ED91FC916115710521F027
:102CB0000088F189E02D16C00684F785E02D2AEE04
:102CC00033E03A8329834090230D5090240D609087
:102CD000250D7090260D4B825C826D827E82BE0136
:102CE0006F5F7F4F1995019709F4BCCF8EEF9FEF6F
:102CF00090932E0D80932D0DAFC22191A0910C0DBC
:102D0000B0910D0DA80FB91F2C9301968C30910531
:102D1000A1F70115110529F0E114F10421F086EF66
:102D200003C086E301C086EBC0900C0DD0900D0D62
:102D3000F60184878091110D85878091100D86871B
:102D400080900E0D90900F0DB401C5010E9449CEE8
:102D500041968816990608F4E9C04FE050E0B601A4
:102D6000C5010E9441B86C01A0900E0DB0900F0DEE
:102D7000B501CE018E599E4F0E9449CE8C0D9D1DEE
:102D80000296A816B90608F4D1C060910C0D709196
:102D90000D0DA601CE018E599E4F0E9441B86C01C7
:102DA000A0900E0DB0900F0DB501CE018E579E4F25
:102DB0000E9449CE8C0D9D1D0296A816B90608F4F6
:102DC000B5C060910C0D70910D0DA601CE018E570E
:102DD0009E4F0E9441B86C0101151105B9F1A090F8
:102DE0000E0DB0900F0DB501C8010E9449CE96019D
:102DF0002E5F3F4F820F931FA816B90608F496C0A6
:102E000060910C0D70910D0DA601C8010E9441B892
:102E10006C01E114F104D1F000910E0D10910F0D31
:102E2000B801C7010E9449CE96012E5F3F4F820F25
:102E3000931F0817190708F479C060910C0D709161
:102E40000D0DA601C7010E9441B86C01A6014550B5
:102E5000510960910C0D70910D0D80E10E9461B8D7
:102E60000E9445A76093160D7093170D8093180D5F
:102E70009093190D60931A0D70931B0D80931C0D88
:102E800090931D0D80910A0D90910B0DDC01ED9139
:102E9000FC910084F185E02D1995892B01F50E94A4
:102EA00045A72091120D3091130DC0901A0DD090AE
:102EB0001B0DE0901C0DF0901D0D4B015C018C185A
:102EC0009D08AE08BF08A8EEB3E00E94D8D68616CB
:102ED0009706A806B906B0F28CEF9FEF23C0CE018B
:102EE0008F579F4F0E94D1A96430710581059105CC
:102EF000E9F4E0910C0DF0910D0D8381811111C069
:102F00000E9445A760931A0D70931B0D80931C0DB2
:102F100090931D0D10921E0D10922E0D10922D0DDE
:102F200011C090E090932E0D80932D0D80910A0D8D
:102F300090910B0DDC01ED91FC910488F589E02D59
:102F400019958AC10091D20A1091D30A62E27BE0FE
:102F50008EE49EE00E9460B1B8018EE49EE00E9483
:102F60009DB28EE49EE00E9487B281E08093400A89
:102F700020E030E043E050E061E4CE018F579F4F06
:102F80000E94D23E60E675E0CE018F579F4F0E94AF
:102F900068DACE018F579F4F0E94F14A20E030E05F
:102FA00042E050E061E4CE018F579F4F0E94D23E35
:102FB00064E675E0CE018F579F4F0E9468DABE012C
:102FC0006F577F4F8EE59EE00E942846CE018F57B7
:102FD0009F4F0E94F14A20E030E041E050E061E480
:102FE000CE018F579F4F0E94D23E64E675E0CE011E
:102FF0008F579F4F0E9468DABE016F577F4F8EE553
:103000009EE00E942846CE018F579F4F0E94F14AB2
:10301000FE01EE5FFE4F119211921EE3DF01812E41
:103020001D928A94E9F71A821982FE0133968EE77F
:10303000DF011D928A95E9F720E030E041E050E0A1
:1030400060E4CE018E5F9E4F0E94D23E40E450E08D
:103050006EE57BE0CE018E5F9E4F0E9418CE40E869
:1030600050E06BED7AE0CE0101960E9436CEBE01B3
:103070006F5F7F4FCE018E5F9E4F0E942CB920E084
:1030800030E041E050E060E4CE018E5F9E4F0E9450
:10309000D23E40E450E065ED7AE0CE018E5F9E4F77
:1030A0000E9418CE40E850E06BEC7AE0CE01019629
:1030B0000E9436CE40E850E068EB7AE0CE010196FF
:1030C0000E9418CEBE016F5F7F4FCE018E5F9E4F74
:1030D0000E942CB920E030E041E050E060E4CE01F5
:1030E0008E5F9E4F0E94D23E40E450E062E17DE15F
:1030F000CE018E5F9E4F0E9418CE40E850E068EAF5
:103100007AE0CE0101960E9436CEBE016F5F7F4FFE
:10311000CE018E5F9E4F0E942CB920E030E041E04E
:1031200050E060E4CE018E5F9E4F0E94D23E40E4AC
:1031300050E061EA7AE0CE018E5F9E4F0E9418CE89
:1031400040E850E06BE97AE0CE0101960E9436CE6D
:10315000BE016F5F7F4FCE018E5F9E4F0E942CB9E4
:103160008091D70A8F5F8093D70AA0919610B09173
:103170009710109709F444C0809141029091420247
:10318000AE014E5B5E4FFA01819391932EE1119255
:103190002A95E9F79E012E533F4FF90181939193B0
:1031A00011921A95E9F716960D911C911797E090D8
:1031B0009610F0909710E114F10479F001151105C3
:1031C00061F0D80118968C918F708530A1F7C801F5
:1031D0000E94C9B9882379F367C020E030E041E05C
:1031E00050E060E4CE018E5F9E4F0E94D23E40E4EC
:1031F00050E06EE37AE0CE018E5F9E4F0E9418CEC3
:103200008091D70A81508093D70A85E090E090930F
:103210009510809394100E9445A76093A70A70931D
:10322000A80A8093A90A9093AA0A65E07BE075CA70
:1032300064E070E08091CF0F9091D00F0E94E87011
:103240007C0162E77BE08EE49EE00E9460B18EE448
:103250009EE00E9487B296CC00912D0D10912E0D0C
:1032600069EF7AE086E59EE00E9460B14AE050E0B6
:10327000B80186E59EE00E9480B261EE7AE086E5C4
:103280009EE00E9460B186E59EE00E9487B20E94A7
:1032900045A76093A70A7093A80A8093A90A909300
:1032A000AA0A8CE090E09FCA60E0C8010E9448B979
:1032B000FC0181859285A385B4858A30910508F447
:1032C00063C020E030E041E050E060E4CE018E5F7A
:1032D0009E4F0E94D23EF8016081718140E450E02F
:1032E000CE018E5F9E4F0E948EDA66E675E0CE01BB
:1032F0008E5F9E4F0E9468DA40E450E06DE47AE011
:10330000CE018E5F9E4F0E9418CEBE016E5B7E4F37
:10331000CE018E5F9E4F0E942CB9CE53DF4F888125
:10332000C25CD040882361F120E030E041E050E011
:1033300060E4CE018E5F9E4F0E94D23ED8016D9117
:103340007C9140E450E0CE018E5F9E4F0E948EDA69
:1033500066E675E0CE018E5F9E4F0E9468DA40E41B
:1033600050E065E47AE0CE018E5F9E4F0E9418CE59
:10337000BE016E537F4FCE018E5F9E4F0E942CB9CF
:10338000F8010281138113CFFC0140E250E088274D
:10339000E457FF4F8F4F0C94FBD665E97AE0CE01DE
:1033A0008E5B9E4F0E9436CECE53DF4F1882C25C9A
:1033B000D04087CF60E97AE0CE018E5B9E4F0E94BD
:1033C00036CE40E450E06FE67AE017C069E67AE076
:1033D000CE018E5B9E4F0E9436CE40E450E065E603
:1033E0007AE00BC06DE57AE0CE018E5B9E4F0E94C5
:1033F00036CE40E450E067E57AE0CE018E539F4F31
:103400000E9436CE5ECFC901CE55DE4F0FB6F8947E
:10341000DEBF0FBECDBFDF91CF911F910F91FF9007
:10342000EF90DF90CF90BF90AF909F908F907F9064
:103430006F905F904F9008952F923F924F925F92BE
:103440006F927F928F929F92AF92BF92CF92DF92B4
:10345000EF92FF920F931F93CF93DF93CDB7DEB719
:10346000C55DD1090FB6F894DEBF0FBECDBF5C01BC
:10347000C853DF4F0883C85CD040C753DF4F188361
:10348000C95CD040822FC653DF4F2883CA5CD0402E
:10349000C553DF4F3883CB5CD040C453DF4F4883E4
:1034A000CC5CD040C353DF4F5883CD5CD040C25377
:1034B000DF4F6883CE5CD040C153DF4F7883CF5C51
:1034C000D040C053DF4FF982E882C05DD0408F709A
:1034D000C82ED12C2090941030909510EE2DFF2DF9
:1034E000309719F08081811121C0D5011B968C91F4
:1034F000882341F0C5010B96C053DF4F9983888321
:10350000C05DD040C114D10409F055C0C053DF4F95
:10351000E881F981C05DD040309761F4F501C5883C
:10352000D688C114D10409F446C010C0C114D10416
:1035300009F041C08081882389F3CE0180539F4FD9
:103540000E940D8A6C01892B49F335C0C653DF4FA9
:103550008881CA5CD0408F7071F56C2DCE01885384
:103560009F4F0E944B74C854DF4F2883C85BD040E4
:10357000C754DF4F3883C95BD040C654DF4F488300
:10358000CA5BD040C554DF4F5883CB5BD040C45496
:10359000DF4F6883CC5BD040C354DF4F7883CD5B73
:1035A000D040C254DF4F8883CE5BD040C154DF4F40
:1035B0009883CF5BD0400E94C33F2B013C018B011D
:1035C000C053DF4FE880F980C05DD040D501ED9158
:1035D000FC918080918062E27DE08BEF9EE00E9412
:1035E00060B14AE050E0B2018BEF9EE00E9480B2F1
:1035F0006BE17DE08BEF9EE00E9460B1B4018BEF48
:103600009EE00E949DB265E17DE08BEF9EE00E940E
:1036100060B1B7018BEF9EE00E949DB26FE07DE04C
:103620008BEF9EE00E9460B16CE07DE08BEF9EE04E
:103630000E9460B1043B11054CF46EEF7CE086E51E
:103640009EE00E9460B186E59EE0AAC0CE0188534C
:103650009F4F0E940973F50180819181892B11F49C
:103660000C94A224C5010E943F634C0191E080E0CC
:10367000181419040CF090E0692E782E55245394F8
:10368000161417040CF0512C8BEF9EE00E9487B2A9
:10369000D50118968C91873009F486C0C053DF4F4E
:1036A000E880F980C05DD040E114F10409F45AC00B
:1036B0006AE475E1C7010E94FFCD892BD9F166E468
:1036C00075E1C7010E94FFCD892BB9F163E37CE06E
:1036D000C7010E94FFCD892B99F16FE27CE0C70101
:1036E0000E94FFCD892B79F16FE075E1C7010E943F
:1036F000FFCD892B59F16AE075E1C7010E94FFCD2A
:10370000892B39F164E175E1C7010E94FFCD892B56
:1037100019F166E27CE0C7010E94FFCD892BF9F028
:1037200062E27CE0C7010E94FFCD892BD9F40EE054
:1037300010E01AC001E010E017C002E010E014C071
:1037400005E010E011C006E010E00EC00AE010E055
:103750000BC00BE010E008C00CE010E005C00DE06D
:1037600010E002C000E010E0C5010E941F8C90E054
:10377000009709F03C0101151105B1F060167106C2
:1037800099F068EE7CE08BEF9EE00E9460B14AE029
:1037900050E0B3018BEF9EE00E9480B28BEF9EE081
:1037A0000E9487B20C94A224C054DF4F1882198261
:1037B0001A821B82C05CD040CC53DF4F1882198222
:1037C0001A821B82C45CD040CE53DF4F8881C25C1A
:1037D000D0408F70CE53DF4F8883C25CD040C0543E
:1037E000DF4F1882C05CD04040E0B501CE0180546C
:1037F0009F4F0E94B473811182C06BEC7CE08BEF11
:103800009EE00E9460B1F50181859285009741F0AC
:10381000DC01ED91FC91028CF38DE02D199503C034
:10382000F501808590E08D30910528F4FC01E85F7A
:10383000FA4F808101C080E08F70282F2295207F71
:10384000CE53DF4F9881C25CD0409F70922BCE53F5
:10385000DF4F9883C25CD040843028F48230C8F4B3
:10386000813069F133C0883039F0893079F580E0F2
:1038700090E0A6E9B2E404C080E090E0A0EAB1E400
:10388000CC53DF4F88839983AA83BB83C45CD04029
:1038900025C084E6CA53DF4F8883C65CD040C95335
:1038A000DF4F8881C75CD0408E7FC953DF4F88834C
:1038B000C75CD040CB53DF4F1882C55CD0408FEF40
:1038C000CC53DF4F8883C45CD04008C0CC53DF4F5B
:1038D000188219821A821B82C45CD04040E0B50174
:1038E000CE0180549F4F0E945C73CE0180549F4F45
:1038F0000E94097360E07AE0C5010E94565DC853DA
:10390000DF4F6881C85CD040643089F038F46623AA
:1039100009F457C3633009F49DC0BEC4673009F48D
:103920001AC108F4B9C46A3008F475C1B5C41814D2
:1039300019047CF562E0CE0180549F4F0E9473749D
:10394000C055DF4F2883C05BD040CF54DF4F388352
:10395000C15BD040CE54DF4F4883C25BD040CD54D2
:10396000DF4F5883C35BD040CC54DF4F6883C45BC8
:10397000D040CB54DF4F7883C55BD040CA54DF4F73
:103980008883C65BD040C954DF4F9883C75BD04063
:103990002EC061E0CE0180549F4F0E947374C855C1
:1039A000DF4F2883C85AD040C755DF4F3883C95AE4
:1039B000D040C655DF4F4883CA5AD040C555DF4F67
:1039C0005883CB5AD040C455DF4F6883CC5AD0407F
:1039D000C355DF4F7883CD5AD040C255DF4F88831F
:1039E000CE5AD040C155DF4F9883CF5AD040C054F3
:1039F000DF4F6881C05CD040CE0188539F4F0E944A
:103A00007374C056DF4F2883C05AD040CF55DF4F64
:103A10003883C15AD040CE55DF4F4883C25AD04078
:103A2000CD55DF4F5883C35AD040CC55DF4F688304
:103A3000C45AD040CB55DF4F7883C55AD040CA55C1
:103A4000DF4F8883C65AD040C955DF4F9883C75A85
:103A5000D0403DC4D50118968C91873009F439C403
:103A6000C5010E941F8C082F10E0853009F06CC73B
:103A70006CEB7CE08BEF9EE00E9460B14AE050E08E
:103A8000B8018BEF9EE00E9480B28BEF9EE00E9417
:103A900087B2F5018085853079F56CE0CE018054E0
:103AA0009F4F0E947374C856DF4F2883C859D04077
:103AB000C756DF4F3883C959D040C656DF4F4883B9
:103AC000CA59D040C556DF4F5883CB59D040C45651
:103AD000DF4F6883CC59D040C356DF4F7883CD5930
:103AE000D040C256DF4F8883CE59D040C156DF4FF9
:103AF0009883CF59D040EBC361E0CE0180549F4FF3
:103B00000E947374C057DF4F2883C059D040CF56EE
:103B1000DF4F3883C159D040CE56DF4F4883C2595A
:103B2000D040CD56DF4F5883C359D040CC56DF4FDD
:103B30006883C459D040CB56DF4F7883C559D040F5
:103B4000CA56DF4F8883C659D040C956DF4F988385
:103B5000C759D040BCC3D50118968C91873009F461
:103B6000B8C3C5010E941F8C082F10E0863009F0F1
:103B700040C06BEA7CE08BEF9EE00E9460B14AE0BF
:103B800050E0B8018BEF9EE00E9480B28BEF9EE088
:103B90000E9487B262E0CE0180549F4F0E947374EE
:103BA000C857DF4F2883C858D040C757DF4F3883E6
:103BB000C958D040C657DF4F4883CA58D040C55770
:103BC000DF4F5883CB58D040C457DF4F6883CC5861
:103BD000D040C357DF4F7883CD58D040C257DF4F16
:103BE0008883CE58D040C157DF4F9883CF58D040FC
:103BF0006EC363E97CE08BEF9EE00E9460B14AE017
:103C000050E0B8018BEF9EE00E9480B28BEF9EE007
:103C10000E9487B299C660E0CE0180549F4F0E94F7
:103C20007374C058DF4F2883C058D040CF57DF4F40
:103C30003883C158D040CE57DF4F4883C258D04058
:103C4000CD57DF4F5883C358D040CC57DF4F6883E0
:103C5000C458D040CB57DF4F7883C558D040CA579F
:103C6000DF4F8883C658D040C957DF4F9883C75865
:103C7000D040C653DF4F8881CA5CD040807F41F07E
:103C8000CE0188539F4F0E946A768B01672B11F4F7
:103C900005E010E0C853DF4F8881C85CD040893010
:103CA00019F4119501951109B2E0CB16D10499F0E0
:103CB0003CF4C114D10409F00CC3552453940BC037
:103CC000F9E0CF16D10409F49EC02AE0C216D1044F
:103CD00009F413C1FEC2CE53DF4F8881C25CD040CD
:103CE000E82FE295EF708E2F90E0FC013197EB30DA
:103CF000F10508F0EEC28827EA56FF4F8F4F0C946B
:103D0000FBD6CC53DF4F8881C45CD040080F111D17
:103D10000F3F110509F02CF417FF05C000E010E07B
:103D200002C00FEF10E0CC53DF4F0883C45CD040DB
:103D3000A6C2CC53DF4F68817981C45CD040060FA6
:103D4000171F053611052CF417FF05C000E010E021
:103D500002C004E610E0012E000C220B330BCC5302
:103D6000DF4F088319832A833B83C45CD04087C21A
:103D7000CC53DF4F688179818A819B81C45CD040BC
:103D80000E940CD8600F711F653671052CF477FF07
:103D900005C060E070E002C064E670E0072E000C31
:103DA000880B990B0E9441D5CC53DF4F68837983F0
:103DB0008A839B83C45CD04062C2CC53DF4F88812E
:103DC0009981C45CD0404AE0409F9001419F300DF2
:103DD0001124820F931F893EA3E09A072CF497FFCA
:103DE00005C080E090E002C088EE93E0092E000C50
:103DF000AA0BBB0BCC53DF4F88839983AA83BB8369
:103E0000C45CD0403CC2CE0188539F4F0E94A27632
:103E1000882301F162E0CE0180549F4F0E94E0743C
:103E2000E9962FAFE997EA963FAFEA97EB964FAF47
:103E3000EB97EC965FAFEC97ED966FAFED97EE9644
:103E40007FAFEE97EF968FAFEF97C158DF4F988314
:103E5000CF57D040CE53DF4F8881C25CD04082958F
:103E60008F70823009F035C2CA53DF4F6881C65C5B
:103E7000D040C953DF4F8881C75CD040782F717024
:103E8000060F171F0E36B1E01B072CF417FF05C0F5
:103E90000DE611E002C000E010E0CA53DF4F0883D6
:103EA000C65CD040C953DF4F8881C75CD04010FB4F
:103EB00080F9C953DF4F8883C75CD04062E0CE01F0
:103EC00080549F4F0E944B74E1962FAFE197E2968A
:103ED0003FAFE297E3964FAFE397E4965FAFE49787
:103EE000E5966FAFE597E6967FAFE697E7968FAFDB
:103EF000E797E8969FAFE897C2C1CE0188539F4FDE
:103F00000E94A2768823F1F062E0CE0180549F4F98
:103F10000E94E074A9962FAFA997AA963FAFAA97DF
:103F2000AB964FAFAB97AC965FAFAC97AD966FAF1C
:103F3000AD97AE967FAFAE97AF968FAFAF97E09647
:103F40009FAFE097CE53DF4F8881C25CD04082950F
:103F50008F70823009F0BDC1CB53DF4F8881C55CC3
:103F6000D040080F111D053611052CF417FF05C0B0
:103F700000E010E002C004E610E0CB53DF4F0883FE
:103F8000C55CD04062E0CE0180549F4F0E944B74CC
:103F9000A1962FAFA197A2963FAFA297A3964FAF3E
:103FA000A397A4965FAFA497A5966FAFA597A69683
:103FB0007FAFA697A7968FAFA797A8969FAFA89712
:103FC0005EC1C653DF4F8881CA5CD040807F09F450
:103FD00080C1E9E0CE16D10409F424C14CF4C11427
:103FE000D104F1F022E0C216D10409F45FC071C11E
:103FF0008BE0C816D10409F437C10CF4D0C0BCE082
:10400000CB16D10409F065C188E0FE01E853FF4FEB
:10401000DE01A054BF4F01900D928A95E1F759C17E
:10402000181419043CF5CE0188539F4F0E946A76FC
:10403000672B682B692B59F562E0CE0180549F4FA6
:104040000E94737469962FAF69976A963FAF6A971B
:104050006B964FAF6B976C965FAF6C976D966FAF2B
:104060006D976E967FAF6E976F968FAF6F97A09696
:104070009FAFA0971814190454F0CE0188539F4F96
:104080000E946A76672B682B692B09F063C4C054C1
:10409000DF4F6881C05CD040C5010E94F48B60E0B6
:1040A00079E0C5010E94565D55245394CE53DF4FED
:1040B0008881C25CD040982F92959F70945F9F70CA
:1040C000923050F4C653DF4F9881CA5CD04092952D
:1040D0009F70923009F45DC4F5011085173039F4F2
:1040E000CE0188539F4F0E94A27681115AC4D501F8
:1040F00019968D919C911A97009741F0DC01ED91F2
:10410000FC91028CF38DE02D199502C0812F90E077
:104110007C01C853DF4F0881C85CD040C753DF4FD4
:104120001881C95CD040C653DF4F2881CA5CD0409B
:10413000C553DF4F3881CB5CD040C453DF4F48813B
:10414000CC5CD040C353DF4F5881CD5CD040C253CC
:10415000DF4F6881CE5CD040C153DF4F7881CF5CA8
:10416000D040CE0180549F4F0E94969529962FAF44
:1041700029972A963FAF2A972B964FAF2B972C96CD
:104180005FAF2C972D966FAF2D972E967FAF2E9702
:104190002F968FAF2F9760969FAF609770C0C353D5
:1041A000DF4F9881CD5CD040CE53DF4F8881C25C19
:1041B000D040282F22952F7019F0223041F089C06D
:1041C0008F708062CE53DF4F8883C25CD040892FCE
:1041D00090E08536910514F084E690E0CB53DF4FF4
:1041E0008883C55CD04062E0CE0180549F4F0E941E
:1041F0004B7421962FAF219722963FAF229723969B
:104200004FAF239724965FAF249725966FAF2597DE
:1042100026967FAF269727968FAF279728969FAF32
:1042200028972DC0C253DF4F6881CE5CD040C15368
:10423000DF4F7881CF5CD0407170CE0180549F4FAA
:104240000E944C42882309F444C062E0CE018054AD
:104250009F4F0E944B7428AF39AF4AAF5BAF6CAF32
:104260007DAF8EAF9FAF0BC0CE0188539F4F0E9492
:104270006494BC01CE0180549F4F0E94869440E01C
:10428000B501CE0180549F4F0E945C7360E07AE0DC
:10429000C5010E94565D1DC0CE0180549F4F0E94F3
:1042A000737428AB39AB4AAB5BAB6CAB7DAB8EABFD
:1042B0009FAB6C2DCE0180549F4F0E944B7428A75A
:1042C00039A74AA75BA76CA77DA78EA79FA75524F0
:1042D0005394F501618472846114710409F43CC142
:1042E000C853DF4F8881C85CD04090E08A30910588
:1042F00008F0DCC0FC018827EF55FF4F8F4F0C946E
:10430000FBD61814190454F166E87CE08BEF9EE0AC
:104310000E9460B1D5011996ED91FC911A97019018
:10432000F081E02D84889588C053DF4FE880F980C4
:10433000C05DD04061E0CE0180549F4F0E947374F5
:10434000CC24C39489019A01AB01BC01F50181859C
:104350009285F40119958C0166E05BC066E77CE00C
:1043600063C0181419043CF5D301ED91FC918488C5
:104370009588C053DF4FE880F980C05DD04062E08F
:10438000CE0180549F4F0E947374CC24C394890142
:104390009A01AB01BC01F50181859285F401199563
:1043A0008C0165E0C5010E94F48B60E071E0C501FD
:1043B0000E94565DCFC064E67CE036C0C5010E9415
:1043C0001F8C853079F1D301ED91FC91848895881B
:1043D000C053DF4FE880F980C05DD04062E0CE017D
:1043E00080549F4F0E94737429833A834B835C836C
:1043F0006D837E838F839887CC24C39489019A012F
:10440000AB01BC01F50181859285F40119958C0100
:1044100062E0C5010E94F48B60E071E0C5010E947A
:10442000565D87C064E57CE08BEF9EE00E9460B142
:104430008BC2C053DF4FE880F980C05DD040D3010C
:10444000ED91FC910488F589E02DC52CC054DF4F17
:104450000881C05CD040CF53DF4F1881C15CD04091
:10446000CE53DF4F2881C25CD040CD53DF4F38811F
:10447000C35CD040CC53DF4F4881C45CD040CB53A9
:10448000DF4F5881C55CD040CA53DF4F6881C65C9E
:10449000D040C953DF4F7881C75CD040C301199524
:1044A0008C0147C0181419040CF441C0C053DF4FED
:1044B000E880F980C05DD040D301ED91FC91048883
:1044C000F589E02DCC24C394C054DF4F0881C05C33
:1044D000D040CF53DF4F1881C15CD040CE53DF4F67
:1044E0002881C25CD040CD53DF4F3881C35CD040BF
:1044F000CC53DF4F4881C45CD040CB53DF4F588151
:10450000C55CD040CA53DF4F6881C65CD040C953F8
:10451000DF4F7881C75CD040C30119958C01C0542E
:10452000DF4F6881C05CD040662319F072CF0FEF77
:104530001FEF68E47CE08BEF9EE00E9460B14AE0F0
:1045400050E0B8018BEF9EE00E9480B28BEF9EE0BE
:104550000E9487B2C80132C2F5018085863009F415
:1045600075C038F4843009F447C1853009F4D6C0E9
:10457000CEC1883009F49EC120F0893009F46BC1A6
:10458000C6C10280F381E02D80858F70853009F0EF
:10459000BEC1B5E02B16310409F4B9C1C680D7807D
:1045A0008091D70A8F5F8093D70AC114D10409F490
:1045B00047C0F60180858F708430E1F56185728592
:1045C000CE0101960E940D8DC053DF4FE880F98027
:1045D000C05DD040C853DF4F0881C85CD040C7538E
:1045E000DF4F1881C95CD040C653DF4F2881CA5CB9
:1045F000D040C553DF4F3881CB5CD040C453DF4F30
:104600004881CC5CD040C353DF4F5881CD5CD04053
:10461000C253DF4F6881CE5CD040C153DF4F7881F9
:10462000CF5CD040CE0101960E941C1ACE010196AB
:104630000E942C8CD6011296CD90DC901397B5CFAA
:104640008091D70A81508093D70A61C160E070E001
:10465000C5010E940A8B8C01009709F458C197FF8D
:1046600007C011950195110966246394712C02C04D
:10467000612C712CC80101978634910508F047C15F
:10468000C054DF4FE880C05CD040F12CD02E61E0F8
:10469000802F0E94C2A5672869F0B1E0EB16F104F3
:1046A00029F061E0E6E0EE16F10409F460E0E62EA0
:1046B000F12C12C0F1E0EF16F10451F091E080E02E
:1046C00026E0E216F10409F090E0E92EF82E03C08E
:1046D000EE24E394F12C6E2D8D2D0E9493A563E4BE
:1046E0007CE08BEF9EE00E9460B14AE050E0B801B0
:1046F0008BEF9EE00E9480B261E47CE08BEF9EE055
:104700000E9460B14AE050E0B7018BEF9EE00E944A
:1047100080B28BEF9EE00E9487B2F9C082E0C8169B
:10472000D10409F461C0ACE0CA16D10409F0EFC0AD
:10473000C5010E94EF8A6B017C01EF2849F4D50185
:10474000ED91FC916081718188E695E00E94304294
:10475000CE0180549F4F0E942C7620E030E048EC40
:1047600052E40E94A0D50E940CD8CE52DF4F68833D
:1047700079838A839B83C25DD040CE52DF4FC8804D
:10478000D980C25DD04088E00E94063E2B013C01EA
:104790007B016DE37CE08BEF9EE00E9460B14AE01C
:1047A00050E0CE52DF4F68817981C25DD0408BEFFF
:1047B0009EE00E9480B268E37CE08BEF9EE00E9466
:1047C00060B1B301A201662777272AE08BEF9EE054
:1047D0000E9499B18BEF9EE00E9487B2B701A601BB
:1047E000C5010E94918A93C040E0B501CE0180547A
:1047F0009F4F0E945C738BC0552009F488C0C05441
:10480000DF4F0881C05CD040CF53DF4F1881C15CBF
:10481000D040CE53DF4F2881C25CD040CD53DF4F14
:104820003881C35CD040CC53DF4F4881C45CD0405A
:10483000CB53DF4F5881C55CD040CA53DF4F6881EE
:10484000C65CD040C953DF4F7881C75CD040C501FA
:104850000E945A615CC0552009F459C0C054DF4F12
:104860000881C05CD040CF53DF4F1881C15CD0407D
:10487000CE53DF4F2881C25CD040CD53DF4F38810B
:10488000C35CD040CC53DF4F4881C45CD040CB5395
:10489000DF4F5881C55CD040CA53DF4F6881C65C8A
:1048A000D040C953DF4F7881C75CD040C5010E941A
:1048B0008A602DC0552059F1C054DF4F0881C05C7B
:1048C000D040CF53DF4F1881C15CD040CE53DF4F73
:1048D0002881C25CD040CD53DF4F3881C35CD040CB
:1048E000CC53DF4F4881C45CD040CB53DF4F58815D
:1048F000C55CD040CA53DF4F6881C65CD040C95305
:10490000DF4F7881C75CD040C5010E942862C05447
:10491000DF4F6881C05CD0406623C9F0C853DF4FC9
:104920008881C85CD040853021F4181419047CF4C7
:1049300065E0C5010E94F48B60E071E0C5010E9452
:10494000565D05C08FEF01C08DEF9FEF37C081E04E
:1049500090E034C061E0CE0180549F4F0E94737498
:1049600061962FAF619762963FAF629763964FAFA4
:10497000639764965FAF649765966FAF6597669629
:104980007FAF669767968FAF679768969FAF689778
:104990007ECB8F708062CE53DF4F8883C25CD04065
:1049A0009BCBCE53DF4F9881C25CD0409F7090620A
:1049B000CE53DF4F9883C25CD04099CBCB52DF4FB0
:1049C0000FB6F894DEBF0FBECDBFDF91CF911F9120
:1049D0000F91FF90EF90DF90CF90BF90AF909F909E
:1049E0008F907F906F905F904F903F902F900895A1
:1049F000089583E090E008958091AC0A9091AD0A0B
:104A000008952F923F924F925F926F927F928F9272
:104A10009F92AF92BF92CF92DF92EF92FF920F934D
:104A20001F93CF93DF93CDB7DEB72E970FB6F894D1
:104A3000DEBF0FBECDBF1C010E949C9CD10114960D
:104A40008D919C911597892B79F484E190E00E94D7
:104A500008CBBC01F101828193810E944F8AD10170
:104A600015969C938E931497F1010480F581E02DA7
:104A7000FA87E987EF2B59F462EC7DE086E59EE04A
:104A80000E9460B186E59EE00E9487B2E8C2A985D7
:104A9000BA851D921C92F1010280F381E02DFE8700
:104AA000ED8702811381EF2B09F460C20115110516
:104AB00009F45CC2D80118968C918F70853009F08A
:104AC00055C2C8010E94C9B9882309F44FC260E0E9
:104AD000C8010E9448B98C01FC0180858F70853027
:104AE00039F069E67DE086E59EE00E9460B1A0C2F3
:104AF000C8010E94C9B9823031F148F4813009F00F
:104B00006BC0C12CD12C7601460157013BC08630C9
:104B100008F062C062E0C8010E9448B9FC019085BB
:104B20009F70933029F4C184D284E384F4840EC04E
:104B3000923049F461857285838594850E9441D5C0
:104B40006B017C0103C0C12CD12C760161E0C8014E
:104B50000E9448B9FC0190859F70933029F48184AC
:104B60009284A384B4840EC0923049F46185728526
:104B7000838594850E9441D54B015C0103C0812C43
:104B8000912C540160E0C8010E9448B9FC01908555
:104B90009F70933029F441845284638474840AC0E2
:104BA000923021F561857285838594850E9441D577
:104BB0002B013C0120E030E0A901C301B2010E94B9
:104BC0003AD587FF19C077FA709477F87094E1E0CE
:104BD000F0E0FC87EB8712C01C861B86C12CD12C11
:104BE0007601460157012601370108C01C861B8645
:104BF000412C512C320102C01C861B86AD85BE851E
:104C00001496ED91FC91159780858295807F85950E
:104C1000859585958595823039F0833091F481852D
:104C20009285A385B48511C061857285838594853D
:104C30000E9441D5E985FA856287738784879587C5
:104C40000AC080E090E0A0EAB1E4E985FA858287B5
:104C50009387A487B5878CE390E00E9408CB8C01F2
:104C600089859A850296D8015F969C938E935E976C
:104C700089859A8506965D969C938E935C97898527
:104C80009A850A9691969C938E939097DA961C92A9
:104C9000F80112AA13AA14AA15AA80E090E0AFE7BF
:104CA000B3E486AB97ABA0AFB1AF84E690E0A0E0F1
:104CB000B0E086A797A7A0ABB1AB8B859C85918F01
:104CC000808F20E030E0A901C301B2010E943AD5F3
:104CD00087FD7DC020E030E0A901C501B4010E943C
:104CE0003AD587FD74C020E030E0A901C701B601C4
:104CF0000E943AD587FD6BC081E090E0D8015B96B9
:104D00009C938E935A97DB968C93DB97F8014082A5
:104D100051826282738214968D929D92AD92BC9262
:104D20001797C086D186E286F3861C964D925D92D7
:104D30006D927C921F972DEC3CEC4CEC5DE3C50131
:104D4000B4010E94A0D54B015C01F801608B718B0E
:104D5000828B938B2DEC3CEC4CEC5DE3C701B601F0
:104D60000E949AD76B017C01D80154966D937D9374
:104D70008D939C935797EB85FC85319741F5A30163
:104D8000920160E070E0CB010E942DD7D8011C9603
:104D90006D937D938D939C931F97A501940160E083
:104DA00070E0CB010E942DD7F801608B718B828B54
:104DB000938BA701960160E070E0CB010E942DD794
:104DC000D80154966D937D938D939C9357970E9431
:104DD00045A7F80186A497A4A0A8B1A8DC01CB013F
:104DE00088199909AA09BB0982A393A3A4A3B5A30F
:104DF000D1011496ED91FC91159711830083011553
:104E0000110509F419C1F80182AD81113BC0068C6E
:104E1000F78DE02DC080D180E280F380D801969696
:104E2000CD92DD92ED92FC9299975C96ED91FC917A
:104E30005D9780819181A281B381F80182A793A7B8
:104E4000A4A7B5A746A857A860AC71ACA30192016E
:104E5000C701B6010E9442D818166CF0F80142A8AA
:104E600053A864A875A8A3019201C701B6010E94C6
:104E70003AD587FF07C0D80196964D925D926D9204
:104E80007C92999781E0F80182AFC501B4010E943C
:104E90003FD59B01AC0160E070E48CE995E40E9491
:104EA0009AD76B017C019B01AC01D80150966D91A2
:104EB0007D918D919C9153970E94A0D5F801608BB4
:104EC000718B828B938BA701960164897589868982
:104ED00097890E949AD7D80154966D937D938D93AC
:104EE0009C93579788E893E1A0E0B0E0F80186A78B
:104EF00097A7A0ABB1ABD1011296ED91FC9113979E
:104F00000190F081E02D008111816EE97DE08EE459
:104F10009EE00E9460B1B8018EE49EE00E949DB2C6
:104F20008EE49EE00E9487B2F10182819381198212
:104F30001A821B821C821D821E821F8218862B8170
:104F40002F70E12CF12C01E01A813C8140E05E8160
:104F50006F8178850E941C1AD1011496ED91FC9105
:104F6000159781E090E0938B828B7BC0C8010E94F3
:104F7000C9B9E82ED80118968C918F70FF24F3944C
:104F8000853009F4F12C6AE87DE086E59EE00E9418
:104F900060B14AE050E061E070E086E59EE00E948A
:104FA00080B268E87DE086E59EE00E9460B161E045
:104FB00070E0ED85FE85EF2B11F460E070E04AE0D3
:104FC00050E086E59EE00E9480B266E87DE086E5DE
:104FD0009EE00E9460B161E070E0012B11F460E09E
:104FE00070E04AE050E086E59EE00E9480B264E80E
:104FF0007DE086E59EE00E9460B16F2D70E04AE0A2
:1050000050E086E59EE00E9480B262E87DE086E5A1
:105010009EE00E9460B161E070E0F1E0FE1510F4E6
:1050200060E070E04AE050E086E59EE00E9480B2D9
:1050300086E59EE00E9487B261EB7DE086E59EE01A
:105040000E9460B186E59EE00E9487B2D10114966D
:10505000ED91FC91159782E090E0938B828B80E03C
:1050600090E02E960FB6F894DEBF0FBECDBFDF9155
:10507000CF911F910F91FF90EF90DF90CF90BF9055
:10508000AF909F908F907F906F905F904F903F90E8
:105090002F9008950C94A0CBCF92DF92EF92FF92C5
:1050A0000F931F93CF93DF93CDB7DEB728970FB63B
:1050B000F894DEBF0FBECDBF6C01822F2B838F70A3
:1050C000E82EF12C002331F0E114F10419F4EE2460
:1050D000E394F12C60E070E1F601828193810E94FB
:1050E000A58BF1E0EF16F10481F082E0E816F104FF
:1050F00041F0EF2851F568E57DE08BEF9EE00E94DE
:1051000060B18B81807F59F10AC0602FF6018281E6
:1051100093810E94F48B013011F00230B1F4F6015A
:10512000828193810E94EF8A672B682B692B51F053
:1051300080E00E94063EAB01BC01F60182819381B2
:105140000E94918A81E090E00CC06CE47DE08BEFDE
:105150009EE00E9460B18BEF9EE00E9487B280E0EB
:1051600090E028960FB6F894DEBF0FBECDBFDF915A
:10517000CF911F910F91FF90EF90DF90CF90089506
:10518000CF93DF93EC0167E775E08EE59EE00E9428
:1051900028466D858C810E9493A56D858D810E9426
:1051A00093A540E050E0BA018A819B810E94918AD8
:1051B0001092AD0A1092AC0A81E090E0DF91CF919D
:1051C00008952F923F924F925F926F927F928F92AB
:1051D0009F92AF92BF92CF92DF92EF92FF920F9386
:1051E0001F93CF93DF93CDB7DEB760970FB6F894D8
:1051F000DEBF0FBECDBF4C01FC01E280F38060E05A
:1052000070E1C7010E94DD8B892B09F46EC260E05A
:1052100070E2C7010E94DD8B892B79F48091000236
:10522000882309F462C260E070E2C7010E94A58B86
:1052300080910002815080930002F401E280F380AB
:10524000C7010E94EF8A2B013C0119821A821B823E
:105250001C821D821E821F8218868B818F708B8319
:10526000198240E0B701CE0101960E94B47360E05C
:10527000CE0101960E9469759A878987F40182811F
:1052800093810E941F8C823011F0853011F41A86B0
:105290001986F40186819AEC980F9031B0F521853A
:1052A0003285A90160E070E04D875E876F87788B5B
:1052B000C384D484E12CF12C0E94C7A69C878B87E1
:1052C000092E000CAA0BBB0B9C01AD012C193D094A
:1052D0004E095F09AFEFB0E00E94C5D62D853E852F
:1052E0004F8558892C193D094E095F090E94A6D6A1
:1052F000190137FDF2C15FEF2516310409F00CF4F6
:10530000EEC122242A94312CEAC1411451046104D3
:10531000710409F4D5C16FEF7FEF7C876B8722247E
:105320002A94322CF401878190859C01990F440BBB
:10533000550B2D873E874F87588B0E9445A79B01B1
:10534000AC01AA24AA94BA2C6501ED84FE840F85D1
:105350001889C301B2010E941C3E882309F4A7C129
:105360006EE37DE08BEF9EE00E9460B18BEF9EE0EC
:105370000E9487B2E12CF12CF40116816AE37DE0F2
:105380008BEF9EE00E9460B1612F110F770B4AE016
:1053900050E08BEF9EE00E9480B264E37DE08BEFF3
:1053A0009EE00E9460B14AE050E06B857C858BEF07
:1053B0009EE00E9480B262E37DE08BEF9EE00E945F
:1053C00060B14AE050E0B1018BEF9EE00E9480B2F4
:1053D0006FE27DE08BEF9EE00E9460B14AE050E01A
:1053E00069857A858BEF9EE00E9480B267E27DE05E
:1053F0008BEF9EE00E9460B14AE050E0B7018BEF76
:105400009EE00E9480B28BEF9EE00E9487B2F6EF92
:10541000EF16FFEFFF060CF080C0F4016585858173
:105420000E9493A5F401828193810E94EF8A672BE9
:10543000682B692B51F480E00E94063EAB01BC0151
:10544000F401828193810E94918AF40114818EEF8C
:10545000810F65858C3020F084ED810F8330C8F496
:10546000AA27BB27AE19BF09662351F09D01A1E011
:10547000BFEF0E940AD729E130E040E050E080C051
:105480002FEF30E00E9412D729E130E040E050E0F9
:105490008AC0F40185819EEF980F9C3020F08C52D9
:1054A000833008F0D2C081E06827812F0E9493A545
:1054B000F4018585AA27BB27AE19BF09882359F0B7
:1054C0002FEF30E00E9412D729E130E040E050E0B9
:1054D0000E94A6D612C09D01A1E0BFEF0E940AD78C
:1054E00029E130E040E050E00E94A6D6DA01C9018F
:1054F00081509F4FAF4FBF4F9C012634310544F080
:10550000B9012F3F310531F02CF06FEF70E002C090
:1055100066E470E0F401858195C0FBE0EF16F104CC
:105520000CF499C0F401658584810E9493A5F4016F
:10553000828193810E94EF8A672B682B692B51F43B
:1055400080E00E94063EAB01BC01F40182819381A0
:105550000E94918AF40115818EEF810F65858C3050
:1055600020F084ED810F833078F5662399F0970160
:10557000A1E0BFEF0E940AD723E330E040E050E013
:105580000E94A6D6DA01C90181509F4FAF4FBF4F8D
:105590009C010BC02FEF30E0D7010E9412D723E30C
:1055A00030E040E050E00E94A6D62634310544F0B9
:1055B000B9012F3F310531F02CF06FEF70E002C0E0
:1055C00066E470E0812F3EC0F40184819EEF980F65
:1055D0009C3018F08C528330C0F581E06827812F11
:1055E0000E9493A5F4018585882369F02FEF30E0B0
:1055F000D7010E9412D729E130E040E050E00E943C
:10560000A6D6B90112C09701A1E0BFEF0E940AD748
:1056100029E130E040E050E00E94A6D6DA01C9015D
:1056200081509F4FAF4FBF4FBC016F3F710509F0D5
:105630002CF477FF05C060E070E002C06FEF70E00F
:10564000F40184810E94FEA550C081E06827812F6B
:105650000E9493A54AC065E875E08EE59EE00E9431
:105660002846F401658584810E9493A5F40165852F
:1056700085810E9493A540E050E0BA01F401828147
:1056800093810E94918A60E070E1F40182819381AC
:105690000E946B8B60E070E2F401828193810E9432
:1056A0006B8B809100028F5F809300021EC0FFEF22
:1056B0002F163F0649F0E984FA84E218F3085CCE1D
:1056C0002FEF3FEF3C872B87E984FA843FE7E31A0B
:1056D000F10822242A94322C4FCE212C312C411453
:1056E00051046104710439F31DCE80E090E06096AE
:1056F0000FB6F894DEBF0FBECDBFDF91CF911F91E3
:105700000F91FF90EF90DF90CF90BF90AF909F9060
:105710008F907F906F905F904F903F902F90089563
:105720000895FC01838594859C0144E03595279577
:105730004A95E1F756E0959587955A95E1F7281730
:10574000390719F081E090E0089582E090E0089533
:1057500080E090E008958091B60A9091B70A08958C
:105760000C94A0CB2F923F924F925F926F927F92B8
:105770008F929F92AF92BF92CF92DF92EF92FF9261
:105780000F931F93CF93DF93CDB7DEB7AF970FB6CD
:10579000F894DEBF0FBECDBF5C010E8F1F8F28A314
:1057A00039A34AA35BA36CA37DA3CFA61C8A1B8A43
:1057B000DC0118968D919C91199701979E8B8D8B8A
:1057C000E114F104D1F0CE0145969F938F93029797
:1057D0009F938F938CE895E09F938F93FF92EF9226
:1057E0000E9432DB0FB6F894DEBF0FBECDBF01972B
:1057F00021F48B899C899E8B8D8BFE8DF8A70D895A
:105800001E896B897C894AE050E08BEF9EE00E9404
:1058100080B260EE7DE08BEF9EE00E9460B14AE0D6
:1058200050E0B8018BEF9EE00E9480B26AED7DE00F
:105830008BEF9EE00E9460B14AE050E068A58BEFDC
:105840009EE00E94EFB18BEF9EE00E9487B2198626
:105850001A861B861C861D861E861F86188A8B85C7
:105860008F7080648B871986D50118968D919C91D5
:1058700019972D893E89281739071CF001979E8BAF
:105880008D8B8B899C8997FF02C01C8A1B8ACB88D1
:10589000DC88F601EE0FFF1FEE0FFF1FFAA7E9A746
:1058A000C601880F991F8C010C0D1D1D1CA70BA78D
:1058B0008D899E898C159D050CF474C118A5113035
:1058C00021F0123009F41BC12AC12090B80A30908F
:1058D000B90AD10112968D919C911397C816D906D9
:1058E00008F050C11E968C911E971B96AC901B978A
:1058F00019960D911C911A9718964C9018971C9612
:10590000BC91BEA3E82EF12CF101F585FFA38A110D
:1059100064C02BA53CA5020F131F442009F443C00B
:10592000512C612C712CF801EB0FF11D608170E09E
:10593000762F6627072E000C880B990BA301920186
:105940000E9484D68824922EA32EB42EF801EE0D48
:10595000FF1D608170E0762F6627072E000C880BF4
:10596000990BA30192010E9484D6D9019927882717
:10597000882A992AAA2ABB2AF8018FA1E80FF11DCB
:10598000608170E0762F6627072E000C880B990B3C
:10599000A30192010E9484D6D501C401822B932BCE
:1059A000A42BB52BA0C0F8019EA1E90FF11D8081A9
:1059B000F801EE0DFF1D2081422F50E060E070E005
:1059C000BA0155274427582BF801AFA1EA0FF11D62
:1059D00080818A019B01082B84C029A53AA5020F6A
:1059E000131F8A2D90E09EA78DA7442009F45AC06A
:1059F000512C612C712CF801EE0DFF1D608170E0BF
:105A0000762F6627072E000C880B990BA3019201B5
:105A10000E9484D6B22EAA2499248824EDA5FEA53E
:105A2000E00FF11F608170E0762F6627072E000CD3
:105A3000880B990BA30192010E9484D6D901992762
:105A40008827882A992AAA2ABB2AF8019FA1E90F48
:105A5000F11D608170E0762F6627072E000C880B01
:105A6000990BA30192010E9484D6822A932AA42A28
:105A7000B52AF801AEA1EA0FF11D608170E0762F22
:105A80006627072E000C880B990BA30192010E9438
:105A900084D6B42FA32F922F882788299929AA2941
:105AA000BB2921C0F801EE0DFF1D8081EDA5FEA5EB
:105AB000E00FF11F2081422F50E060E070E0BA015A
:105AC00055274427782BF801BFA1EB0FF11D8081EA
:105AD000482BF8012EA1E20FF11D80818A019B0164
:105AE000182BD901C801892B8A2B8B2B09F04AC0AE
:105AF0002FEF3FEF4FEF50E0B601C10141C0809161
:105B0000B80A9091B90ADC0112962D913C91139735
:105B1000C216D306B8F520E030E0A90130C0EE246B
:105B2000EA94FE2C0E8D1F8D28A139A14AA15BA1FC
:105B30006CA17DA1CE0109960E94969529833A8396
:105B40004B835C836D837E838F8398878091B80AB3
:105B50009091B90AFC0122813381C216D30690F4D8
:105B60006F852E85022F10E020E030E0322F212FAC
:105B7000102F0027262B6D85A9019801262BB60131
:105B80000E943EA0FFEFCF1ADF0A09A51AA50C5FFD
:105B90001F4F1AA709A72BA53CA52D5F3F4F3CA778
:105BA0002BA786CE3FA5332309F4CEC00091B80AB7
:105BB0001091B90AD80119968D919C911A97892B49
:105BC00009F4B8C0F801C784D088E188F2880E943F
:105BD000E6A66C157D058E059F0548F40E94E6A695
:105BE000D8011F966D937D938D939C9352970E943D
:105BF000E6A6F801C784D088E188F288DC01CB01F1
:105C00008C199D09AE09BF098C329140A105B105DF
:105C1000C8F2F894D80114968D919C9115979A8B9F
:105C2000898B1996ED91FC911A977F01BFEFEB1AC2
:105C3000FB0A80818D8FF80190810388F489E02D23
:105C4000D80155968C91992309F430C09081982BF6
:105C50009C8F9081809589238B8F8B8D888F88E096
:105C60008F8B5C8D6B8D4D8D3F89288D89899A89AD
:105C7000D701508347FD252F3A952083262F39F0F1
:105C8000441F00C000006083000000C0F2CF38E075
:105C90004D9160830000019761F7D8015496FC9301
:105CA000EE9353974D8F3F8B288F3AC09081982B5E
:105CB0009C8F9081809589238B8F8B8D8A8F88E034
:105CC000898F5C8D6B8D4D8D398D2A8D89899A894F
:105CD000D701508347FD252F00C000C0208300C09E
:105CE00000C000C000C000C060830000262F3A95AD
:105CF00041F0441F000000C000C000C000C000C050
:105D0000E8CF38E04D9100C0608300C0019709F7EB
:105D1000D8015496FC93EE9353974D8F398F2A8F69
:105D20009A8B898B78940E94E6A6F8016787708B1E
:105D3000818B928B65ED7DE08BEF9EE00E9460B1E0
:105D40008BEF9EE00E9487B281E090E0AF960FB6A5
:105D5000F894DEBF0FBECDBFDF91CF911F910F91A1
:105D6000FF90EF90DF90CF90BF90AF909F908F907B
:105D70007F906F905F904F903F902F900895CF93BA
:105D8000DF9362E975E08EE59EE00E942846C091AF
:105D9000B80AD091B90A4C815D8160E070E08985D4
:105DA0009A850E9480D4209771F089859A850E94F7
:105DB000A0CB8E819F8197FD03C060E00E94C2A5A9
:105DC000CE010E94A0CB1092B70A1092B60A81E0D1
:105DD00090E0DF91CF9108952F923F924F925F9282
:105DE0006F927F928F929F92AF92BF92CF92DF92EB
:105DF000EF92FF920F931F93CF93DF93CDB7DEB750
:105E000061970FB6F894DEBF0FBECDBF0E9445A7C5
:105E10009B01AC016091BE0A7091BF0A8091C00ADB
:105E20009091C10AAA24AA94BA2C650118E8E12E1F
:105E300013E1F12E00E010E00E941C3E882309F4DB
:105E40006DC3E0909210F0909310D70112968C9150
:105E5000823089F465E17EE08BEF9EE00E9460B1C4
:105E60008BEF9EE00E9487B28091921090919310E8
:105E70000E94E06EE8C18091BC0A9091BD0A892B16
:105E800009F067C083E190E00E9408CB8C0186E8AE
:105E900098E7F801928B818BF682E582148210825A
:105EA00089E0818381E0828383831093BD0A00931C
:105EB000BC0A0E9445A74B015C01F0E18F0EF7E29E
:105EC0009F1EA11CB11CD8011596ED91FC9116974F
:105ED0008FEF83871486DF0113963B961D92EA1796
:105EE000FB07E1F7F8011482DD24D394BE01665F5D
:105EF0007F4FD80115968D919C9116970E94B56F92
:105F0000181644F40E9445A7681579058A059B0573
:105F100008F4A4C100E010E0E12CF12C2091B40AB7
:105F20003091B50A8091BC0A9091BD0AE216F30641
:105F300074F46091B20A7091B30A600F711F0E94ED
:105F40003EC5BFEFEB1AFB0A085F1F4FE7CFFC010E
:105F500012828091BA0A9091BB0A2091B40A3091C2
:105F6000B50A821793070CF46AC00E9445A71B016B
:105F70002C016BE07EE08EE59EE00E948BB2E0910A
:105F80009210F0919310309751F08FEF8387148621
:105F9000DF0113963B961D92AE17BF07E1F7E09124
:105FA000AE0AF091AF0A80E090E02091B40A3091FF
:105FB000B50A821793073CF4208131812E7F21930B
:105FC00031930196F2CF66246394712C80919210E4
:105FD00090919310009709F482C26091B40A709175
:105FE000B50A23E0660F771F2A95E1F72091B20AE0
:105FF0003091B30A620F731F0E94B56F18160CF030
:106000006EC28090B40A9090B50AF4E18F169104A4
:106010000CF065C20E9445A79B01AC01AA24AA947A
:10602000BA2C650118E8E12E13E1F12E00E010E032
:10603000C201B1010E941C3E811151C294C1009164
:10604000B20A1091B30A9C0143E0220F331F4A9514
:10605000E1F7020F131FF8012081283209F0EEC08A
:10606000AE014F5F5F4FB8018091BC0A9091BD0AAD
:106070000E94746F882369F12A8130E0C901982F4A
:106080008827990F990F990F6981F8E06F9FB001E8
:1060900011249C01262B372BD8018C918031E1F4FF
:1060A000688570E08F81FB01E81BF109CF019695AF
:1060B000982F8827979587950E94E7D66051710998
:1060C000207F13E0220F331F1A95E1F7620F731F31
:1060D00004C060E874EE01C0B9016138F4EE7F07D6
:1060E0007CF0072E000C880B990B0E9441D520E014
:1060F00030E040E05CE30E94A0D59B01AC0104C00D
:1061000020E030E04EEF52ECE091B00AF091B10A9D
:10611000309789F08091BA0A9091BB0ABC01A3E044
:10612000660F771FAA95E1F7A091B20AB091B30A62
:106130006A0F7B1F19950091BA0A1091BB0A43E0C0
:10614000000F111F4A95E1F78091B20A9091B30AAE
:10615000080F191FE090BC0AF090BD0AD8018C917D
:10616000803149F0B801C7010E94876FD82E88237B
:1061700009F460C002C03CE0D32EF701858196810E
:106180000E94E06E882309F455C0B801D701159626
:106190008D919C9116970E94966EF701408164E460
:1061A000858196810E94746ED70112968C91882306
:1061B00009F440C0E7EFED0DE33040F4F0E0EE0FFE
:1061C000FF1FEB5FFC4F4080518004C09EEE492EC4
:1061D00092E0592E0115110539F1F70183818823C9
:1061E00019F18081811120C00E9445A74B015C01FB
:1061F000052C000C66087708AE014F5F5F4FB801B1
:10620000C7010E941E6F8981811114C00E9445A799
:10621000DC01CB0184199509A609B70988159905F0
:10622000AA05BB0548F306C0B201550C880B990BB3
:106230000E940BA78091BA0A9091BB0A0196909395
:10624000BB0A8093BA0A0E9445A76093BE0A709366
:10625000BF0A8093C00A9093C10A60C167E0CE0173
:106260000A960E94236E9989891373C062EA75E0C9
:106270008EE59EE00E949DB2F8018081811138C0B8
:10628000858196810E94E06EBE01665F7F4FD801D6
:1062900015968D919C9116970E94966E40E064EB46
:1062A000F801858196810E94746ED8011596ED9053
:1062B000FC901697C7010E94306EC7010E94E73C10
:1062C00067E882EE9CE00E94F23960E882EE9CE092
:1062D0000E94F239C7010E94D93CC7010E94306E6A
:1062E000F82EF801858196810E94E06EF5FE38C097
:1062F000AE014F5F5F4FBE01665F7F4FC8010E94D6
:106300001E6FD8011196FC908A85803109F401C175
:10631000BE01665F7F4FC8010E94876F8F1518F41A
:10632000F80181810BC08A85803111F48CE006C0B0
:10633000BE01665F7F4FC8010E94876FD80111962A
:106340008C93119714968C9114978F5F14968C935D
:10635000CDCD64EA75E08EE59EE00E949DB2C6CD8B
:10636000D801DC92C5CFA090B20AB090B30A7401F4
:1063700083E0EE0CFF1C8A95E1F7EA0CFB1C67E05A
:10638000C7010E94236EF701978189131FCE00E099
:1063900010E008151905CCF548E050E0B701C5013B
:1063A0000E9436DA28E0A20EB11C892B59F5000FA5
:1063B000111FE091AE0AF091AF0AE00FF11F80814A
:1063C000918181609183808364E07EE08BEF9EE029
:1063D0000E9460B18091B40A9091B50AA3E0880F41
:1063E000991FAA95E1F72091B20A3091B30A820F62
:1063F000931F0E94C0C56DEF7DE08BEF9EE00E9471
:106400008BB2E4CD0F5F1F4FC4CF8091BC0A909137
:10641000BD0A892B09F4DACDE091B40AF091B50AEE
:10642000EE0FFF1F8091AE0A9091AF0AE80FF91F9F
:10643000718260820091B40A1091B50A68EF7DE024
:106440008BEF9EE00E9460B14AE050E0B8018BEF14
:106450009EE00E9480B261EF7DE08BEF9EE00E94A3
:1064600060B18091B40A9091B50A63E0880F991FDA
:106470006A95E1F72091B20A3091B30A820F931F17
:106480000E94C0C58BEF9EE00E9487B26091B40A63
:106490007091B50AE3E0660F771FEA95E1F7809106
:1064A000B20A9091B30A680F791FDB018C91883290
:1064B00061F48091BC0A9091BD0A0E943EC5809112
:1064C0009210909193100E94FA3D8091B40A90919D
:1064D000B50A01969093B50A8093B40A77CD0091DE
:1064E000B40A1091B50A62EE7DE08BEF9EE00E9447
:1064F00060B14AE050E0B8018BEF9EE00E9480B2AC
:106500008BEF9EE00E9487B21092BB0A1092BA0AEB
:106510009ACEFCE0FF1508F403CF08CF61960FB6C2
:10652000F894DEBF0FBECDBFDF91CF911F910F91C9
:10653000FF90EF90DF90CF90BF90AF909F908F90A3
:106540007F906F905F904F903F902F9008950F93A2
:106550001F93CF93DF938C010E949C9CC8010E94E3
:10656000F5C166EA75E08EE59EE00E9428468091BE
:10657000B80A9091B90A892B09F586E190E00E944A
:1065800008CBEC01F801238534854285042E000CEC
:10659000550B608571850E94ADA0D093B90AC09358
:1065A000B80A8E819F8197FD07C061E00E94C2A555
:1065B00060E08E810E9493A581E0898381E090E074
:1065C0009093B70A8093B60ADF91CF911F910F91F4
:1065D00008958F929F92AF92BF92CF92DF92EF92E7
:1065E000FF920F931F93CF93DF9300D000D0CDB7CE
:1065F000DEB78090C20A9090C30A8114910409F416
:10660000B5C08091D70A8F5F8093D70A0E9445A7B3
:106610009B01AC016091CA0A7091CB0A8091CC0AAF
:106620009091CD0AAA24AA94BA2C65011FE0E12E0C
:10663000F12C00E010E00E941C3E882309F44DC0BC
:10664000F4010681178101151105C9F1F801808552
:106650008F70863081F563EB75E0C8010E948F561C
:106660000097D9F0FC0120852F702530B1F4E68029
:10667000F780E114F104F9F0FA82E982B801CE0161
:1066800001960E94AB9D62E070E0CE0101960E94EF
:10669000B950F701E280F380ECCF1A83098360E000
:1066A00070E0CE0101960E94AB9D62E070E0CE01E9
:1066B00001960E94B950F80102811381C4CF0E9453
:1066C00045A76093CA0A7093CB0A8093CC0A909333
:1066D000CD0A1092100F1092110F0E9445A79B0136
:1066E000AC016091C60A7091C70A8091C80A909166
:1066F000C90AAA24AA94BA2C650118E8E12E13E16C
:10670000F12E00E010E00E941C3E882351F1E09140
:10671000C20AF091C30A0681178101151105B9F06B
:10672000F80180858F70863071F41A83098360E0E8
:1067300070E0CE0101960E94AB9D61E070E0CE0159
:1067400001960E94B950F80102811381E6CF0E94A0
:1067500045A76093C60A7093C70A8093C80A9093AE
:10676000C90A8091D70A81508093D70A26960FB61E
:10677000F894DEBF0FBECDBFDF91CF911F910F9177
:10678000FF90EF90DF90CF90BF90AF909F908F9051
:1067900008950E9400A3A8950E94FC0F039724F07F
:1067A0000E9424AB0E94E9320C94289E2F923F92C3
:1067B0004F925F926F927F929F92AF92BF92CF92D1
:1067C000DF92EF92FF920F931F93CF93DF93CDB79A
:1067D000DEB7CE55D1090FB6F894DEBF0FBECDBFE0
:1067E0008091D70A8F5F8093D70AE0919610F0913D
:1067F00097103097B9F006811781E0909610F090CD
:106800009710E114F10471F00115110559F0F80128
:1068100080858F708530A9F7C8010E94C9B9823080
:1068200080F3E7C18091D70A81508093D70A809185
:10683000941090919510059709F439C50E9445A7C9
:106840009B01AC016091CE0A7091CF0A8091D00A71
:106850009091D10AAA24AA94BA2C650118EEE12ECF
:1068600013E0F12E00E010E00E941C3E882309F4A2
:106870001EC510E0CC24C394D12C54E0252E312C1D
:10688000E091C40AF091C50A309709F410C51111BE
:106890000EC580858F70853009F090C1F9AFE8AFE3
:1068A00023961FAE1EAE2397CE01C8960E943B8C46
:1068B00021968FAD2197883009F434C1893009F4CD
:1068C00040C0843009F069C18091291090912A104C
:1068D000892B09F022C160E074E0CE01C8960E94C5
:1068E000DD8B892B09F46AC019821A821B821C82F3
:1068F0001D821E821F8218868B818F708B83198266
:1069000041E0BE01685C7F4FCE0101960E94B473E6
:1069100064E27EE08BEF9EE00E9460B160E074E094
:10692000CE01C8960E946B8B09811A812B813C8114
:106930004D815E816F817885CE01C8960E945A6133
:10694000ECC08091291090912A10892B09F0E5C0A4
:1069500060E074E0CE01C8960E94DD8B892B09F4BB
:10696000F3C119821A821B821C821D821E821F8221
:1069700018868B818F708B83198241E0BE01685C21
:106980007F4FCE0101960E94B47366E87EE08BEFE4
:106990009EE00E9460B160E074E0CE01C8960E9463
:1069A0006B8B09811A812B813C814D815E816F81C6
:1069B0007885CE01C8960E948A60AFC0EAACFBAC75
:1069C000F70180858F70853009F02FC1C7010E94C3
:1069D000C9B9A82EB12CF2E0AF16B1040CF425C150
:1069E000D0922A10C092291060E070E0CE01C896C3
:1069F0000E940A8B3C0161E070E0CE01C8960E94C3
:106A00000A8B8C01F5E0AF16B1040CF47CC164E094
:106A1000C7010E9448B9FC01E184F28426E040E805
:106A200055E260E070E08AE99BE00E94FCBC609265
:106A3000310D8AE99BE09093300D80932F0D1092D9
:106A40003C0E10923E0E10923D0EF1E0EF16F10456
:106A500009F40CC10CF4F0C092E0E916F10409F05D
:106A6000F7C01093330D0093320DD092350DC092C4
:106A7000340D83E00E9445BA982E911028C1E09011
:106A8000360DF090370DC7010F2C000CAA0BBB0B75
:106A900089839A83AB83BC8380E190E09E838D835E
:106AA000E8ADF9ADA080B18066E57EE08BEF9EE0B9
:106AB0000E9460B1B5018BEF9EE00E949DB26FE431
:106AC0007EE08BEF9EE00E9460B1BE016F5F7F4F62
:106AD0008BEF9EE00E94938D0E9487B2B701CE019A
:106AE000C8960E94AF5FA090C40AB090C50AF50195
:106AF000828193819A8389831B861A86CE010196AF
:106B00000E943B8CAB2809F0C2C0CE0101960E94C6
:106B10002C8C10922A1010922910CE01C8960E9437
:106B2000915FB9C38091291090912A10892BA9F700
:106B300060E074E0CE01C8960E94DD8B892B69F37A
:106B400019821A821B821C821D821E821F82188655
:106B50008B818F708B83198241E0BE01685C7F4F0F
:106B6000CE0101960E94B4736BED7EE08BEF9EE048
:106B70000E9460B160E074E0CE01C8960E946B8B09
:106B800009811A812B813C814D815E816F817885DD
:106B9000CE01C8960E942862C0CFCE01C8960E943E
:106BA000915F61E070E0CE01C8960E949247892B08
:106BB00009F071C3CE01C8960E942C8CE091C40AE2
:106BC000F091C50A309709F472C382819381909342
:106BD000C50A8093C40A892B09F052CEE091961021
:106BE000F0919710868197819093C50A8093C40A8B
:106BF0005EC31A8309831B861A86CE0101960E9402
:106C00003B8CCE0101960E94438A882331F062E0DA
:106C100070E0CE0101960E949247F8010281138133
:106C2000CE0101960E942C8CE8CD63E77EE08BEFCD
:106C30009EE00E9460B171CFEF2811F51093330DE3
:106C40000093320DD092350DC092340D81E012CFF9
:106C5000E3E0EE16F104A1F41093330D0093320D2E
:106C6000D092350DC092340D84E004CF1093330DD3
:106C70000093320DF092350DE092340D82E0FACEA1
:106C80006BE57EE08BEF9EE00E9460B1F6CECE0118
:106C900001960E94438A882309F437CF898584307E
:106CA00009F033CF60E070E0CE0101960E940A8BBC
:106CB0006816790609F029CF61E070E0CE010196EF
:106CC0000E940A8B0817190709F01FCF20C0892DD1
:106CD00090E0A0E0B0E089839A83AB83BC8380E13D
:106CE00090E09E838D8369E37EE08BEF9EE00E94BF
:106CF00060B1BE016F5F7F4F8BEF9EE00E94938D6E
:106D00000E9487B206CF82E0E82EF12C87CEB70131
:106D1000CE0101960E94AF5FE091C40AF091C50ACE
:106D2000828193819093C50A8093C40A892B09F0CC
:106D3000ECCEE0919610F091971086819781909318
:106D4000C50A8093C40AE1CED0922A10C0922910BD
:106D50000E9468B65C01892B29F0F5018085807F4F
:106D60008660808720E030E043E050E060E2CE01C2
:106D700001960E94D23EE8ADF9AD608171814FE18C
:106D800050E0CE0101960E948EDA67EB75E0CE01ED
:106D900001960E9468DA26E040E855E260E070E083
:106DA0008AE99BE00E94FCBC60E070E0CE01C896DE
:106DB0000E940A8B8093310D8AE99BE09093300DFD
:106DC00080932F0D10923C0E10923E0E10923D0EAD
:106DD00084E398E09093330D8093320DEAE0F0E085
:106DE000F093350DE093340D83E00E9445BA811194
:106DF000F1C061ED7EE08BEF9EE00E9460B126E382
:106E0000622E2DE0722E0AE41DE030E1E32EF12C1B
:106E1000F301819191913F01092E000CAA0BBB0B4C
:106E200089A39AA3ABA3BCA3FEA2EDA2BE016F5D92
:106E30007F4F8BEF9EE00E94938D6FEC7EE00E946F
:106E400060B10615170521F78BEF9EE00E9487B20F
:106E500060913A0D70913B0D80E090E00E9441D529
:106E600020E030E048EC52E40E949AD79B01AC014C
:106E700062EA75E0C5010E941D4880913E0D909127
:106E80003F0D2C01612C712CA30192016DEB75E07B
:106E9000C5010E9406BA6091400D7091410D80E0DD
:106EA00090E00E9441D520E030E048EC52E40E949E
:106EB0009AD79B01AC0164EA75E0C5010E941D48A8
:106EC0006091420D7091430D80E090E00E9441D5A9
:106ED00020E030E040E251E40E949AD79B01AC01EF
:106EE0006FEB75E0C5010E941D482091360D309171
:106EF000370D40E050E061EC75E0C5010E9406BA34
:106F000045284628472809F47FC0EAADFBAD9085A7
:106F10009F70953009F078C061E0CF010E9448B9B8
:106F2000009709F471C0FC0120852F70243009F00E
:106F30006BC061857285CE0181960E940D8DCE0158
:106F400081960E94438A882309F43FC063961CAE51
:106F50001DAE1EAE1FAE639767961CAE1DAE1EAE75
:106F60001FAE679762968FAD62978F7062968FAFF4
:106F7000629760961FAE609764E670E0CE01815B19
:106F80009F4F0E94977468962FAF689769963FAF9E
:106F900069976A964FAF6A976B965FAF6B976C96DF
:106FA0006FAF6C976D967FAF6D976E968FAF6E9744
:106FB0006F969FAF6F97E12CF12C89019A01AB017D
:106FC000BC01CE0181960E941C1ACE0181960E94BE
:106FD0002C8C1AC090E0A0E0B0E089A39AA3ABA3E8
:106FE000BCA380E190E09EA38DA369EB7EE08BEFD4
:106FF0009EE00E9460B1BE016F5D7F4F8BEF9EE00F
:107000000E94938D0E9487B28091360D83FF2EC01F
:107010008EE398E09093330D8093320DD092350D2E
:10702000C092340D83E00E9445BA81110BC02091BB
:10703000360D3091370D40E050E064EC75E0C5014D
:107040000E9406BA10922A1010922910CE01C896FA
:107050000E943F631816190624F4CE01C8960E94B8
:10706000BB47D0922A10C092291008C020E030E01F
:10707000A90164EC75E0C5010E9406BA62E370E004
:1070800080E090E00E940BA783E190E09093330DA5
:107090008093320D3092350D2092340D83E00E94A2
:1070A00045BA8111A0C06FEA7EE08BEF9EE00E949E
:1070B00060B196E3E92E9DE0F92E0EE31DE0F701A5
:1070C000619171917F014AE050E08BEF9EE00E9458
:1070D00080B26DEA7EE08BEF9EE00E9460B10E15FB
:1070E0001F0569F78BEF9EE00E9487B20091360D75
:1070F0001091370D01151105D1F0B801012E000CCA
:10710000880B990B0E9441D52DEE3EE94CE35EE3DE
:107110000E94A0D522E538EB42E152E40E942DD72F
:107120009B01AC0167EF76E0C5010E941D486091AC
:10713000380D7091390D072E000C880B990B0E94A9
:1071400041D52DEE3EE94CE35EE30E94A0D522E559
:1071500038EB42E152E40E942DD72B013C019B0108
:10716000AC016BEB75E0C5010E941D4860913C0DC0
:1071700070913D0D16161706A4F4072E000C880B0F
:10718000990B0E9441D520E030E040E251E40E949A
:107190009AD79B01AC0168EC75E0C5010E941D48BF
:1071A00008C020E030E0A90168EC75E0C5010E944C
:1071B00006BA20E030E040E252E4C301B2010E948E
:1071C00042D8181644F5012B31F10E940AB88823E1
:1071D00029F08091D60A882309F44EC0CE01C896C2
:1071E0000E94BB4718C090E0A0E0B0E089A39AA33A
:1071F000ABA3BCA380E190E09EA38DA367E97EE0F2
:107200008BEF9EE00E9460B1BE016F5D7F4F8BEF00
:107210009EE00E94938D80E091E00E9408CB8C015B
:10722000892BD9F01CA21BA21EA21DA28FEF9FEFDB
:1072300098A78FA38FE093E09AA389A31AA619A613
:107240001CA70BA780E091E098AB8FA71EA61DA6F8
:10725000B501CE0181960E945CA30E940AB88823E2
:1072600021F08091D60A882381F0C8010E94A0CB2A
:10727000C5010E94EB474DCCE8ADF9AD608171814D
:107280008CEC95E00E943042A9CFB801CE01019666
:107290000E943042EACF0E9445A76093CE0A7093C5
:1072A000CF0A8093D00A9093D10A11E083CCC25ABE
:1072B000DF4F0FB6F894DEBF0FBECDBFDF91CF9189
:1072C0001F910F91FF90EF90DF90CF90BF90AF9004
:1072D0009F907F906F905F904F903F902F90089578
:1072E0004091400B262F30E0240F311D2132310513
:1072F000DCF42091640B2430C9F4FC0180E090E0C0
:10730000861758F43091400B2191DC01A05EB44FF8
:10731000A30FB11D2C930196F3CF8091400B680F02
:107320006093400B80E0089581E0089582E0089525
:1073300008950895E091910B8091900BE81730F437
:10734000F0E0E650F54F808190E008958FEF9FEFD9
:1073500008959091910B8091900B981750F4E92F1C
:10736000F0E0E650F54F208130E09F5F9093910B65
:1073700002C02FEF3FEFC90108958091900B90E07C
:107380002091910B821B91090895CF92DF92EF9289
:10739000FF920F931F93CF93DF937C01CB018A0160
:1073A0002091F90A222389F0EB016B01C40ED51E4E
:1073B000CC15DD0569F06991D701ED91FC91019043
:1073C000F081E02DC7011995F3CF642F0E94703929
:1073D000C801DF91CF911F910F91FF90EF90DF9047
:1073E000CF900895CF93DF931F92CDB7DEB7698317
:1073F0002091F90A2223D1F020918E0B203240F007
:1074000021E030E0FC013383228380E090E015C06E
:1074100080918F0BE82FF0E0E752F54F9981908330
:107420008F5F80938F0B80938E0B05C061E0CE0140
:1074300001960E94703981E090E00F90DF91CF912A
:107440000895DC0116968D919C911797009739F05D
:10745000DC01ED91FC910190F081E02D199481E027
:1074600090E00895DC0116968D919C9117970097F6
:1074700039F0DC01ED91FC910680F781E02D199443
:1074800008951092640B81E08093660B1092650B57
:1074900061E084E10E9493A561E085E10E9493A5EB
:1074A000E9EBF0E080818E7F808380818D7F808317
:1074B00088E48093B80085E48093BC000895CF935E
:1074C000DF9391E090931F0B8823B9F0C091B8002F
:1074D000D091BA008091BC008A7B8093BC0060E0B0
:1074E00084E10E9493A560E085E10E9493A50E943B
:1074F000413AD093BA00C093B800DF91CF9108957C
:1075000085ED8093BC0080911B0B90911C0BA0918A
:107510001D0BB0911E0B0796A11DB11D23E0B69562
:10752000A795979587952A95D1F72091BC0024FFC0
:107530001CC040911B0B50911C0B60911D0B709156
:107540001E0B452B462B472B81F30097A105B10558
:1075500041F025E32A95F1F700000197A109B1094F
:10756000E4CF80911A0B0C945F3A1092640B08954B
:107570001F920F920FB60F9211240BB60F922F93FA
:107580003F934F935F936F937F938F939F93AF93AB
:10759000BF93EF93FF938091B900887F803609F401
:1075A0009CC068F5883209F45BC090F4803109F41E
:1075B00054C038F4882309F4F6C0883009F44DC06B
:1075C000F6C0883109F44CC0803209F45DC0EFC0C8
:1075D000803409F468C048F4803309F455C0883316
:1075E00009F0E5C08093630BD8C0803509F44FC023
:1075F000883509F45DC0883409F0D9C0D6C088390F
:1076000009F4C7C0A8F4883709F467C038F488368D
:1076100009F463C0803709F460C0C9C0883809F430
:10762000B8C0803909F45FC0803809F0C0C05BC0C1
:10763000803B09F486C038F4803A09F466C0883A81
:1076400009F47FC0B4C0803C09F4A7C0883C09F4A9
:10765000A4C0883B09F48AC0AAC08091890B10C0DD
:107660009091880B8091870B981770F5E091880BAB
:1076700081E08E0F8093880BF0E0E959F44F808110
:107680008093BB0085EC86C08093630B8EC0E09135
:10769000880B81E08E0F8093880B8091BB00F0E017
:1076A000E959F44F80839091880B8091870B6EC0CD
:1076B000E091880B81E08E0F8093880B8091BB0056
:1076C000F0E0E959F44F80838091660B81116DC021
:1076D00081E08093650B84EA61C083E08093640B52
:1076E0001092620BCFCF8091620B803208F051C0B4
:1076F000E091620B81E08E0F8093620B8091BB0062
:10770000F0E0EE5BF44F8083BDCF85EC8093BC004E
:107710001092640B8091620B803230F4E091620B26
:10772000F0E0EE5BF44F10826091620B70E0E0914C
:107730008A0BF0918B0B82E49BE019951092620BFF
:1077400036C084E08093640B1092410B1092400B82
:10775000E0918C0BF0918D0B19958091400B81116C
:1077600005C081E08093400B1092200BE091410B0B
:1077700081E08E0F8093410BF0E0E05EF44F80815A
:107780008093BB009091410B8091400B981708F4B7
:1077900079CF85E88093BC000AC085EC8093BC005B
:1077A0001092640B04C01092630B0E94803AFF9108
:1077B000EF91BF91AF919F918F917F916F915F9169
:1077C0004F913F912F910F900BBE0F900FBE0F90D6
:1077D0001F9018958F929F92AF92BF92CF92DF9297
:1077E000EF92FF920F931F93CF93DF9310918E0B25
:1077F000113208F0C2C0062FD091D80A0E94E6A626
:107800006B017C01C091640BCC2311F180911B0BA7
:1078100090911C0BA0911D0BB0911E0B892B8A2BF4
:107820008B2B81F30E94E6A680901B0B90901C0B83
:10783000A0901D0BB0901E0BDC01CB018C199D0993
:10784000AE09BF0988169906AA06BB06D8F681C0FC
:1078500082E08093640B0093660B8FEF8093630B41
:107860001092880B1093870BA9EDBAE0E7E6FBE0D6
:1078700080E0181721F09D9191938F5FFACF1092BD
:10788000890B9091890B8D2F880F892B8093890B01
:107890008091650B813089F51092650B0E94E6A6F8
:1078A0006B017C018091890B8093BB0080911B0B45
:1078B00090911C0BA0911D0BB0911E0B892B8A2B54
:1078C0008B2BA9F00E94E6A600911B0B10911C0BBC
:1078D00020911D0B30911E0BDC01CB018C199D09F1
:1078E000AE09BF09081719072A073B0790F18091D5
:1078F000BC0083FDD7CF85EC01C085EE8093BC0032
:107900000E94E6A66B017C018091640B823039F500
:1079100080911B0B90911C0BA0911D0BB0911E0B25
:10792000892B8A2B8B2B81F30E94E6A600911B0BDF
:1079300010911C0B20911D0B30911E0BDC01CB0113
:107940008C199D09AE09BF09081719072A073B07BB
:10795000D8F680911A0B0E945F3AC5E013C080915F
:10796000630B8F3F79F08091630B803241F08091FF
:10797000630B803331F0C4E005C0C1E003C0C2E056
:1079800001C0C3E010928F0B10928E0B1092F90A77
:107990008C2FDF91CF911F910F91FF90EF90DF908F
:1079A000CF90BF90AF909F908F90089561E00C941E
:1079B000EA3B82EE9CE00C94D63C81E08093F90A8D
:1079C0006093D80A10928F0B10928E0B0895FC01D1
:1079D000618182EE9CE00C94DD3C1F93CF93DF939A
:1079E000EC01162F0E94E73C61EE82EE9CE00E94C3
:1079F000F239612F82EE9CE00E94F239CE01DF91D4
:107A0000CF911F910C94D93C8F929F92AF92BF92CD
:107A1000CF92DF92EF92FF920F931F93CF93DF935A
:107A2000F62ED42F0E94E6A64B015C01C091640B98
:107A3000CC2339F180911B0B90911C0BA0911D0B55
:107A4000B0911E0B892B8A2B8B2B81F30E94E6A60B
:107A500000911B0B10911C0B20911D0B30911E0BE4
:107A6000DC01CB0188199909AA09BB090817190774
:107A70002A073B07D8F680911A0B0E945F3AC0E0B4
:107A800090C0D13208F0D0E281E08093640B809303
:107A9000660B9FEF9093630B1092880B9D0F909352
:107AA000870B8093890B8091890B6F2D660F682B54
:107AB0006093890B8091650B813089F51092650B7D
:107AC0000E94E6A66B017C018091890B8093BB002C
:107AD00080911B0B90911C0BA0911D0BB0911E0B64
:107AE000892B8A2B8B2BA9F00E94E6A680901B0B7A
:107AF00090901C0BA0901D0BB0901E0BDC01CB01D5
:107B00008C199D09AE09BF0988169906AA06BB06FD
:107B100090F18091BC0083FDD7CF85EC01C085EE4C
:107B20008093BC000E94E6A66B017C018091640BEF
:107B3000813031F580911B0B90911C0BA0911D0B96
:107B4000B0911E0B892B8A2B8B2B81F30E94E6A60A
:107B500080901B0B90901C0BA0901D0BB0901E0BE7
:107B6000DC01CB018C199D09AE09BF098816990665
:107B7000AA06BB06D8F680911A0B0E945F3A11C084
:107B80008091880B8D1710F4D091880BE7E6FBE00D
:107B9000AAEFBAE0C0E0CD1721F081918D93CF5FBD
:107BA000FACF1092910BC093900B8C2FDF91CF9155
:107BB0001F910F91FF90EF90DF90CF90BF90AF900B
:107BC0009F908F90089541E0FC01618182EE9CE0DE
:107BD0000E94043D82EE9CE00E94A9390895CF9353
:107BE000DF93EC0163EC0E94ED3CCE01DF91CF917D
:107BF0000C94E33DCF93DF93EC010E94EF3D682F9F
:107C00006460CE01DF91CF910C94B56ECF93C82FF5
:107C10000E9445A704C09695879577956795CA9564
:107C2000D2F7611571058105910521F461E070E0DD
:107C300080E090E0CF9108954F925F926F927F9293
:107C4000AF92BF92CF92DF92EF92FF920F931F936A
:107C5000CF93DF9300D01F92CDB7DEB72B013C014D
:107C600029833A834B835C83A60195016E0D7F1DAA
:107C7000801F911F0E9484D629813A814B815C81AB
:107C8000621773078407950770F4241535054605B8
:107C9000570510F421E017C021E046165706680684
:107CA000790688F00FC0461657066806790650F424
:107CB00021E089819A81AB81BC8184159505A60557
:107CC000B70508F020E0822F0F900F900F900F90D3
:107CD000DF91CF911F910F91FF90EF90DF90CF90A8
:107CE000BF90AF907F906F905F904F9008958F926C
:107CF0009F92AF92BF92CF92DF92EF92FF920F933B
:107D00001F93CF93DF93CDB7DEB72B970FB6F894C1
:107D1000DEBF0FBECDBF8C01CE0101967C016C0190
:107D20008AE0882E912CA12CB12CC6018E199F09B6
:107D3000411551056105710581F0CB01BA01A5011D
:107D400094010E9484D6942F852F605DF601619383
:107D50006F01A901692F782FE8CFFC013197EE0D53
:107D6000FF1DD8019E012150310940814D9331976B
:107D7000E217F307D1F7F801E80FF91F10822B96ED
:107D80000FB6F894DEBF0FBECDBFDF91CF911F912C
:107D90000F91FF90EF90DF90CF90BF90AF909F90AA
:107DA0008F9008958F929F92AF92BF92CF92DF9261
:107DB000EF92FF920F931F93CF93DF938C014A01B1
:107DC0005901E090D40AF090D50AC62F660FDD0B5A
:107DD000E114F10471F1F70180858F70863049F567
:107DE00069ED75E0C7010E948F566C01F2E08F16B5
:107DF000910439F083E08816910451F461E478E04D
:107E000002C06EED75E0C7010E948F567C0102C072
:107E1000E12CF12CC114D10471F0F60180858F7032
:107E2000843049F461857285AE01C8010E94ACDAE4
:107E300008C0E12CF12CAE016AEF7EE0C8010E947F
:107E400036CEAE0166E675E0C8010E948EDAE11416
:107E5000F10441F0F70180858F70843019F4618559
:107E600072850FC0F2E08F169104A1F083E08816AE
:107E7000910461F08A94892899F46091D20A7091F2
:107E8000D30AAE01C8010E948EDA0AC0AE0164EFC7
:107E90007EE003C0AE0161EF7EE0C8010E9418CE13
:107EA000AE0166E675E0C8010E948EDAA114B10445
:107EB00029F0AE01B501C8010E948EDAC801DF9138
:107EC000CF911F910F91FF90EF90DF90CF90BF90D7
:107ED000AF909F908F900895CF92DF92EF92FF9294
:107EE0000F931F93CF93DF936B017C01EA010E94F4
:107EF0000CD88B011F936F9386E798E09F938F9325
:107F0000DF93CF930E9403DB0F900F900F900F90A1
:107F10000F900F9020E030E0A901C701B6010E9448
:107F200042D8181624F0F7FAF094F7F8F094099074
:107F30000020E9F721978EE28883B80117FF03C07C
:107F4000719561957109072E000C880B990B0E94A1
:107F500041D59B01AC01C701B6010E942DD720E09D
:107F600030E040E251E40E94A0D50E940CD8605D50
:107F700069831A82DF91CF911F910F91FF90EF904B
:107F8000DF90CF900895CF93DF931F921F92CDB7CC
:107F9000DEB78091B0119091B111009711F48CEB84
:107FA00091E1BE016F5F7F4F681B790B072E000CBC
:107FB000880B990B0F900F90DF91CF910895EF925E
:107FC000FF920F931F93CF93DF93FC01892B81F1D5
:107FD000A081B181109761F18C91882349F1E080F3
:107FE000F180D7018C91882359F08D3249F080536C
:107FF0008A3030F0BFEFEB1AFB0AF182E082EFCF5C
:108000008F01C7010E94D8CDD82FC92F6CE270E034
:10801000C7010E9473DA009721F4F80111821082DF
:1080200004C00196D8018D939C938D2F9C2F02C084
:1080300080E090E0DF91CF911F910F91FF90EF9042
:1080400008959FE9980F963010F4875508959FEB97
:10805000980F963010F48753089580538A3008F0B3
:1080600080E00895CF93DF93DA01382FEC018C2F55
:10807000831B8617C8F4CE01E991F0E024E0F59562
:10808000E7952A95E1F7E95CFC4F20812C93FC01F0
:108090008081E82FEF70F0E0E95CFC4F8081119661
:1080A0008C9311971296E3CFFA01E60FF11DE60FBC
:1080B000F11D1082DF91CF9108958F929F92AF9220
:1080C000BF92CF92DF92EF92FF920F931F93CF93C5
:1080D000DF93CDB7DEB7C855D1090FB6F894DEBF30
:1080E0000FBECDBF6296EFAE62976396FFAE639709
:1080F00064960FAF649765961FAF659766962FAF2E
:10810000669767963FAF679768964FAF689769968F
:108110005FAF6997009709F483C1D62E8C01FC01EB
:1081200080858295807F8595859585958595853017
:1081300019F0863091F174C18091D70A8F5F8093D6
:10814000D70AF801A680B780A114B10401F16296A4
:10815000EFAC62976396FFAC639764960FAD64973C
:1081600065961FAD659766962FAD669767963FAD8E
:10817000679768964FAD689769965FAD69976D2D63
:10818000C5010E945D40F501A280B380DDCF8091E2
:10819000D70A81508093D70A43C163EB75E0C801C9
:1081A0000E948F560097E1F06296EFAC629763965B
:1081B000FFAC639764960FAD649765961FAD6597A6
:1081C00066962FAD669767963FAD679768964FADF9
:1081D000689769965FAD69976D2D0E945D402CC1CF
:1081E00063EE75E0C8010E948F564C0168EE75E0A1
:1081F000C8010E948F565C01DD2021F0F1E0DF16FE
:1082000041F03FC06DEE75E0C8010E948F567C01C1
:108210001AC067EF75E0C8010E948F567C016CEFB1
:1082200075E0C8010E948F566C01E114F10409F059
:10823000FFC06DEE75E0C8010E948F567C01C1142D
:10824000D10409F0EFC062EF75E0C8010E948F56BB
:108250006C01E114F10441F0F70180858F708430E6
:1082600019F4E184F28402C0E12CF12CC114D10490
:1082700051F0F60180858F70843029F401851285D4
:1082800011C0E12CF12C0FEF10E020E033E040E1D1
:1082900050E0BE016F5B7F4FCE018F5A9F4F0E940F
:1082A00051718C018114910489F1F4016185728509
:1082B0008BEF9EE0E114F10491F00E949DB26BE01F
:1082C0007FE08BEF9EE00E9460B1B7018BEF9EE0F4
:1082D0000E949DB28BEF9EE00E9487B208C00E9470
:1082E0009DB266E07FE08BEF9EE00E9460B1CE0120
:1082F0008F5A9F4F0E940973A114B10459F4F401DD
:1083000080858F70843009F089C04EC0A114B104FB
:1083100009F484C0F501618572858BEF9EE00E94AF
:108320009DB261E07FE08BEF9EE00E9460B1B801FA
:108330008BEF9EE00E949DB28BEF9EE00E9487B281
:108340000115110561F1F50180858F70843039F5D3
:108350006185728540E450E0CE0101960E94ACDA5E
:108360000E940AB88823D9F08091D60A811117C0DB
:108370006FE270E0CE0101960E9473DA892B51F40E
:10838000F5012185328543E050E060E4CE0101969D
:108390000E94D23EB801CE0101960E942CB98114F0
:1083A000910409F0ACCF3AC0F40161857285CE0129
:1083B00001960E940D8DCE0101960E94438A88236A
:1083C00049F1E114F10441F040E050E0B701CE0181
:1083D00001960E946D421EC0E12CF12C62960FADF9
:1083E000629763961FAD639764962FAD6497659609
:1083F0003FAD659766964FAD669767965FAD679799
:1084000068966FAD689769967FAD6997CE010196C2
:108410000E941C1ACE0101960E942C8C81E00CC097
:1084200080E00AC0892B09F017CFE12CF12C21CF75
:10843000892B09F011CF07CFC85ADF4F0FB6F89438
:10844000DEBF0FBECDBFDF91CF911F910F91FF9087
:10845000EF90DF90CF90BF90AF909F908F90089556
:108460000F931F93CF93DF938C01EB01209741F083
:1084700060910E0D70910F0DCE010E9449CE02C089
:1084800080E090E020E0AC01BE01C801DF91CF9117
:108490001F910F910C94CAB8FC019281892F82958B
:1084A0008F7019F0823021F016C09F709062928315
:1084B0009B016E3681E078072CF477FF05C020E041
:1084C00030E002C02DE631E02683878130FB80F961
:1084D000878381E0089580E008956F927F928F9264
:1084E0009F92AF92BF92CF92DF92EF92FF920F9343
:1084F0001F93CF93DF93CDB7DEB7EA970FB6F8940B
:10850000DEBF0FBECDBF78AF6FAB5AAF49AF672BA1
:1085100009F4B3C2FA01309719F02081211109C082
:10852000FC012385222329F09C01255F3F4F3AAFB0
:1085300029AF6C01E9ADFAAD309721F4F601A588B9
:10854000B6880AC080818823C9F3CE01C9960E94EB
:108550000D8A5C01892B91F300E010E0EFA8F8ACE4
:108560004701800E911EF4018081882351F0082E6E
:10857000000C990B0E9414DAF40180830F5F1F4FE7
:10858000EDCFE114F10441F1F7018081882321F15D
:108590008D3229F190ED980F9A3008F1853211F162
:1085A0008B3719F1833221F129E1822E2FE0922EAF
:1085B00001E010E0C4010E940FCEAC01B401C7017C
:1085C0000E9428CE892BB1F00F5F1F4FF9E08F0E6C
:1085D000911C0931110571F70FEF1FEF0BC000E07F
:1085E00010E008C008E010E005C00EEF1FEF02C069
:1085F00007E110E061EF7FE08BEF9EE00E9460B149
:108600004AE050E0B8018BEF9EE00E9480B28BEF11
:108610009EE00E9487B219A61AA61BA61CA61DA63C
:108620001EA61FA618AA8BA58F708BA709A785E089
:10863000A816B10451F096E0A916B10459F0A1149E
:10864000B10469F0772473940BC07724739408E124
:1086500010E006C07724739407E110E001C0712C8C
:108660006A2C6A2DCE0189960E944B7429873A871D
:108670004B875C876D877E878F87988B0A301105C3
:108680008CF40830110524F50E3FEFEF1E070CF4B3
:10869000E6C10F3FFFEF1F0709F00CF4EEC1012BFD
:1086A00071F1DDC10731110509F497C108311105D8
:1086B00009F0D5C160E0CE0189960E947374298BC0
:1086C0003A8B4B8B5C8B6D8B7E8B8F8B988F17C00F
:1086D000CE01C7960E94DF3F2BA52F70206A2BA7E3
:1086E000092E000CAA0BBB0B482F8DA79EA7AFA786
:1086F000B8ABE9ACFAAC09A51AA53CA5B7C119827B
:108700001A821B821C828B818F7080668B831982F8
:10871000EFA9F8AD309709F460C08081882309F48F
:108720005CC08FA898ACF4018081882359F08D3209
:1087300049F080538A3030F0FFEF8F1A9F0A98AECD
:108740008FAAEFCFC4010E94D8CD8C016EE270E0F9
:10875000C4010E9473DA009769F0FC0181818033C3
:108760004CF08A3354F4E82E880FFF08F0E3EF1A38
:10877000F10806C0E12CF12C03C099E0E92EF12CA0
:108780006CE270E0C4010E9473DA009719F418AE2D
:108790001FAA03C0019698AF8FABE114F104A1F0BA
:1087A0002AE0209FC001219F900D11241016110670
:1087B0001CF0F194E194F1088C010E0D1F1D012EA7
:1087C000000C220B330B0CC0012E000C220B330BC0
:1087D0008B818F70806A8B8303C000E010E098016A
:1087E00089819A81AB81BC8189A39AA3ABA3BCA3E5
:1087F0000DA31EA32FA338A7662DCE0181960E943C
:108800004B7429833A834B835C836D837E838F8390
:108810009887FBA0F2948FE0F8224E0181E3880E46
:10882000911C00E010E08FA998AD892B71F0033006
:10883000110559F00F5F1F4FCE01C7960E94DF3F11
:10884000F401819391934F01EECFFAE0AF16B1049A
:1088500089F08BE0A816B10411F199E0A916B104D2
:1088600019F5CE0181960E946A76CE0189960E9402
:108870004C42F5C0CE0181960E946A768BA5982F56
:1088800092959F7019F0923021F0E9C08F7080624C
:108890008BA7653610F064E670E06EA7E0C0CE01ED
:1088A00081960E946A7694C081E090E0F11002C047
:1088B00080E090E0800F911F8230910501F11CF45F
:1088C000019741F0CCC08330910549F1049709F438
:1088D00052C0C5C0772051F088E0FE01B196DE019C
:1088E000999601900D928A95E1F7B9C0CE018196D3
:1088F0000E946A76CE0189960E949774B0C019A929
:10890000CE0181960E946A768BA58F7080638BA7BB
:108910006FA788A970FB80F988AB1EA7A0C01BA514
:10892000E9A808A9FBA8CE018196772061F00E94F2
:108930006A761F7010621BA76FA770FB00F908AB67
:10894000EEA6FDA68CC00E946A761F7010621BA75F
:108950006FA770FB00F908ABEEA62F2D30E0AFEF4C
:10896000B0E00E94D8D624E630E040E050E00E941B
:10897000A6D62DA774C01BA5E9A808A9FBA8CE01FF
:108980008196772061F00E946A761F7010621BA7A3
:108990006FA770FB00F908ABEEA6FDA617C00E94FA
:1089A0006A761F7010621BA76FA770FB00F908ABF7
:1089B000EEA62F2D30E0AFEFB0E00E94D8D624E62F
:1089C00030E040E050E00E94A6D62DA76DA97EA918
:1089D000CE0189960E94869442C060E0CE018996BD
:1089E0000E94737429A33AA34BA35CA36DA37EA337
:1089F0008FA398A7FE0131967F0100E010E08FA9B8
:108A000098AD892B71F004301105E9F00F5F1F4F0D
:108A1000CE01C7960E94DF3FF701819391937F01BA
:108A2000EECF0330110521F004301105C1F40BC065
:108A30009D812B8139818BA58F7080648BA73FA787
:108A40002EA79DA70CC09F812D813B8149818BA5BD
:108A50008F7080658BA74FA73EA72DA798ABE9AC79
:108A6000FAAC09A51AA52BA53CA54DA55EA56FA539
:108A700078A9C6010E941C1A02C080E090E0EA9624
:108A80000FB6F894DEBF0FBECDBFDF91CF911F911F
:108A90000F91FF90EF90DF90CF90BF90AF909F909D
:108AA0008F907F906F9008954F925F926F927F9218
:108AB0008F929F92AF92BF92CF92DF92EF92FF92EE
:108AC0001F93CF93DF93EC016A017B019A01AB0105
:108AD000C701B6010E94A2D8882319F061E076E0B0
:108AE00027C046015701E894B7F82FEF3FEF4FE753
:108AF0005FE7C501B4010E94A2D881110DC02FEF1C
:108B00003FEF4FE75FE7C501B4010E943AD5181661
:108B10001CF465E076E00CC02FEF3FEF4FE75FE419
:108B2000C701B6010E9442D81816A4F469E076E0A5
:108B3000CE01DF91CF911F91FF90EF90DF90CF900A
:108B4000BF90AF909F908F907F906F905F904F906D
:108B50000C9484B12FEF3FEF4FE75FECC701B601F4
:108B60000E943AD587FDE2CF20E030E0A901C7019D
:108B7000B6010E943AD587FF0AC06DE2CE010E947D
:108B800059B15C01F7FAF094F7F8F09402C0A12C07
:108B9000B12C2AE037ED43EA5BE3C701B6010E943E
:108BA0002ED72B013C010E9413D86B017C010E943F
:108BB0003FD59B01AC01C301B2010E942DD72B010F
:108BC0003C012AE0B701A601CE010E9499B17C01C7
:108BD000EA0CFB1C6EE2CE010E9459B1E80EF91EB0
:108BE00013E0115021F120E030E040E251E4C301F4
:108BF000B2010E94A0D52B013C010E9413D84B0169
:108C0000A12CB12C2AE0B501A401CE010E9499B19A
:108C1000E80EF91EC501B4010E943FD59B01AC01CD
:108C2000C301B2010E942DD72B013C01DACFC7014D
:108C3000DF91CF911F91FF90EF90DF90CF90BF9089
:108C4000AF909F908F907F906F905F904F9008951E
:108C50000F931F93CF93DF93EC010E9484B18C019B
:108C6000CE010E9487B2800F911FDF91CF911F919B
:108C70000F9108951F93CF93DF93182F6091050DE7
:108C800082EE9CE00E94DD3C612F82EE9CE00E941F
:108C9000F23982EE9CE00E94D63C69E070E080E010
:108CA00090E00E940BA742E06091050D82EE9CE0EF
:108CB0000E94043D82EE9CE00E94A939182F82EEAA
:108CC0009CE00E94A939D12F20E0C22F9E01282BC1
:108CD000C901DF91CF911F9108950F931F93CF93F7
:108CE000DF93182FEB016091F00C8091EE0C9091C6
:108CF000EF0C0E94DD3C8091EE0C9091EF0CDC01BA
:108D0000ED91FC910190F081E02D612F19958E017C
:108D10000C5F1F4F8091EE0C9091EF0CDC01ED91F8
:108D2000FC910190F081E02D699119950C171D07B8
:108D300089F78091EE0C9091EF0C0E94D63C88232D
:108D400019F082E090E002C080E090E0DF91CF91E6
:108D50001F910F9108950F931F93CF93DF93082FC7
:108D6000EB01142F6091F00C8091EE0C9091EF0CC0
:108D70000E94DD3C8091EE0C9091EF0CDC01ED91B6
:108D8000FC910190F081E02D602F19958091EE0CFF
:108D90009091EF0C0E94D63C81111EC0412F609132
:108DA000F00C8091EE0C9091EF0C0E94043DCE01EE
:108DB000810F911D8C018091EE0C9091EF0CDC01E4
:108DC000ED91FC910084F185E02D1995892B39F006
:108DD000C017D10739F403C082E090E010C080E0F2
:108DE00090E00DC08091EE0C9091EF0CDC01ED91C4
:108DF000FC910284F385E02D19958993DCCFDF91F6
:108E0000CF911F910F9108958230910599F038F418
:108E1000009769F00197A1F465E176E013C0833013
:108E2000910559F0049761F467E376E00BC06DE0BB
:108E300076E008C06EE176E005C068E276E002C048
:108E400065E476E08EE59EE00C949DB2EF92FF9291
:108E50001F93CF93DF93C82F7B016091F00C80911B
:108E6000EE0C9091EF0C0E94DD3C8091EE0C909105
:108E7000EF0CDC01ED91FC910190F081E02D6C2F65
:108E800019958091EE0C9091EF0C0E94D63C8823AE
:108E900019F0C2E0D0E002C0C0E0D0E041E0609153
:108EA000F00C8091EE0C9091EF0C0E94043D11E0CB
:108EB0008091EE0C9091EF0CDC01ED91FC9100841F
:108EC000F185E02D1995892B69F08091EE0C909138
:108ED000EF0CDC01ED91FC910284F385E02D1995F6
:108EE000182FE6CFF7011083CE01DF91CF911F91AC
:108EF000FF90EF9008951092910B1092900B1092AA
:108F00008F0B10928E0B0E94413A88E999E390935F
:108F10008D0B80938C0B89E999E390938B0B809355
:108F20008A0B08950F931F93CF93DF93FC018185E4
:108F300092850097C9F08B01EF01DC01ED91FC9166
:108F40000484F585E02D1995892B71F089859A8522
:108F5000DC01ED91FC910480F581E02DB801DF91F9
:108F6000CF911F910F91199480E090E0DF91CF9104
:108F70001F910F910895EF92FF920F931F93CF933C
:108F8000DF93CDB7DEB728970FB6F894DEBF0FBEDC
:108F9000CDBF19821A821B821C821D821E821F82F3
:108FA00018862B812F70E12CF12C02E01A813C8174
:108FB00040E05E816F8178850E941C1A28960FB66A
:108FC000F894DEBF0FBECDBFDF91CF911F910F91FF
:108FD000FF90EF9008950F931F93CF93DF93EC01D1
:108FE000209731F10A811B8188858295807F859544
:108FF00085958595859583FD06C08E819F81009717
:1090000011F00E94EB4788858F70843031F4898598
:109010009A85009711F00E94A0CB888199810097D2
:1090200011F00E94A0CBCE010E94A0CBE801D8CFC6
:10903000DF91CF911F910F9108958F929F92AF92E0
:10904000BF92EF92FF920F931F93CF93DF938C0108
:109050007B0149015A010E9468B6EC01892B09F194
:109060008885807F8360888789869A86AB86BC8660
:1090700088819981009711F00E94A0CBC7010E94BE
:109080001CDA99838883BE01C801DF91CF911F91BB
:109090000F91FF90EF90BF90AF909F908F900C94A6
:1090A000E9B9DF91CF911F910F91FF90EF90BF90A1
:1090B000AF909F908F9008957F928F929F92AF92E2
:1090C000BF92CF92DF92EF92FF920F931F93CF93B5
:1090D000DF93CDB7DEB7A6970FB6F894DEBF0FBE0D
:1090E000CDBF8C01762E942E852E20E2B22ECE019D
:1090F00001967C01FC012B2D11922A95E9F78AEE4D
:1091000093E09AA389A38FEF8BA38CA38DA38EA347
:10911000680183E4C80ED11C43E450E0BE016F5DDA
:109120007F4FC6010E947D7D019609F4B9C081E0A0
:1091300089838A8386E0A82EAB821C82F801648131
:109140007581868197810E9403D76D837E838F838B
:10915000988789869A8680E890E09C878B874CE187
:1091600050E0B701C6010E94D278F7012B2D119271
:109170002A95E9F7480188E0880E911CF401D7018F
:1091800001900D92AA94E1F740E150E0B701C601C9
:109190000E94D278F7011192BA94E9F796E0A92ECD
:1091A000B12C40E250E0B701C6010E94D278F1E054
:1091B000AF1AB108B1F783E6898392E89A8393E501
:1091C0009B838C8385E38D8381E08E837F829DE307
:1091D000988797E099878A8786E0F401DE011B96DD
:1091E00001900D928A95E1F78CE0898B8A8B68E576
:1091F00076E0CE0143960E9487DAF8016385CE01BE
:1092000049960E943FAEF8016485CE014B960E94BC
:109210003FAEF8016585CE014D960E943FAE4EE10E
:1092200050E0B701C6010E94D278F3E07F121EC061
:1092300082E3898384E08A83F80196859B839785FE
:109240009C8390899D8391899E8396E39F838887E1
:10925000828D8987838D8A87848D8B87858D8C8786
:109260004CE050E0B701C6010E94D27887E38983C1
:1092700086E08A8391E09B8393E09C838D838FE0DB
:109280008E838AE38F838BE388878FEF898749E01A
:1092900050E0B701C6010E94D278C6010E94AA7CA4
:1092A000A6960FB6F894DEBF0FBECDBFDF91CF916B
:1092B0001F910F91FF90EF90DF90CF90BF90AF90F4
:1092C0009F908F907F9008952F923F924F925F9240
:1092D0006F927F928F929F92AF92BF92CF92DF92C6
:1092E000EF92FF920F931F93CF93DF9300D000D0A4
:1092F000CDB7DEB78C010E9474CC2FEC37E040E094
:1093000050E00E94A6D6DC01CB010196A11DB11D43
:10931000F80184839583A683B78380839183A28396
:10932000B3835801F3E4AF0EB11CC5010E94717AFA
:1093300064E470E0C5010E947D7C882309F436C195
:109340000E9445A72B013C01812C912CC8018E5B0A
:109350009F4F9E838D8348EEC42E43E0D42EE12C94
:10936000F12C52E0252EAD81BE818C91833009F421
:1093700004C1811120C0F80184819581A681B78143
:109380000196A11DB11D84839583A683B7830E9496
:1093900045A76419750986099709A70196010E94D6
:1093A00084D6A90161E0C8010E945C4881E0AD81DA
:1093B000BE818C93CAC08430F9F4F8018481958110
:1093C000A681B7810196A11DB11D84839583A683D3
:1093D000B7830E9445A76419750986099709A701F3
:1093E00096010E9484D6A90163E0C8010E945C48EE
:1093F000AD81BE812C92A9C0813059F5F80142ADF2
:1094000053AD64AD75AD9E012F5F3F4FC8010E9403
:1094100054AE382EF2E08F1392C089819A81AB81CD
:10942000BC81F80184839583A683B7830E9445A7F6
:109430006419750986099709A70196010E9484D6C7
:10944000A90163E0C8010E945C48AD81BE813C92E5
:109450007CC0823009F079C0F80142AD53AD64ADF3
:1094600075AD9E012F5F3F4FC8010E9454AE382E4C
:10947000F5E08F135DC0E3E0AD81BE81EC93F801B0
:1094800082A193A1A4A1B5A1892B8A2B8B2B41F496
:1094900084E893E0A0E0B0E082A393A3A4A3B5A3E3
:1094A000F80186A197A1A0A5B1A5892B8A2B8B2BAA
:1094B00061F482A193A1A4A1B5A1B695A7959795B2
:1094C000879586A397A3A0A7B1A7F80182A593A526
:1094D000A4A5B5A5892B8A2B8B2BA9F482A193A1D6
:1094E000A4A1B5A1AC01BD0123E076956795579580
:1094F00047952A95D1F7841B950BA60BB70B82A72E
:1095000093A7A4A7B5A7F80186A197A1A0A5B1A587
:1095100086A797A7A0ABB1AB82A593A5A4A5B5A537
:1095200082AB93ABA4ABB5AB88248394912C0DC0D4
:10953000F6E08F1304C0AD81BE811C9206C0BFEF60
:109540003B1203C0ED81FE811082F1E08F16910481
:1095500009F409CF0E9445A7DC01CB0184199509C4
:10956000A609B709F80126A937A940AD51AD2817BA
:1095700039074A075B0708F0F6CEC5010E94717AE9
:10958000F80184819581A681B7810196A11DB11D45
:1095900084839583A683B7830E9445A7F801FE962E
:1095A0006083718382839383C40102C080E090E072
:1095B00026960FB6F894DEBF0FBECDBFDF91CF91D8
:1095C0001F910F91FF90EF90DF90CF90BF90AF90E1
:1095D0009F908F907F906F905F904F903F902F90D3
:1095E00008950F931F93CF93DF93EC0100910E0D1D
:1095F00010910F0DB8010E9449CE209709F440C088
:10960000099608171907E0F10E940AB88823C1F1EA
:109610008091140D9091150D019611F481E090E068
:109620009093150D8093140DE0910C0DF0910D0D9C
:109630008091150D8583E0910C0DF0910D0D8091B9
:10964000140D868360910C0D70910D0D47E050E074
:10965000CE010E9441B8E0910C0DF0910D0DE80F84
:10966000F91F1082AC014450510960910C0D7091AA
:109670000D0D82E8DF91CF911F910F910C9461B88D
:1096800080E0DF91CF911F910F9108951F93CF93A9
:10969000DF931F921F92CDB7DEB76CE271E080E0DE
:1096A00090E00E940BA71FB7F8948091980B81114E
:1096B00027C0E6EDF0E18491E0E9F0E19491E82F34
:1096C000F0E0EE0FFF1FEF5BFF4EA591B491EC9120
:1096D000E92321F461E085E30E9493A561E085E33D
:1096E0000E94C2A58CB580618CBD8CB580648CBD98
:1096F00061E084E30E94C2A561E083E30E94C2A509
:109700008091980B8F5F8093980B1FBF809104010D
:109710008860809304018091040184608093040137
:1097200080910501847080930501CE0101960E940D
:109730001DC689819A810E94B96B67E080E090E044
:109740000E94BFB765E58BE190E00E94BFB765E579
:109750008AE190E00E94BFB70E94B86B80E090E47D
:1097600090939F1180939E1180E090E69093A711B3
:109770008093A61180E098E49093A1118093A011AA
:1097800080E098E69093A9118093A81180E090E57D
:109790009093A3118093A21180E090E79093AB1176
:1097A0008093AA1180E098E59093A5118093A4116D
:1097B00080E098E79093AD118093AC110F900F90DB
:1097C000DF91CF911F910895AF92BF92CF92DF9218
:1097D000EF92FF920F931F93CF93DF931F921F92ED
:1097E000CDB7DEB75C018B016A0179010E94464B5F
:1097F000CE0101960E941DC689819A810E94B96B93
:1098000046E050E062E97BE089E090E00E9490B79A
:10981000C50102960E94A36BC60102960E94B16B1D
:10982000C70102960E94AA6B0E94B86BF801828160
:109830009381A481B5818093DC0C9093DD0CA0937F
:10984000DE0CB093DF0C0F900F90DF91CF911F9142
:109850000F91FF90EF90DF90CF90BF90AF90089561
:10986000CF92DF92EF92FF92CF93DF93CDB7DEB727
:1098700068970FB6F894DEBF0FBECDBFFA012AEE8F
:1098800033E03A8329835FEF5B835C835D831E82D1
:1098900038872F83C280D380E480F580C986DA863A
:1098A000EB86FC863E872D87FB01428153816481D4
:1098B00075814F87588B698B7A8B3C8B2B8BFC0186
:1098C00082819381A481B5818D8B9E8BAF8BB88F64
:1098D0009E012F5F3F4FAE01495F5F4FBE01635F47
:1098E0007F4FCE0143960E94E44B68960FB6F894E2
:1098F000DEBF0FBECDBFDF91CF91FF90EF90DF9025
:10990000CF9008950F931F93CF93DF93CDB7DEB71A
:1099100068970FB6F894DEBF0FBECDBFFB01DC0128
:1099200012964D915D916D917C9115974D8B5E8B4B
:109930006F8B788F8AEE93E09A83898321E0288F5A
:109940000D891E892F89388D0B831C832D833E83BF
:1099500098878F83028113812481358109871A8733
:109960002B873C879E878D874F87588B698B7A8B97
:10997000AE014F5F5F4FBE01695F7F4FCE010D9615
:109980000E94304C68960FB6F894DEBF0FBECDBF74
:10999000DF91CF911F910F910895CF93DF93CDB7B2
:1099A000DEB762970FB6F894DEBF0FBECDBFFC01E5
:1099B00082819381A481B5818F87988BA98BBA8B83
:1099C0002AEE33E03A83298341E04A8B4F85588958
:1099D00069897A894B835C836D837E8338872F8383
:1099E00089879A87AB87BC87BE016F5F7F4FCE01A7
:1099F00007960E94824C62960FB6F894DEBF0FBEA7
:109A0000CDBFDF91CF910895CF92DF92EF92FF9279
:109A10000F931F93CF93DF936C01EB017B0182E0E7
:109A2000E80EF11C00E010E0C601800F911F0E94BB
:109A30005ED6F70181937F010F5F1F4F0430110540
:109A400099F78A81882361F08F3F61F48B818F3F82
:109A500049F48C818F3F31F481E09D819F3F19F45F
:109A600080E001C081E090E0DF91CF911F910F91E4
:109A7000FF90EF90DF90CF900895EF92FF920F93B9
:109A80001F93CF93DF937C018B010E5F1F4FC0E0CC
:109A9000D0E0F80161918F01C7018C0F9D1F0E94DA
:109AA00066D62196C430D105A1F7DF91CF911F91E1
:109AB0000F91FF90EF900895FC01DC018D918111D1
:109AC000FDCF40E050E020E030E08AE09191992322
:109AD00001F1243031055CF59E3271F44F3F5105A0
:109AE00009F02CF5DB01A20FB31F12964C932F5FE8
:109AF0003F4F40E050E0EACF849FD001859FB00DFA
:109B00001124492F990F550B405351094A0F5B1FE0
:109B1000DDCF4F3F510509F054F4243031053CF4BA
:109B2000FB01E20FF31F428381E090E0089580E0A3
:109B300090E008954F925F926F927F928F929F92E2
:109B4000AF92BF92CF92DF92EF92FF920F931F934B
:109B5000CF93DF93CDB7DEB768970FB6F894DEBF2B
:109B60000FBECDBF6C018A015901DC0114968D91A5
:109B70009C911597DC011F968D919C915097DC016B
:109B80001696ED90FC9017972B01770F66087708D3
:109B9000E114F10409F464C1B2E0AB16B10439F088
:109BA00083E0A816B10449F463E676E002C06FE5ED
:109BB00076E0C7010E948F56FC01309709F44AC134
:109BC00081859285A385B48584159505A605B7057D
:109BD00009F040C166E676E0C7010E948F565C013D
:109BE0006BE676E0C7010E948F56D6011296ED9182
:109BF000FC91139762E0828193810E9448B96C01C5
:109C0000003448F4F801FF27EE0FFF1FE15DF24F2B
:109C10000781108502C00FEF1FEF198A1A8A1B8A6D
:109C20001C8A1D8A1E8A1F8A188E8B898F708B8BC7
:109C3000198AA114B10409F43DC0F50180858F7023
:109C40008430C1F5818492849AEFA92E9FE0B92EC9
:109C5000612C712C81149104D1F0B501C4010E94D2
:109C6000FFCD892B51F485E0869DF001879DF00D95
:109C70001124E250F04F64910CC0FFEF6F1A7F0A7D
:109C800085E0A80EB11CA9E06A16710419F761E01D
:109C900070E0B62E862F660F990BAA0BBB0BFC014A
:109CA0003197E930F10590F58827E555FF4F8F4F43
:109CB0000C94FBD68B898F70806A8B8B20E030E010
:109CC0000D8B1E8B2F8B388FBB24B3941FC08B89B9
:109CD0008F70806A14C08B898F70806B10C08B89E5
:109CE0008F70806B8B8B11270BC08B898F70806B73
:109CF0008B8B102F002704C08B898F7080668B8B15
:109D000020E030E00D8B1E8B2F8B388FF701808089
:109D100091800FEF10E020E033E040E150E0BE0121
:109D20006F5F7F4FCE0141960E9451718C0169E3B4
:109D300070E18BEF9EE00E9460B1B8018BEF9EE076
:109D40000E949DB262E370E18BEF9EE00E9460B1E1
:109D50006B2DBB0C770B4AE050E08BEF9EE00E942E
:109D600080B260E370E18BEF9EE00E9460B1B401CD
:109D70008BEF9EE00E949DB28BEF9EE00E9487B227
:109D8000C114D10409F463C0D60118968C918F7068
:109D9000863009F05CC0F701E080F180B701C601B0
:109DA0000E948F566C01009709F451C06FE676E06F
:109DB0000E948F568C010097E9F0DC0119968D9076
:109DC0009D90AD90BC901C976989662321F070E04E
:109DD00080E090E004C0CE0141960E946A7686162B
:109DE0009706A806B90699F1F801618772878387FB
:109DF000948721C067E270E18BEF9EE00E9460B122
:109E0000B7018BEF9EE00E949DB28BEF9EE00E9417
:109E100087B22989222321F030E040E050E006C0DB
:109E2000CE0141960E946A769B01AC016FE676E016
:109E3000C6010E9406BAE988FA880B891C892D8917
:109E40003E894F89588D6FEFC6010E945D4081E0C9
:109E500090E008C0D7011296ED90FC90139798CE31
:109E600080E090E068960FB6F894DEBF0FBECDBFDD
:109E7000DF91CF911F910F91FF90EF90DF90CF90E6
:109E8000BF90AF909F908F907F906F905F904F901A
:109E90000895AF92BF92CF92DF92EF92FF920F930D
:109EA0001F93CF93DF93CDB7DEB728970FB6F89403
:109EB000DEBF0FBECDBF6C01162F5A01DC018D91A4
:109EC0009C911197892B09F442C11496ED91FC9154
:109ED0001597309709F43BC180816F3FB9F484FF37
:109EE00034C14330510509F430C1118112951F70FE
:109EF0006EE071E18BEF9EE00E9460B14AE050E0BD
:109F0000612F8BEF9EE00E94EFB102C084FD1FC164
:109F1000D6011496ED91FC91159701810F701017E1
:109F200069F11396FC906CE071E18BEF9EE00E946A
:109F300060B14AE050E06F2D8BEF9EE00E94EFB1E0
:109F40006AE071E18BEF9EE00E9460B14AE050E070
:109F5000602F8BEF9EE00E94EFB167E071E18BEF25
:109F60009EE00E9460B14AE050E0612F8BEF9EE0DE
:109F70000E94EFB18BEF9EE00E9487B2812F90E0AC
:109F80008D30910508F09CC0FC01D6011496ED902F
:109F9000FC9015978827EC54FF4F8F4F0C94FBD6FD
:109FA000F7019181292F2F70253009F489C0D6013E
:109FB0008D919C91263048F42230A9F463E776E035
:109FC0000E948F56F701608159C0273049F02A302E
:109FD00051F469E776E00E948F56F70160816BC00B
:109FE00062E776E055C060E876E038C065E876E084
:109FF000D6018D919C910E948F56F7012081622F8E
:10A000006170322F309530FB20F921C06AE876E08C
:10A01000D6018D919C910E948F56F701208121FBE2
:10A02000662760F931E0362730FB21F910C060E97E
:10A0300076E0D6018D919C910E948F56F701208188
:10A0400022FB662760F931E0362730FB22F92083B6
:10A0500035C060E876E0D6018D919C910E948F56C4
:10A0600060E02CC066E976E002C06BE976E0F601BC
:10A07000808191810E948F56D7016C9161701EC0C2
:10A0800061EA76E002C067EA76E0F60180819181BC
:10A090000E948F56D7016C91669561700FC06EEA71
:10A0A00076E002C064EB76E0F601808191810E9447
:10A0B0008F56D7016C9162FB662760F9009759F4BF
:10A0C000D6011496ED91FC9115971F708181807FC8
:10A0D000182B11833AC0D6011496ED91FC91159777
:10A0E000B3E0AB16B10411F11F702181207F122B58
:10A0F000118319821A821B821C821D821E821F827A
:10A1000018860B810F700B831982E12CFA801C8159
:10A1100020E03E814F8158850E945D40D601149613
:10A12000ED91FC91159780818F7E0EC081818F709B
:10A13000982F9295907F892B8183D6011496ED916B
:10A14000FC91159780818061808381E001C080E06F
:10A1500028960FB6F894DEBF0FBECDBFDF91CF912A
:10A160001F910F91FF90EF90DF90CF90BF90AF9035
:10A1700008952F923F924F925F926F927F928F92AB
:10A180009F92AF92BF92CF92DF92EF92FF920F9386
:10A190001F93CF93DF93CDB7DEB7CD55D1090FB65F
:10A1A000F894DEBF0FBECDBFDC0114962D913C911B
:10A1B0001597232B09F4DEC13B014C0165969FAF37
:10A1C0008EAF65978EE294E063969FAF8EAF6397F4
:10A1D0006996BFAFAEAF699786E194E067969FAF8F
:10A1E0008EAF67976130710509F454C10CF4BFC19B
:10A1F000643071050CF0BBC1D40112968C9180348F
:10A2000051F128F0823439F108F4B1C1805884301A
:10A2100008F0ADC1A3016FEFC4010E94494FF401E2
:10A2200012811695117003818AEC800F803108F03D
:10A23000A4C16BE676E0808191810E948F567C01FB
:10A24000009709F49AC1DC0118968C918F708530C3
:10A2500009F093C136C16BE676E0D4018D919C91F3
:10A260000E948F568C01F40183819091100F9813F6
:10A2700009C09091110F903429F48091120F9091A0
:10A28000130F0BC08093100F90E49093110F0E9456
:10A29000C7A69093130F8093120F3C01011511056F
:10A2A00009F4E3C0D80118962C912F70253009F0DD
:10A2B000DCC0C8010E94C9B96C968FAF6C9784301E
:10A2C00008F46BC063E0C8010E9448B9FC018185B5
:10A2D00092853AE0D32ED89E9001D99E300D11245C
:10A2E0006B963FAF2EAF6B9762E0C8010E9448B9F2
:10A2F000DC0119968D919C911A97D89E7001D99E78
:10A30000F00C112457010F2C000CCC08DD0861E083
:10A31000C8010E9448B96E969FAF8EAF6E9760E0FD
:10A32000C8010E9448B9FC012184328443845484CA
:10A33000C301072C000CAA0BBB0B9C01AD01221919
:10A340003309440955096B966EAD7FAD6B97CB0110
:10A35000770FAA0BBB0BBC01CD016A197B098C09D5
:10A360009D090E9474D66E96AEADBFAD6E971996DC
:10A370002D913D914D915C911C972219330944090F
:10A3800055090E94A6D6A20EB31EC41ED51E6C96F9
:10A39000BFAD6C97B53099F415C08AE0869D500129
:10A3A000879DB00C11240B2C000CCC08DD08E12C8F
:10A3B000F12CE0E0F8E26B96FFAFEEAF6B9781E037
:10A3C00090E009C064E0C8010E9448B9DC01199618
:10A3D0008D919C911A976B96EEADFFAD6B97AF0187
:10A3E000FF0F660B770B4A155B056C057D0534F492
:10A3F0005A016B0166246A9423E0722EA7010F2C88
:10A40000000C660B770BA416B506C606D70624F417
:10A410005A016B01612C712C6C96FFAD6C97F23078
:10A4200009F021C36301770CEE08FF0860E0C80162
:10A430000E9448B9FC0181859285A385B485C81620
:10A44000D906EA06FB060CF4E9C261E0C8010E94E5
:10A4500048B9FC0181859285A385B4858C159D053D
:10A46000AE05BF050CF4DEC282C02AE0289F500171
:10A47000299FB00C11240B2C000CCC08DD08E12C1A
:10A48000F12C20E038E26B963FAF2EAF6B9781E066
:10A4900090E0E9C2F4018281853059F0863009F0FC
:10A4A00066C061E070E0CE018B5A9F4F0E94E28E41
:10A4B0005EC061E070E0CE018F5A9F4F0E946D69CF
:10A4C00056C08091100F801388C28091110F803484
:10A4D00009F083C28091120F9091130F5C01990FC4
:10A4E000CC08DD0860E0C7010E9448B9FC01818505
:10A4F0009285A385B485A816B906CA06DB060CF4B6
:10A500006AC061E0C7010E9448B955245394FC0118
:10A5100081859285A385B4858A159B05AC05BD050B
:10A520000CF459C0D4011496ED91FC9115978181DA
:10A53000E82FEF708E2F90E0FC013197EC30F105A1
:10A5400008F44BC0F40104811581D8018C9183FB80
:10A55000992790F9951509F43BC2982F907E09F43C
:10A56000CEC1982F907E90528F71892B8C9380E072
:10A5700090E0BBC38FEF9FEFB8C3202F30E0F9010D
:10A58000E455F14E8491F901E55AFF4E0491F90129
:10A59000EF55FF4EF490FF20A1F081110E943DA5E0
:10A5A000EF2DF0E0EE0FFF1FE951FF4EA591B491A2
:10A5B000EC910E2331E020E009F430E0832F922F5C
:10A5C00002C080E090E0212F30E0552453942817FA
:10A5D000390709F4A7CF512CA5CF8827EF53FF4F98
:10A5E0008F4F0C94FBD60E9445A79B01AC014427DA
:10A5F0005527D4011496ED91FC9115978281938192
:10A60000BC0180E090E0AA24AA94BA2CC12CD12CE1
:10A6100018EEE12E13E0F12E00E010E00E941C3E47
:10A62000882309F48FCFF4010081118166E976E077
:10A63000C8010E948F56892B09F0DCC16BE976E0D6
:10A64000C8010E948F56892B09F0D4C1E4C00E9432
:10A6500045A79B01AC0144275527D4011496ED91E1
:10A66000FC91159782819381BC0180E090E0AA243F
:10A67000AA94BA2CC12CD12C1CE2E12EFF24F39415
:10A6800000E010E01AC00E9445A79B01AC014427DE
:10A690005527D4011496ED91FC91159782819381F1
:10A6A000BC0180E090E0AA24AA94BA2CC12CD12C41
:10A6B00016E9E12EF12C00E010E00E941C3E8823F8
:10A6C00009F440CFA30164E0E6C00E9445A79B01C6
:10A6D000AC0144275527D4011496ED91FC911597B0
:10A6E00082819381BC0180E090E0AA24AA94BA2CD4
:10A6F000C12CD12C18EEE12E13E0F12E00E010E079
:10A700000E941C3E882309F41DCFF40100811181B1
:10A7100061EA76E0C8010E948F56892B09F06DC16D
:10A7200067EA76E0C8010E948F56892B09F065C15F
:10A7300072C00E9445A79B01AC0144275527D40154
:10A740001496ED91FC91159782819381BC0180E074
:10A7500090E0AA24AA94BA2CC12CD12C1CE2E12EA0
:10A76000FF24F39400E010E01AC00E9445A79B016B
:10A77000AC0144275527D4011496ED91FC9115970F
:10A7800082819381BC0180E090E0AA24AA94BA2C33
:10A79000C12CD12C16E9E12EF12C00E010E00E9432
:10A7A0001C3E882309F4CECEA30169E074C00E9448
:10A7B00045A79B01AC0144275527D4011496ED9180
:10A7C000FC91159782819381BC0180E090E0AA24DE
:10A7D000AA94BA2CC12CD12C18EEE12E13E0F12E44
:10A7E00000E010E00E941C3E882309F4ABCEF40187
:10A7F000008111816EEA76E0C8010E948F56892B94
:10A8000009F009C164EB76E0C8010E948F56892BDC
:10A8100009F001C1F5C0A3016DE06DC00E9445A71C
:10A820009B01AC0144275527D4011496ED91FC916E
:10A83000159782819381BC0180E090E0AA24AA94BC
:10A84000BA2CC12CD12C1CE2E12EFF24F39400E0A1
:10A8500010E01AC00E9445A79B01AC014427552770
:10A86000D4011496ED91FC91159782819381BC01DE
:10A8700080E090E0AA24AA94BA2CC12CD12C16E92D
:10A88000E12EF12C00E010E00E941C3E882309F428
:10A8900059CEA3016CE0C4010E94494FF401048128
:10A8A00015810E9445A7D80113967C936E93129749
:10A8B00049CE0E9445A79B01AC0144275527D401EE
:10A8C0001496ED91FC91159782819381BC0180E0F3
:10A8D00090E0AA24AA94BA2CC12CD12C18E5E12E20
:10A8E00012E0F12E00E010E00E941C3E882309F4E3
:10A8F00029CEA30160E0C4010E94494F23CE0E94EB
:10A9000045A7F80173836283D40112968C91129744
:10A9100080FF15C0552009F42ACE1496ED91FC91C4
:10A9200015978081886080831496ED91FC9115972E
:10A930006081617070E0C4010E94A58D18CE652D04
:10A9400070E0C4010E94A58DD4011496ED91FC9194
:10A9500015978181552099F08F70823069F028F425
:10A9600081112DC0A30161E024C0853029F087301A
:10A9700031F5A3016AE01DC0A30166E01AC0E82F0B
:10A98000EF708E2F90E0FC013197ED30F105B8F4B7
:10A990008827E353FF4F8F4F0C94FBD6A30162E04F
:10A9A00008C0A30165E005C0A30167E002C0A301E0
:10A9B00060E0C4010E94494F882309F4D8CDD40136
:10A9C0001496ED91FC911597808150FA83F903C09C
:10A9D0008F718066F8018083CACD0093100F80E4E8
:10A9E0008093110F802F0E94C7A69093130F80931E
:10A9F000120F74CDA30163E07ECFA30168E07BCF8B
:10AA000060E976E0C8010E948F56892B09F003CFD8
:10AA1000A30166E070CFA3016BE06DCFC12CD12CF8
:10AA2000760104C0C12CD12C7601C394D4011496B4
:10AA3000ED91FC91159782819381092E000CAA0B50
:10AA4000BB0B8C159D05AE05BF0509F490CDB60175
:10AA5000C4010E94A58DD4011496ED91FC91159727
:10AA6000D382C28284CDD4011496ED91FC911597C6
:10AA700022813381A301421B530B9A0157FF03C06C
:10AA8000319521953109821793071CF480818F71CC
:10AA900012C04081842F829586958770282F30E0E0
:10AAA000263031054CF48F5F982F9295990F907E48
:10AAB000842F8F71892B8083D4011496ED91FC91A2
:10AAC0001597808182958695877090E00597BCF0F8
:10AAD000C701FF0CAA0BBB0BA816B906CA06DB06FA
:10AAE00071F06B962EAD3FAD6B97C901330FAA0B7A
:10AAF000BB0BA816B906CA06DB0609F038CD828161
:10AB000093818615970509F432CDC601B5010E94DF
:10AB100041D520E030E040E251E40E949AD7D62EA1
:10AB2000C72EB82EA92ED40113961C9163E071E1B3
:10AB30008BEF9EE00E9460B14AE050E0612F8BEF06
:10AB40009EE00E94EFB161E071E18BEF9EE00E9418
:10AB500060B14D2D5C2D6B2D7A2D8BEF9EE00E9408
:10AB600054458BEF9EE00E9487B263EB75E0F401E1
:10AB7000808191810E948F5619821A821B821C82C9
:10AB80000B810F7000670B832D2D4D2D5C2D6B2DD0
:10AB90007A2D4D835E836F837887E980FA801C81EC
:10ABA0003E814F8158856FEF0E945D40D4010D9129
:10ABB0001C9163EE75E0C8010E948F567C0168EE1F
:10ABC00075E0C8010E948F568C01009799F1FC0135
:10ABD00080858F70843071F56185728540E450E026
:10ABE000CE0101960E94ACDA6FE270E0CE010196D0
:10ABF0000E9473DA892B61F4D80119962D913C914A
:10AC00001A9743E050E060E4CE0101960E94D23EE4
:10AC1000AE014F5B5F4F6D2D7C2D8B2D9A2D0E94C9
:10AC20006C3F0E940AB8882329F08091D60A8823B5
:10AC300009F453C0E114F10409F447C0F701808519
:10AC40008F70843009F041C061857285CE01019614
:10AC50000E940D8DCE0101960E94438A882389F1BE
:10AC600025961CAE1DAE1EAE1FAE259724962FADA9
:10AC700024972F70206724962FAF24974D2D8D2D6C
:10AC80009C2DAB2DBA2D29968CAF9DAFAEAFBFAF2B
:10AC90002997E12CF12C22960FAD229723961FAD18
:10ACA000239725963FAD259727965FAD2797289642
:10ACB0006FAD289729967FAD2997CE0101960E9406
:10ACC0001C1ACE0101960E942C8CD4011496ED9191
:10ACD000FC911597738262824ACCBE016F5B7F4FF5
:10ACE000CE0101960E942CB9A5CFC35ADF4F0FB6F3
:10ACF000F894DEBF0FBECDBFDF91CF911F910F91B2
:10AD0000FF90EF90DF90CF90BF90AF909F908F908B
:10AD10007F906F905F904F903F902F9008950F938A
:10AD20001F93CF93DF938B01FC01C681D7812097BE
:10AD300059F0B801888199810E9455DA892B21F058
:10AD40000A80DB81C02DF3CFCE01DF91CF911F911F
:10AD50000F9108950C94068164ED72E18EE49EE0FB
:10AD60000E9460B1E0E0F0E01994BF92CF92DF92D0
:10AD7000EF92FF920F931F93CF93DF93CDB7DEB780
:10AD8000A8970FB6F894DEBF0FBECDBF6B01122F90
:10AD9000B32E7A0194E0E2EFF3E0DE011196019028
:10ADA0000D929A95E1F7FE0135968CE1DF011D9237
:10ADB0008A95E9F7AE014F5F5F4F68E0C6010E94D8
:10ADC00032401A8A8091241090912510892B09F421
:10ADD0006BC08BEF9EE00E9487B26AE271E18BEF5D
:10ADE0009EE00E9460B1412F5B2DB7018BEF9EE08A
:10ADF0000E94544568E271E18BEF9EE00E9460B1D1
:10AE0000BE016F5F7F4F8BEF9EE00E949DB266E2B6
:10AE100071E18BEF9EE00E9460B18BEF9EE00E949B
:10AE200087B2BE016F5F7F4F80919810909199100B
:10AE30000E948F566C0120E030E04EEF52EC612F03
:10AE40007B2DC7010E943AD5882371F120E030E0C4
:10AE50004AEA52E4612F7B2DC7010E943AD588232C
:10AE600019F120E030E0A901612F7B2DC7010E947C
:10AE70003AD58823C9F019A21AA21BA21CA20BA1C1
:10AE80000F700067212F812F9B2DD7018DA39EA3CB
:10AE9000AFA3B8A7E9A0FAA01CA13EA14FA158A555
:10AEA0006FEFC6010E945D40A8960FB6F894DEBF12
:10AEB0000FBECDBFDF91CF911F910F91FF90EF900B
:10AEC000DF90CF90BF900895CF93C1E068EE73E01C
:10AED00080E090E00E940BA74AE050E06C2F8EE4E7
:10AEE0009EE00E94EFB1CF5FC43181F7CF9108950A
:10AEF0000F931F93CF93DF93CDB7DEB728970FB68D
:10AF0000F894DEBF0FBECDBF0E9406806DE271E1F6
:10AF10008EE49EE00E9460B1CE0101960E940EADCB
:10AF2000CE0101960E94B8AC0AEE13E01A830983A1
:10AF30001B821C821D821E82CE0107960E941DC6A6
:10AF40008F8198850E94B96B44E050E0BE016D5F2F
:10AF50007F4F81E090E00E9460B70E94B86BCE0105
:10AF600001960E94B8AC1A8309831B821C821D8241
:10AF70001E82CE0107960E941DC68F8198850E9471
:10AF8000B96B44E050E0BE016D5F7F4F85E090E01B
:10AF90000E9460B70E94B86BCE0101960E94B8ACC7
:10AFA00063E571E18EE49EE00E9460B128960FB6E1
:10AFB000F894DEBF0FBECDBFDF91CF911F910F91EF
:10AFC00008955F926F927F928F929F92AF92BF92FD
:10AFD000CF92DF92EF92FF920F931F93CF93DF9365
:10AFE000CDB7DEB76D970FB6F894DEBF0FBECDBFFD
:10AFF00000912410109125100115110509F440C588
:10B000008091D70A8F5F8093D70A6BEB76E0C801F7
:10B010000E948F56909397108093961061EC76E083
:10B02000C8010E948F569093D50A8093D40A60ED90
:10B0300076E0C8010E948F569093C30A8093C20A9B
:10B0400068EC76E0C8010E948F569093D00F8093F1
:10B05000CF0F6DEC76E0C8010E948F569093CE0F13
:10B060008093CD0F009709F4A3C00E94C9B9082F9F
:10B0700010E00115110509F49BC0000F111F000F0E
:10B08000111F8091CA0F9091CB0F892B09F07FC0BF
:10B09000C8010E9408CB9093CB0F8093CA0F1092E7
:10B0A0004410109243101092D20F1092D10F1092B0
:10B0B000421010924610109245107801013082E043
:10B0C00018071CF0E12CA2E0FA2EC70101960E949D
:10B0D00008CB909348108093471090934110809331
:10B0E00040108E0D9F1D90933B1080933A100E944C
:10B0F00045A760933C1070933D1080933E10909351
:10B100003F1080E090E0E0914710F0914810E80F88
:10B11000F91F10820196E816F906ACF782E090E07C
:10B12000909344108093431080E98093C90010925B
:10B13000C8001092CD0083E08093CC008EE0809315
:10B14000CA00F0922F02E0922E0220914710309117
:10B15000481080912E0290912F02820F931F90939E
:10B160003B1080933A10232B09F45AC36DEF72E120
:10B170008EE59EE00E9460B16AE070E0C8010E9426
:10B18000D7B988E29BE9909339108093381061E732
:10B1900074E18EE49EE00E9460B14AE050E0B801A4
:10B1A0008EE49EE00E9480B28EE49EE00E9487B210
:10B1B00063ED76E080912410909125100E948F56C7
:10B1C0008C01009709F442C00E94C9B981112FC3B4
:10B1D0003DC00E94C33F4B015C0169E073E18BEF0E
:10B1E0009EE00E9460B12AE030E0B501A4018BEF3F
:10B1F0009EE00E94E2B18BEF9EE00E9487B265E57F
:10B2000074E18EE49EE00E9460B14AE050E0B60135
:10B210008EE49EE00E9480B28EE49EE00E9487B29F
:10B220000E94C33F6B017C016FE474E18BEF9EE0F1
:10B230000E9460B12AE030E0B701A6018BEF9EE0EA
:10B240000E94E2B18BEF9EE00E9487B20091241031
:10B250001091251067ED76E0C8010E948F569093FB
:10B2600028108093271064E577E0C8010E948F566C
:10B270009093991080939810009709F4B3C120918E
:10B280009A102111AFC1DC011696ED90FC90179732
:10B290008091921090919310892B09F0DDC06DEA96
:10B2A00073E18BEF9EE00E9460B18BEF9EE00E9405
:10B2B00087B20E94C33F4B015C0167EA73E18BEFE9
:10B2C0009EE00E9460B12AE030E0B501A4018BEF5E
:10B2D0009EE00E94E2B18BEF9EE00E9487B281E186
:10B2E00090E00E9408CB8C0188E1F80181831282F2
:10B2F0001082108A17860E947B4710939310009348
:10B300009210012B39F465E973E186E59EE00E9415
:10B3100060B15AC080EA90E00E9408CB9093B30AD3
:10B320008093B20A0E94C33F4B015C0169E873E15C
:10B330008BEF9EE00E9460B12AE030E0B501A401ED
:10B340008BEF9EE00E94E2B18BEF9EE00E9487B2FD
:10B3500088E290E00E9408CB9093AF0A8093AE0AF7
:10B360000E94C33F4B015C016CE773E18BEF9EE0F1
:10B370000E9460B12AE030E0B501A4018BEF9EE0AD
:10B380000E94E2B18BEF9EE00E9487B28091B20AE8
:10B390009091B30A892B31F08091AE0A9091AF0A57
:10B3A000892BB9F40E94C33F4B015C0164E673E151
:10B3B00086E59EE00E9460B12AE030E0B501A4017C
:10B3C00086E59EE00E94E2B186E59EE00E9487B29B
:10B3D0004CC085EB96E59093B10A8093B00A0E9429
:10B3E0007B4780919210909193100E94E73C82EEEF
:10B3F0009CE00E94D63C811132C061E573E18BEF85
:10B400009EE00E948BB20091921010919310C8019F
:10B410000E94E73C40E060EFC8010E94746EC801E2
:10B420000E94D93CE0919210F091931081E08083CA
:10B4300061E373E18BEF9EE00E948BB280919210EA
:10B44000909193100E94E06E882331F065E273E1E1
:10B450008BEF9EE00E948BB281E090E008C067E134
:10B4600073E18BEF9EE00E948BB280E090E0282F8A
:10B47000217020939A10892B31F06FE374E18EE4F0
:10B480009EE00E9460B11092B50A1092B40ACC24DA
:10B49000C394D12CE114F10409F4A4C080919A1052
:10B4A000882309F49FC0D70118968C9118978F7044
:10B4B000863009F093C00D911C91FE0131965F0119
:10B4C0004801F0E18F0E911C3501D8018C910E944A
:10B4D0002140582EF80181810E9421405294E0EFD2
:10B4E0005E228529D5018D935D010E5F1F4F801669
:10B4F000910659F78091B40A9091B50A843191056B
:10B500000CF06CC0880F991FE091AE0AF091AF0A61
:10B51000E80FF91FD182C082A091B40AB091B50A98
:10B5200053E0AA0FBB1F5A95E1F78091B20A9091A0
:10B53000B30AA80FB91F88E0F30101900D928A9514
:10B54000E1F70091B40A1091B50A65ED73E18BEF54
:10B550009EE00E9460B14AE050E0B8018BEF9EE0AF
:10B560000E9480B26EEC73E18BEF9EE00E9460B1AE
:10B570008091B40A9091B50A63E0880F991F6A958B
:10B58000E1F72091B20A3091B30A820F931F0E9413
:10B59000C0C58BEF9EE00E9487B2E091B40AF091A3
:10B5A000B50A73E0EE0FFF1F7A95E1F78091B20ABA
:10B5B0009091B30AE80FF91F8081883231F48091AD
:10B5C0009210909193100E94FA3D8091B40A90914C
:10B5D000B50A01969093B50A8093B40AF701E28008
:10B5E000F38058CF1092C50A1092C40AE0919610C9
:10B5F000F09197103097F9F0C680D780009196109F
:10B60000109197100115110579F0C114D10461F062
:10B61000D60118968C918F708530A1F7C6010E94D3
:10B62000C9B9823078F335C1F8018681978190934A
:10B63000C50A8093C40A8BEF9EE00E9487B2E09116
:10B64000C20AF091C30A309709F46BC08091D70AFF
:10B650008F5F8093D70A068117815E01F8E1AF0EF4
:10B66000B11C96E1692E94E0792E2EE2822E24E020
:10B67000922E0115110509F44FC0D80118968C912E
:10B680008F70863009F044C0198F088F60E070E039
:10B69000C5010E94AB9D8C8D9D8D892BC9F1809138
:10B6A000241090912510892B99F1E88CF98CF701E1
:10B6B00080858F708630B1F463EB75E0C7010E941E
:10B6C0008F56009709F039C1FA82E98260E070E094
:10B6D000CE0101960E94AB9D62E070E0CE01019622
:10B6E0000E94B950EC8DFD8D10821182128213825E
:10B6F0008A8D843008F040C1823008F053C162E086
:10B700008B8D0E94C2A5EC8DFD8D8181807F818310
:10B71000F80102811381ADCF8091D70A81508093C7
:10B72000D70A6AE174E18EE49EE00E9460B162E1B2
:10B7300074E18EE49EE00E9460B181E02091961059
:10B7400030919710232B09F480E00E94FB8069E080
:10B7500074E18EE49EE00E9460B181E02091C20A13
:10B760003091C30A232B09F480E00E94FB806AEF2A
:10B7700073E18EE49EE00E9460B16FEE73E18EE4AF
:10B780009EE00E9460B181E0209127103091281046
:10B79000232B09F480E00E94FB8068EE73E18EE4C5
:10B7A0009EE00E9460B181E02091CF0F3091D00FD8
:10B7B000232B09F480E00E94FB806FED73E18EE49F
:10B7C0009EE00E9460B181E0209198103091991024
:10B7D000232B09F480E00E94FB808EE49EE00E940F
:10B7E00087B20E94C33F6B017C016AED73E18EE476
:10B7F0009EE00E9460B12AE030E0B701A6018EE42D
:10B800009EE00E94E2B18EE49EE00E9487B281E059
:10B810008093CC0F8091D70A81508093D70A30C192
:10B8200066EE72E18EE59EE00E948BB2AACC6FEFCD
:10B83000680FC8010E9448B9DC011996CD90DD90CF
:10B84000ED90FC901C9790911210992359F08091E3
:10B8500070008E7F809370001092121010922A0256
:10B860001092290282E18093280291110E94996D21
:10B870005601C6010E94C16D01E010E0A016B1069C
:10B880000CF4A7CC60E0C8010E94F76D0F5F1F4F5A
:10B89000F5CFDA82C9821B861A86CE0101960E94F4
:10B8A0003B8CCE0101960E94438A8823E1F18A8570
:10B8B0009B850097E1F0DC01ED91FC910484F58516
:10B8C000E02D1995892B49F08A859B85DC01ED9146
:10B8D000FC910284F385E02D19958A859B85DC0116
:10B8E000ED91FC910680F781E02D19951CC060E078
:10B8F00070E0CE0101960E940A8B8C0197FFBDC0BB
:10B90000119501951109AA24A394B12CCE01019699
:10B910000E941F8CE82EF12C8985853009F452C0D5
:10B92000863009F474C0D6011296CD90DC9013973E
:10B93000CE0101960E942C8C61CEFC0120852F70D7
:10B94000253009F0C1CEC680D780C114D10409F4D6
:10B95000C9CEDA82C982B701CE0101960E94AB9DA1
:10B96000ED81FE811082118212821382D60112961D
:10B97000CD90DC901397E9CF8630D9F060F4853014
:10B9800009F0C6CEBC82AB829A828982CE01019632
:10B990000E945591BDCE803439F0823409F0B8CE82
:10B9A00060E003C060E0ACCE62E08B8D0E94C2A577
:10B9B000AFCEBC82AB827A826982CE0101960E94B0
:10B9C0006C90A6CEEF2829F462E0CE0101960E9489
:10B9D000F48B61E0802F0E94C2A560E0802F0E945E
:10B9E00093A567E374E18BEF9EE00E9460B14AE0AB
:10B9F00050E0B8018BEF9EE00E9480B262E374E1F8
:10BA00008BEF9EE00E9460B160E374E131C0902E44
:10BA100061E0802F0E94C2A561E0AB2821F0EA948A
:10BA2000EF2829F403C0EA94EF2809F060E0E62E3D
:10BA3000F12C892D0E9493A56BE274E18BEF9EE0BF
:10BA40000E9460B14AE050E0B8018BEF9EE00E9496
:10BA500080B269E274E18BEF9EE00E9460B14AE03F
:10BA600050E0B7018BEF9EE00E9480B267E274E184
:10BA70008BEF9EE00E9460B156CFA12CB12C46CF37
:10BA80006D960FB6F894DEBF0FBECDBFDF91CF919C
:10BA90001F910F91FF90EF90DF90CF90BF90AF90EC
:10BAA0009F908F907F906F905F900895AF92BF921C
:10BAB000CF92DF92EF92FF920F931F93CF93DF937A
:10BAC000CDB7DEB7CC55D1090FB6F894DEBF0FBEA7
:10BAD000CDBF6C017B015B01AA2488E0B82273FD15
:10BAE0000DC00E94C33F663971058105910530F094
:10BAF0008091941090919510059781F4B701662775
:10BB00007370C6010E94A58B6CEE74E18BEF9EE012
:10BB10000E9460B1AA24AA94BA2CF0C169961CAE06
:10BB20001DAE1EAE1FAE69976D961CAE1DAE1EAE4D
:10BB30001FAE6D9768968FAD68978F7068968FAFC0
:10BB4000689766961FAE669741E0B601CE018B5AA4
:10BB50009F4F0E94B47360E073E0C6010E94DD8BCA
:10BB6000E82AF92A1AAA19AAFE01F39682E1DF014E
:10BB70001D928A95E9F77A961192119286E0DF017B
:10BB80001D928A95E9F7F0FE21C066968FAD669703
:10BB900090E08831910590F4FC018827E652FF4F30
:10BBA0008F4F0C94FBD66AE475E102C066E475E140
:10BBB000CE01835B9F4F0E9408CE08C068E375E109
:10BBC0008BEF9EE00E9460B1E894F0F868968FAD2C
:10BBD000689782958F70813008F45FC0833018F0C9
:10BBE000883009F05AC00E940AB8882309F482C13B
:10BBF0008091D60A81117EC120E030E043E050E020
:10BC000060E3CE0101960E94D23ED601ED91FC91F7
:10BC1000608171814FE250E0CE0101960E948EDA80
:10BC200004E610E020E032E044E150E0BE016F5C49
:10BC30007F4FCE018B5A9F4F0E945171F1FE06C07B
:10BC400066968FAD6697823009F02FC1F0FE25C051
:10BC5000BE01635B7F4FCE0101960E942CB969E261
:10BC600075E18BEF9EE00E9460B1BE016F5F7F4F78
:10BC70008BEF9EE00E949DB266E275E18BEF9EE045
:10BC80000E9460B1BE01635B7F4F8BEF9EE00E941C
:10BC90009DB28BEF9EE00E9487B2F1FE8EC020E045
:10BCA00030E043E050E060E3CE0101960E94D23ED6
:10BCB000D601ED91FC91608171814FE250E0CE019F
:10BCC00001960E948EDA66E675E0CE0101960E942A
:10BCD00068DA68968FAD689782958F70845082304D
:10BCE00018F567E1CE018B5A9F4F0E947374269618
:10BCF0002FAF269727963FAF279728964FAF2897C5
:10BD000029965FAF29972A966FAF2A972B967FAF18
:10BD10002B972C968FAF2C972D969FAF2D970FEFCB
:10BD200010E020E033E004C00FEF10E020E032E04C
:10BD300044E150E0BE016F5C7F4FCE018B5A9F4FB4
:10BD40000E94517140E350E062E275E1CE0101963C
:10BD50000E9418CE6CE175E18BEF9EE00E9460B10D
:10BD6000BE016F5F7F4F8BEF9EE00E949DB269E145
:10BD700075E18BEF9EE00E9460B1BE016F5C7F4F6A
:10BD80008BEF9EE00E949DB28BEF9EE00E9487B2F7
:10BD90000E940AB8882309F4ADC08091D60A8111A7
:10BDA000A9C0BE016F5C7F4FCE0101960E942CB9E5
:10BDB00060E072E0C6010E946B8BF0FE97C0669651
:10BDC0008FAD66978A3059F028F4813071F0863053
:10BDD00061F016C08B3031F08C3059F011C06FE03B
:10BDE00075E109C06AE075E106C0F601808585301D
:10BDF00039F464E175E1CE01835B9F4F0E9408CE68
:10BE000020E030E043E050E060E3CE0101960E9484
:10BE1000D23ED601ED91FC91608171814FE250E0FC
:10BE2000CE0101960E948EDA66E675E0CE0101969B
:10BE30000E9468DA40E350E066E075E1CE010196C9
:10BE40000E9418CE60E075E18BEF9EE00E9460B129
:10BE5000BE016F5F7F4F8BEF9EE00E949DB26DEF42
:10BE600074E18BEF9EE00E9460B1BE01635B7F4F87
:10BE70008BEF9EE00E949DB28BEF9EE00E9487B206
:10BE80000E940AB88823B1F18091D60A811132C08C
:10BE9000BE01635B7F4FCE0101960E942CB960E02A
:10BEA00071E0C6010E946B8B21C0853009F4CECEB3
:10BEB000BE016F5C7F4FCE0101960E942CB962E3F8
:10BEC00075E18BEF9EE00E9460B1BE016F5F7F4F16
:10BED0008BEF9EE00E949DB26FE275E18BEF9EE0DA
:10BEE0000E9460B1BE016F5C7F4FCFCEAA24A394A5
:10BEF000B12C04C0B701C6010E94A58BC501C45A6C
:10BF0000DF4F0FB6F894DEBF0FBECDBFDF91CF91EC
:10BF10001F910F91FF90EF90DF90CF90BF90AF9067
:10BF20000895CF93DF93EC0160E073E00E94DD8B16
:10BF3000009791F0209194103091951026303105A2
:10BF400059F4BC01CE010E94565D60E073E0CE0161
:10BF5000DF91CF910C946B8BDF91CF910895CF92AD
:10BF6000DF92EF92FF920F931F93CF93DF93CDB7A2
:10BF7000DEB728970FB6F894DEBF0FBECDBF6C01B9
:10BF80008B0162E070E00E940A8B7C0119821A82A8
:10BF90001B821C821D821E821F8218868B818F70DD
:10BFA0008B831982F7FC92C040E0B601CE01019666
:10BFB0000E94B47363E070E0C6010E940A8BAC017A
:10BFC0001816190614F04FE350E081E0E816F1046A
:10BFD00021F4012F110F110B04C082E0E816F104C7
:10BFE0000CF411272FEF30E0D8010E9412D79A01EC
:10BFF000550F440B550B0E94A6D68901C6010E941D
:10C000001F8CE82EF12C60E0CE0101960E9469752C
:10C010000817190771F40115110509F45AC082E0D7
:10C02000E816F10489F085E0E816F10409F051C042
:10C030000BC001151105C1F186E0E816F10441F0CD
:10C0400081E0E816F10421F061E0C6010E94F48B62
:10C0500017FD07C00F3F110531F02CF00FEF10E076
:10C0600002C000E010E08B81982F92959F70915054
:10C07000923018F08F7080618B830D8340E0B601A1
:10C08000CE0101960E945C7382E0E816F10421F073
:10C0900085E0E816F10429F460E071E0C6010E9431
:10C0A000565D60E072E00EC085E0E816F10489F0AC
:10C0B00082E0E816F10469F062E0C6010E94F48BA8
:10C0C00060E071E0C6010E94565D03C080E090E030
:10C0D00002C081E090E028960FB6F894DEBF0FBE54
:10C0E000CDBFDF91CF911F910F91FF90EF90DF9027
:10C0F000CF900895CF93DF93EC0163EC74E18BEF65
:10C100009EE00E9460B160E074E0CE01DF91CF91CB
:10C110000C94A58BBF92CF92DF92EF92FF920F9378
:10C120001F93CF93DF93CDB7DEB728970FB6F89460
:10C13000DEBF0FBECDBF7C0109831A832B833C83F6
:10C140004D835E836F837887CE0101960E9455B937
:10C150006C01023011F0053011F4C12CD12C60E0DB
:10C1600070E0C7010E940A8BB82E192F67ED74E1A9
:10C170008BEF9EE00E9460B14AE050E06B2D712F82
:10C180008BEF9EE00E9480B265ED74E18BEF9EE044
:10C190000E9460B14AE050E0B6018BEF9EE00E9441
:10C1A00080B28BEF9EE00E9487B20091291010911F
:10C1B0002A100115110561F041E0B701CE01019689
:10C1C0000E945C73C7010E947A6000E010E061C0C9
:10C1D00081E090E090932A108093291026E040E8B7
:10C1E00055E260E070E08AE99BE00E94FCBCB092FE
:10C1F000310D8AE99BE09093300D80932F0D1092C2
:10C200003C0E10923E0E10923D0E80ED97E0909302
:10C21000B70D8093B60D1092B90D1092B80DC114E0
:10C22000D10439F085E090E09093BB0D8093BA0D76
:10C2300004C01092BB0D1092BA0D86E00E9445BA60
:10C2400062E370E080E090E00E940BA782ED97E04F
:10C250009093B70D8093B60D1092B90D1092B80D52
:10C2600024E62C9DC0012D9D900D11249093BB0DB3
:10C270008093BA0D86E00E9445BA10922A1010925F
:10C280002910882321F0C7010E947A6002C001E0D2
:10C2900010E0C80128960FB6F894DEBF0FBECDBFE0
:10C2A000DF91CF911F910F91FF90EF90DF90CF9092
:10C2B000BF9008952F923F924F925F926F927F921C
:10C2C0008F929F92AF92BF92CF92DF92EF92FF92A6
:10C2D0000F931F93CF93DF93CDB7DEB72E970FB693
:10C2E000F894DEBF0FBECDBF5C0109831A832B8398
:10C2F0003C834D835E836F837887CE0101960E94D5
:10C3000055B94C01023011F0053011F4812C912CFB
:10C31000F50102811381F80180858F70853009F065
:10C3200051C0C8010E94C9B9E82EF12CF2E0EF1605
:10C33000F1040CF447C060E0C8010E9448B9FC0158
:10C34000818592859C878B8761E0C8010E9448B9EE
:10C35000FC014184528463847484809129109091FB
:10C360002A109E878D8792E0E916F10409F44CC0EB
:10C3700062E0C8010E9448B9FC01818592859A87D4
:10C380008987F3E0EF16F10409F442C063E0C801C5
:10C390000E9448B9FC0121843284F4E0EF16F104D4
:10C3A000A1F064E0C8010E9448B9FC01C184D284B4
:10C3B00021143104D1F08D859E85892B51F0C50162
:10C3C0000E947A6080E090E02AC022E0C22ED12C48
:10C3D000EFCF9101D4010E940AD724E630E040E07B
:10C3E00050E00E94A6D6790105C0ED85FE85EF2BB1
:10C3F00031F7740109851A859601A2016B857C8548
:10C40000C5010E94BE940BC0EFEFFFEFFA87E987EA
:10C410008FE3282E312C92E0C92ED12CCCCF2E9632
:10C420000FB6F894DEBF0FBECDBFDF91CF911F9145
:10C430000F91FF90EF90DF90CF90BF90AF909F90C3
:10C440008F907F906F905F904F903F902F900895C6
:10C450008F929F92AF92BF92CF92DF92EF92FF9214
:10C460000F931F93CF93DF93CDB7DEB76F970FB6C0
:10C47000F894DEBF0FBECDBF7C01088F198F2A8FC5
:10C480003B8F4C8F5D8F6E8F7F8FCE0148960E94C1
:10C4900055B96C01D7011296ED91FC9113978085E7
:10C4A0008F70843009F0C9C0B02E61857285CE01CD
:10C4B00001960E940D8DCE0101960E94438A882329
:10C4C00009F449C08985893009F045C060E070E011
:10C4D000CE0101960E940A8BA82E192F63EE74E1FB
:10C4E0008BEF9EE00E9460B14AE050E06A2D712F10
:10C4F0008BEF9EE00E9480B261EE74E18BEF9EE0D4
:10C500000E9460B14AE050E0B6018BEF9EE00E94CD
:10C5100080B26BED74E18BEF9EE00E9460B1602F02
:10C5200070E04AE050E08BEF9EE00E9480B28BEF1B
:10C530009EE00E9487B20091291010912A100115E7
:10C54000110561F041E0B701CE0148960E945C738D
:10C55000C7010E947A6000E010E06AC081E090E0CC
:10C5600090932A108093291026E040E855E260E07D
:10C5700070E08AE99BE00E94FCBCA092310D8AE940
:10C580009BE09093300D80932F0D10923C0E1092F3
:10C590003E0E10923D0EB2E0BB1609F456C085E087
:10C5A000B81609F452C0B601DD0C880B990B0E9435
:10C5B00041D522E538EB42E152E40E942ED720E03B
:10C5C00030E040E251E40E94A0D52DEE3EE94CE37C
:10C5D0005EE30E949AD74B015C0120E030E0A901A4
:10C5E0000E9442D820E030E040E05FE387FD28C0B1
:10C5F000C501B4010E942ED70E940CD883ED97E0AC
:10C600009093B70D8093B60D1092B90D1092B80D9E
:10C610007093BB0D6093BA0D86E00E9445BA1092EC
:10C620002A1010922910882399F0C7010E947A607D
:10C63000CE0101960E942C8C0EC000E010E00BC0D1
:10C64000C501B4010E942DD7D7CF60E070E0D6CFEE
:10C6500001E010E0EDCFC8016F960FB6F894DEBF91
:10C660000FBECDBFDF91CF911F910F91FF90EF9043
:10C67000DF90CF90BF90AF909F908F9008950F93D1
:10C680001F93CF93DF93CDB7DEB76F970FB6F894B4
:10C69000DEBF0FBECDBF8C01188E198E1A8E1B8E79
:10C6A0001C8E1D8E1E8E1F8E8A8D8F708A8F188E07
:10C6B000D801ED91FC91608171818BEF9EE00E9429
:10C6C0009DB2C8010E94438A81110DC06AEB74E1DA
:10C6D0008BEF9EE00E9460B18BEF9EE00E9487B2DC
:10C6E0008FEF9FEFD1C0C8010E941F8CF801908589
:10C6F0009730B1F0853009F491C030F4813049F0C1
:10C70000823009F48BC00CC0863019F08A50833017
:10C7100038F46BE874E18BEF9EE00E9460B1B2C028
:10C72000D80119968D919C911A970097C9F0DC0158
:10C73000ED91FC910688F789E02D199511E000979D
:10C7400009F410E0892B19F06BE874E102C064E988
:10C7500074E18BEF9EE00E9460B1812F90E094C065
:10C7600040E0B801CE0148960E94B473F80180857C
:10C77000873079F038F4833009F45AC0843009F4F2
:10C7800050C05CC0883009F453C0893009F449C0F6
:10C7900055C00280F381E02D80858F70853009F0CF
:10C7A00056C064EB74E18BEF9EE00E9460B1D8014B
:10C7B0001296ED91FC9113970681178101151105D1
:10C7C00069F1F80180858F70843011F5618572857B
:10C7D000CE0101960E940D8DCE0101960E94438AE2
:10C7E000882391F0CE0101960E943F631816190626
:10C7F0005CF46BE874E18BEF9EE00E9460B1CE01C7
:10C8000001960E942C8C3EC0CE0101960E942C8C79
:10C81000D80112960D911C911397D0CF64E974E161
:10C820000FC060E0CE0148960E9469758C0111C06E
:10C83000CE0148960E946A768B010BC06AEA74E1C9
:10C840008BEF9EE00E9460B180E090E01DC000E0B0
:10C8500010E06FE974E18BEF9EE00E9460B14AE066
:10C8600050E0B8018BEF9EE00E9480B28BEF9EE01B
:10C870000E9487B231E020E0012B09F430E0832FE1
:10C88000922F02C081E090E06F960FB6F894DEBF61
:10C890000FBECDBFDF91CF911F910F910895809171
:10C8A000E90F9091EA0F8170992708958091D80F30
:10C8B0009091D90F08956EED76E08EE59EE00E948E
:10C8C00028461092D90F1092D80F81E090E0089579
:10C8D0000E949C9C69EE76E08EE59EE00E942846D0
:10C8E00026E040E855E260E070E087E39CE00E94CB
:10C8F000FCBC81E090E09093D90F8093D80F08950D
:10C90000EF92FF920F931F93CF93DF937C018B01E4
:10C9100001501109A801BC0187E39CE00E9419B0F5
:10C92000F701329660E0CF018E199F0980179107B9
:10C9300018F48191680FF7CF87E39CE00E94A0B0C4
:10C9400087E39CE00E94EDB061EF76E08EE59EE02B
:10C950000E949DB2E701CE018E199F0980179107B1
:10C96000A8F468816A3050F464EF76E08EE59EE0CA
:10C970000E949DB240E150E0688102C040E150E079
:10C980008EE59EE00E94EFB12196E5CF8EE59EE018
:10C99000DF91CF911F910F91FF90EF900C9487B290
:10C9A000CF92DF92EF92FF920F931F93CF93DF937B
:10C9B000CDB7DEB762970FB6F894DEBF0FBECDBF1E
:10C9C0006C010B871C872D873E874F87588B698B9F
:10C9D0007A8B6FEB75E1C7010E94FFCD892BD9F0EF
:10C9E00069EB75E1C7010E94FFCD892BB9F063EBBC
:10C9F00075E1C7010E94FFCD892B99F0ED851E2FAF
:10CA00001F706FEA75E1C7010E94FFCD892B61F0AD
:10CA1000E12FF0E00BC0EDE0F0E008C0EFE0F0E067
:10CA200005C0EEE0F0E002C0E0E1F0E09B85992374
:10CA300009F45CC13097B1F13197EF30F10508F09E
:10CA400041C18827EE50FF4F8F4F0C94FBD6CE018B
:10CA50000B960E946A7670931110609310109B01E0
:10CA60002A5031092531310508F02CC120EF260F5D
:10CA700020930E109B01770F440B550BD601129695
:10CA8000ED91FC9113970190F081E02D608171810F
:10CA9000ED91FC910684F785E02D06EF16E0C601C6
:10CAA000199510C11982892F90E0FC013197EE3061
:10CAB000F10508F085C08827EF5FFE4F8F4F0C947B
:10CAC000FBD68091E90F8160809308106DE070E0E3
:10CAD0008BE192E00E948064D6011296ED91FC9168
:10CAE00013970190F081E02D60817181ED91FC91AF
:10CAF0000288F389E02D2BEF36E040E057E01EC0BE
:10CB00008091E90F8E7F809308106DE070E08EE0D9
:10CB100092E00E948064D6011296ED91FC911397E9
:10CB20000190F081E02D60817181ED91FC9102888E
:10CB3000F389E02D2BEF36E043E057E0C60119956D
:10CB4000D2C0109202108091E90F8160809308108A
:10CB50006AEA75E131C081E0809302108091E90FAB
:10CB600081608093081065EA75E126C082E08093B9
:10CB700002108091E90F81608093081060EA75E1EE
:10CB80001BC084E0809302108091E90F8160809344
:10CB900008106CE975E110C083E08093021067E033
:10CBA00077E08BEF9EE00E949DB28091E90F81605B
:10CBB0008093081063E975E1CE0101960E9408CECA
:10CBC000D6011296ED91FC9113970190F081E02D22
:10CBD00060817181ED91FC910288F389E02D2BEF4A
:10CBE00036E03CC01982903199F040F49C30F9F461
:10CBF00083E0809304106AEA75E10EC0913189F0F8
:10CC00009231A9F482E08093041063E875E104C0D6
:10CC1000109204106EE875E1CE0101960E9408CED4
:10CC20000CC081E08093041067E875E1F5CFCE0178
:10CC30000B960E946A7660930410D6011296ED91CD
:10CC4000FC9113970190F081E02D60817181ED914D
:10CC5000FC910288F389E02D2CE037E0AE014F5FB4
:10CC60005F4FC60119952EC0CE010B960E946A76C1
:10CC70006093021027C0913019F0923061F022C009
:10CC800080E506C0913019F0923029F007C083E0AA
:10CC90008093071017C01092071014C0CE010B9696
:10CCA0000E946A76609306100DC0913031F0923088
:10CCB00049F480910810877F03C080910810886034
:10CCC000809308101092FC0F81E08093F40F8DE4A4
:10CCD0008093F50F8FE58093F60F65E270E08BEEA1
:10CCE0009FE00E94806481E090E00EC0E031F10599
:10CCF00048F78827E15FFE4F8F4F0C94FBD68FEFEC
:10CD00009FEF02C019825CCF62960FB6F894DEBF27
:10CD10000FBECDBFDF91CF911F910F91FF90EF908C
:10CD2000DF90CF9008954F925F926F927F928F9293
:10CD30009F92AF92BF92CF92DF92EF92FF920F93AA
:10CD40001F93CF93DF93CDB7DEB72A970FB6F89432
:10CD5000DEBF0FBECDBF6130710509F09CC24C0132
:10CD60000E9445A79B01AC016091E50F7091E60F11
:10CD70008091E70F9091E80FAA24AA94BA2C65013C
:10CD800018E8E12E13E1F12E00E010E00E941C3EB5
:10CD90008823B9F080E00E94063E6093E50F70930F
:10CDA000E60F8093E70F9093E80F61E177E08EE55F
:10CDB0009EE00E9428466DE070E081E092E00E94D3
:10CDC000806464E670E080E090E00E940BA787E357
:10CDD0009CE00E9474B0181619060CF059C20BEEB4
:10CDE0001FE080E1E82E80E1F82E0E9445A76093C5
:10CDF0003F0C7093400C8093410C9093420C87E35E
:10CE00009CE00E9452B097FF49C20E9445A7409003
:10CE10003F0C5090400C6090410C7090420CDC0133
:10CE2000CB0184199509A609B70940903B0C509095
:10CE30003C0C60903D0C70903E0C84159505A60549
:10CE4000B705E8F287E39CE00E9474B0892B59F0A3
:10CE500062E070E080E090E00E940BA787E39CE036
:10CE60000E9452B0EFCF80910F109091E40F89177C
:10CE700009F40EC28093E40F80910E1090E040966A
:10CE800090931110809310108091F80F90E0909380
:10CE9000E30F8093E20F8091021090E09093E10FF6
:10CEA0008093E00F8091041090E09093DF0F8093C7
:10CEB000DE0F8091061090E09093DD0F8093DC0FE1
:10CEC0008091081090E09093EA0F8093E90F809191
:10CED000071090E09093DB0F8093DA0F80910A1097
:10CEE000F401A281B381208131810D90BC91A02DEC
:10CEF0006D917C91D9015296ED91FC91539729E166
:10CF000037E080FF03C040E057E002C043E057E055
:10CF1000C40119958091DA0F9091DB0F803891054B
:10CF2000A9F4D4011296ED91FC9113970190F08130
:10CF3000E02D60817181ED91FC910288F389E02DF3
:10CF400020E237E040E057E0C40119958091DA0F04
:10CF50009091DB0F892BA9F4D4011296ED91FC91ED
:10CF600013970190F081E02D60817181ED91FC912A
:10CF70000288F389E02D20E237E043E057E0C40166
:10CF8000199566E277E08EE59EE00E949DB26AE028
:10CF900070E08091E90F9091EA0F0E94D7B98091DB
:10CFA000E90FF401A281B381208131810D90BC9100
:10CFB000A02D6D917C91D9015296ED91FC915397E2
:10CFC0002DE237E083FF03C040E057E002C043E0BA
:10CFD00057E0C40119958091E90FF401A281B38152
:10CFE000208131810D90BC91A02D6D917C91D90152
:10CFF0005296ED91FC91539724E337E081FF03C0F3
:10D0000040E057E002C043E057E0C4011995209189
:10D01000DC0F3091DD0F032E000C440B550BD401B7
:10D020001296ED91FC9113970190F081E02D6081B3
:10D030007181ED91FC910684F785E02D00E417E005
:10D04000C40119958091DE0F9091DF0F892BA9F40F
:10D05000D4011296ED91FC9113970190F081E02D8F
:10D0600060817181ED91FC910288F389E02D2CE0C3
:10D0700037E047E457E0C40119958091DE0F9091A5
:10D08000DF0F0197A9F4D4011296ED91FC9113974B
:10D090000190F081E02D60817181ED91FC91028819
:10D0A000F389E02D2CE037E04CE457E0C4011995FA
:10D0B0008091DE0F9091DF0F0297A9F4D4011296B0
:10D0C000ED91FC9113970190F081E02D60817181C9
:10D0D000ED91FC910288F389E02D2CE037E043E5E7
:10D0E00057E0C40119958091DE0F9091DF0F0397EF
:10D0F000A9F4D4011296ED91FC9113970190F0815F
:10D10000E02D60817181ED91FC910288F389E02D21
:10D110002CE037E047E557E0C40119958091DC0F1A
:10D120009091DD0FF401A281B381208131810D90B6
:10D13000BC91A02D6D917C91D9015296ED91FC91FD
:10D14000539720E437E0892B19F443E057E002C0FD
:10D1500040E057E0C4011995209110103091111052
:10D16000032E000C440B550BD4011296ED91FC914B
:10D1700013970190F081E02D60817181ED91FC9118
:10D180000684F785E02D06EF16E0C401199520917D
:10D19000E20F3091E30F2F3F3105B9F0032E000C61
:10D1A000440B550BD4011296ED91FC91139701900D
:10D1B000F081E02D60817181ED91FC910684F7850D
:10D1C000E02D0CE517E0C401199519828091E00F5C
:10D1D0009091E10F009719F46AEA75E11DC0813062
:10D1E000910519F465EA75E117C08230910519F4CB
:10D1F00060EA75E111C08330910519F463E975E1C6
:10D200000BC08430910519F46CE975E105C08D36C9
:10D21000910531F46FE775E1CE0101960E9408CEC9
:10D220002091E00F3091E10F032E000C440B550BC1
:10D23000D4011296ED91FC9113970190F081E02DAD
:10D2400060817181ED91FC910684F785E02D02E605
:10D2500017E0C40119958091E90FF401A281B3810F
:10D26000208131810D90BC91A02D6D917C91D901CF
:10D270005296ED91FC9153972BEF36E080FF04C05E
:10D28000AE014F5F5F4F02C043E057E0C401199504
:10D2900088EE93E00BC080E090E008C0F801819335
:10D2A0008F01EE16FF0609F0A0CDCCCD2A960FB661
:10D2B000F894DEBF0FBECDBFDF91CF911F910F91CC
:10D2C000FF90EF90DF90CF90BF90AF909F908F90A6
:10D2D0007F906F905F904F9008952F923F924F9262
:10D2E0005F926F927F928F929F92AF92BF92CF92F6
:10D2F000DF92EF92FF920F931F93CF93DF93CDB7FF
:10D30000DEB762970FB6F894DEBF0FBECDBF5C01EB
:10D310008091D30F811103C068E675E158C160E0C8
:10D3200083E00E9493A561E070E080E090E00E94BD
:10D330000BA7BE016F5F7F4F80E00E942647892BBD
:10D3400009F043C1898183FF40C144E0BE016F5FA2
:10D350007F4F82E00E94AB46009791F429813A8189
:10D360003227232732273093FC0C2093FB0C2B8190
:10D370003C813227232732273093FA0C2093F90C73
:10D380000E94044768E677E08EE59EE00E949DB229
:10D390006091FB0C7091FC0C80E090E00E943FD506
:10D3A000D62E372E2C01462F572FBC018EE59EE03E
:10D3B0000E9454456EE677E08EE59EE00E949DB2A5
:10D3C0006091F90C7091FA0C80E090E00E943FD5DA
:10D3D000C62E272E898B9A8B462F572FBC018EE5A0
:10D3E0009EE00E94544566E777E08EE59EE00E944D
:10D3F0009DB242E0BE016F5F7F4F81E10E94AB466C
:10D4000049815A81892B21F454274527542702C08A
:10D4100040E050E060E070E04093D40F5093D50FAF
:10D420006093D60F7093D70F2AE030E08EE59EE030
:10D430000E9438B220E030E44CE156E46D2D732DAB
:10D44000C2010E943AD587FF6DC0D5011296ED91B9
:10D45000FC9113970081118162E877E0C8010E9476
:10D460008F563C0166E877E0C8010E948F564C0158
:10D4700019821A821B821C820B810F7000670B833A
:10D480002D2D8D2D932DD2018D839E83AF83B88753
:10D49000E980FA801C813E814F8158856FEFC3017E
:10D4A0000E945D4019821A821B821C820B810F70C0
:10D4B00000670B832C2D8C2D922DA989BA898D8321
:10D4C0009E83AF83B887E980FA801C813E814F81BB
:10D4D00058856FEFC4010E945D402BE837E04D2D69
:10D4E000532DB201C5010E942A9F20E937E04C2D3F
:10D4F000522D69897A89C5010E942A9F4091D40FD3
:10D500005091D50F6091D60F7091D70FCE01019633
:10D510000E94773E46E957E0BE016F5F7F4FC5012D
:10D520000E94F39E6CE977E08EE59EE00E9428461B
:10D53000BE016F5F7F4F80EE0E942647892B19F452
:10D5400019811F3F39F46EE977E08EE59EE00E9475
:10D55000284634C015FF06C06FEB77E08EE59EE0ED
:10D560000E949DB214FF06C063ED77E08EE59EE059
:10D570000E949DB213FF06C066EE77E08EE59EE046
:10D580000E949DB212FF06C06BEF77E08EE59EE031
:10D590000E949DB211FF06C062E178E08EE59EE038
:10D5A0000E949DB210FF06C068E278E08EE59EE022
:10D5B0000E949DB28EE59EE00E9487B261E083E00A
:10D5C0000E9493A581E090E00CC06DE475E18BEFC3
:10D5D0009EE00E9460B18BEF9EE00E9487B280E0E7
:10D5E00090E062960FB6F894DEBF0FBECDBFDF911C
:10D5F000CF911F910F91FF90EF90DF90CF90BF9050
:10D60000AF909F908F907F906F905F904F903F90E2
:10D610002F9008950895CF93DF931F92CDB7DEB773
:10D620006983DC01ED91FC910280F381E02D41E002
:10D6300050E0BE016F5F7F4F19950F90DF91CF9142
:10D640000895DC01ED91FC91068CF78DE02D199584
:10D6500091E089270895862F089581E0862708950F
:10D66000CF93DF931F92CDB7DEB78983209113103C
:10D670003981E0911410F0911510822F90E080957F
:10D680009095F8940080082200824BE000C05DE095
:10D6900000005A95E9F7008008220894379508F4AD
:10D6A000022A00824A9599F778940F90DF91CF91E2
:10D6B00008950F931F93CF93DF931F92CDB7DEB7DB
:10D6C0008C01DC01ED91FC910084F185E02D199530
:10D6D000892B51F0BE016F5F7F4FF80184850E9456
:10D6E000EC7A898190E002C08FEF9FEF0F90DF917D
:10D6F000CF911F910F910895FC0184850C943D7B7F
:10D70000CF93DF931F92CDB7DEB741E050E0BE016B
:10D710006F5F7F4FFC0184850E943D7B18161906C0
:10D720001CF4898190E002C08FEF9FEF0F90DF9192
:10D73000CF910895FC018485843011F00C944379D5
:10D7400080E090E0089544E050E0BC018FE090E07C
:10D750000C9490B744E050E0BC0185E090E00C945C
:10D7600090B744E050E0BC0181E090E00C9490B7A9
:10D7700008958CBD9DBD08956F927F928F929F9268
:10D78000AF92BF92CF92DF92EF92FF921F93CF930F
:10D79000DF931F921F92CDB7DEB75C013B016A0198
:10D7A000FC011485143041F481E090E0F50193838D
:10D7B000828380E090E05BC07A014130584018F0ED
:10D7C000E12C88E0F82ECE0101960E941DC68981C9
:10D7D0009A810E94B96B812F0E9423AE4C0163E0B5
:10D7E00070E0812F0E94CE7A873111F08C3121F4C4
:10D7F0008E149F0440F302C0E12CF12CCE0101965F
:10D800000E941DC689819A810E94B96B9701A3016C
:10D8100060E070E0812F0E94BEAD60E270E0812F79
:10D820000E940DC662E070E0812F0E94CE7A84FDD6
:10D8300014C063E070E0812F0E94CE7A811104C091
:10D84000812F0E94027AB0CFCE0101960E941DC6A0
:10D8500089819A810E94B96BE5CF40E162E070E076
:10D86000812F0E94F879EF2809F49ECFC6010F900E
:10D870000F90DF91CF911F91FF90EF90DF90CF90AD
:10D88000BF90AF909F908F907F906F9008958F92F0
:10D890009F92AF92BF92DF92EF92FF920F931F93EE
:10D8A000CF93DF931F921F92CDB7DEB7FC01248583
:10D8B000243009F082C05A018B017C01D12C8D2DBE
:10D8C0000E945E7C811103C0F701D48607C08B7F64
:10D8D0008831D1F3D394F4E0DF12F1CFF7018485DE
:10D8E000843009F46AC020912B0230912C022F5F02
:10D8F0003F4F11F420E030EC30932C0220932B02A8
:10D9000040912B0250912C0220E061E00E94257A88
:10D91000F80182818F3F51F483818F3F99F4848194
:10D920008F3F81F485818F3F69F444C081110AC023
:10D93000F8018381811106C08481811103C0858132
:10D940008823C1F1A114B104A9F1F701D484CE0157
:10D9500001960E941DC689819A810E94B96BB80107
:10D960006E5F7F4F8D2D0E94057DB5018D2D0E942C
:10D97000F47C64E070E08D2D0E940DC60E9445A7E6
:10D980004B015C01F4E98F0EF1E19F1EA11CB11C5B
:10D99000C7010E9422C6873141F161E070E080E05A
:10D9A00090E00E940BA70E94F87FC7010E9422C648
:10D9B000811106C084E0F701848780E090E01DC0FB
:10D9C0000E9445A786169706A806B90608F7F7012C
:10D9D00084850E94027A84E0F70184876FEC76E107
:10D9E0008EE59EE00E948BB2E8CF64EC76E18EE596
:10D9F0009EE00E948BB281E090E00F900F90DF914B
:10DA0000CF911F910F91FF90EF90DF90BF90AF905B
:10DA10009F908F90089578941F920F920FB60F9257
:10DA200011240BB60F92CF92DF92EF92FF920F93D9
:10DA30001F932F933F934F935F936F937F938F9396
:10DA40009F93AF93BF93CF93DF93EF93FF93809117
:10DA500070008E7F809370000FE310E08BE1E82E62
:10DA6000F12C9BE2C92ED12CC0911610D091171029
:10DA70002097F9F40332110508F43BC00352110951
:10DA8000E0911410F0911510908120911310822FC5
:10DA90008095982390839BE0D7011197F1F79150DF
:10DAA000D9F78081822B8083C6010197F1F780E04E
:10DAB0000DC00B301105E8F00B501109E091181062
:10DAC000F0911910EC0FFD1F319780810E94306B8F
:10DAD0002196D0931710C09316108091290290912F
:10DAE0002A028C179D0708F0BFCF109217101092D2
:10DAF000161080917000816080937000FF91EF910B
:10DB0000DF91CF91BF91AF919F918F917F916F9155
:10DB10005F914F913F912F911F910F91FF90EF9047
:10DB2000DF90CF900F900BBE0F900FBE0F901F9005
:10DB3000189581E08093121080912802282F30E000
:10DB4000F901EF55FF4EE491F0E0EE0FFF1FEE56A6
:10DB5000F14E459154915093151040931410F901D2
:10DB6000E55AFF4EE491E093131061E00E94C2A5D4
:10DB700083E08093B100E0E7F0E080818160808302
:10DB80000895CF93DF931816190644F08091700022
:10DB90008E7F809370001092121019C0EC0180915A
:10DBA0001810909119100E94A0CBCE01C130D24024
:10DBB00014F080E092E090932A02809329020E9460
:10DBC00008CB9093191080931810892B29F4109288
:10DBD0002A021092290208C080911210811104C0FB
:10DBE000DF91CF910C94996DDF91CF910895FF92C1
:10DBF0000F931F93CF93DF938C01F62E8091121019
:10DC0000811102C00E94996DE8012197C11582E03F
:10DC1000D80798F48091290290912A0280179107E1
:10DC200018F4C8010E94C16D8091181090911910CC
:10DC3000009719F0C80FD91FF882DF91CF911F917B
:10DC40000F91FF900895DC0180E0615040F09D91BC
:10DC5000E82FE927F0E0EC53FA4E8491F6CF0895CF
:10DC6000AF92BF92CF92DF92EF92FF921F93CF932A
:10DC7000DF93EC010E9445A76B017C0128EEC20EE8
:10DC800023E0D21EE11CF11C8BE4A82EB12C0E94D3
:10DC900045A76C157D058E059F0598F460EFCE01B4
:10DCA0000E94ED3CCE010E94E33D182F80FF11C081
:10DCB000EF85F889309709F01995C5010197F1F7BB
:10DCC000E6CF81E08A836AE378E08EE59EE00E94F9
:10DCD0002846812FDF91CF911F91FF90EF90DF9029
:10DCE000CF90BF90AF9008950F931F93CF93DF9382
:10DCF000EC01162F042F0E94306E002319F0CE0184
:10DD00000E94FA3DCE010E94E73C65EA82EE9CE06B
:10DD10000E94F239612F82EE9CE00E94F239CE011E
:10DD2000DF91CF911F910F910C94D93CEF92FF920C
:10DD30000F931F93CF93DF938C017B0140E065E548
:10DD40000E94746EE70188E0E80EF11C699140E0E2
:10DD5000C8010E94746ECE15DF05C1F7DF91CF9127
:10DD60001F910F91FF90EF9008951F93CF93DF9332
:10DD7000EC01162F0E94306ECE010E94E73C62ED4E
:10DD800082EE9CE00E94F239612F70E06095709500
:10DD900084E0660F771F8A95E1F7612B82EE9CE0A5
:10DDA0000E94F239CE010E94D93CCE010E94E33D8F
:10DDB000181711F084E08A83DF91CF911F910895A5
:10DDC0001F93CF93DF93EC010E94306E80FD31C032
:10DDD000CE010E94EF3D60E0CE010E94B56ECE0103
:10DDE0000E94306ECE010E94E73C64EB82EE9CE024
:10DDF0000E94F239CE010E94D93CCE010E94306EC1
:10DE0000182F82FF03C082E08A8304C08A81823097
:10DE100009F41A828881882341F0CE010E94EF3DE7
:10DE2000682F6160CE010E94B56E11FB882780F9D2
:10DE300001C080E0DF91CF911F910895CF92DF92D2
:10DE4000EF92FF920F931F93CF93DF937C01EB012F
:10DE50008A01FC01858196810E94E06E8823C9F1C8
:10DE6000BE01F701858196810E94966E40E06EEBBF
:10DE7000F701858196810E94746EE8016801F9E0DE
:10DE8000CF0ED11CF70105811681C8010E94306EAA
:10DE9000C8010E94E73C66E982EE9CE00E94F239EC
:10DEA000C8010E94D93CC8010E94306E61EEC801D1
:10DEB0000E94ED3CC8010E94E33D8993CC16DD062B
:10DEC00009F7F701858196810E94E06E91E081302B
:10DED00009F090E0892FDF91CF911F910F91FF9072
:10DEE000EF90DF90CF900895CF93DF93EA010E94E7
:10DEF0001E6F882339F068E0CE010E94236E91E006
:10DF00002885281390E0892FDF91CF910895CF9332
:10DF1000DF93CDB7DEB729970FB6F894DEBF0FBEFB
:10DF2000CDBFAE014F5F5F4F0E94746F882389F0B1
:10DF30008D818F3361F020F48F3159F489E00CC06A
:10DF40008F3519F08F3739F004C08BE005C08AE0B7
:10DF500003C080E001C08CE029960FB6F894DEBFC4
:10DF60000FBECDBFDF91CF9108956F927F928F92B8
:10DF70009F92AF92BF92CF92DF92EF92FF920F9358
:10DF80001F93CF93DF93FC01248521119EC0872E20
:10DF9000762EEC010E94E06E811108C065E478E005
:10DFA0008EE59EE00E9428468FEF90C0CE010E9431
:10DFB000306E40E060EFCE010E94746EC12CD12C17
:10DFC00066246A94EE24E394F12C0C2D06950695B4
:10DFD000069510E08C2D8770570101C0AA0C8A9518
:10DFE000EAF78B85082E000C990BC816D90634F475
:10DFF000FE01E00FF11F93809A2006C099249394AC
:10E00000C816D90609F0912CCE010E94306ECE01BF
:10E010000E94E73C68E782EE9CE00E94F239911092
:10E0200002C060E001C060E882EE9CE00E94F2392C
:10E03000CE010E94D93CCE010E94306E282F207460
:10E04000982F907885FF11C02223A9F042E050E07C
:10E05000682F8EE59EE00E94EFB161E578E08EE5E5
:10E060009EE00E9428468EEF31C0211104C091111C
:10E0700004C06C2C08C0992331F0FE01E00FF11FA1
:10E0800083818A2907C0FE01E00FF11F8A2D809548
:10E09000938189238383FFEFCF1ADF0A80E4C816B8
:10E0A000D10409F092CF6B86EFEF6E1202C081E0CF
:10E0B0008C87DE011396E72DF82D2B968D91819399
:10E0C000CA17DB07D9F781E001C080E0DF91CF916B
:10E0D0001F910F91FF90EF90DF90CF90BF90AF9086
:10E0E0009F908F907F906F900895AF92BF92CF9244
:10E0F000DF92EF92FF920F931F93CF93DF93CDB7F1
:10E10000DEB7AF970FB6F894DEBF0FBECDBF7C0170
:10E110005B016A010AEE13E01A8309831B821C82E9
:10E120001D821E82CE0109960E9473791BA70AA741
:10E130001CA61DA61EA61FA68091DC0C9091DD0CCE
:10E14000A091DE0CB091DF0C8EA39FA3A8A7B9A766
:10E150008B839C83AD83BE8318861F82AE01465D90
:10E160005F4FB501CE0101960E9451A78130910504
:10E17000B1F4D701ED91FC910684F785E02D1DA344
:10E180000CA38CA59DA5AEA5BFA58EA39FA3A8A7F4
:10E19000B9A7A601BE016C5D7F4FC7011995AF9667
:10E1A0000FB6F894DEBF0FBECDBFDF91CF911F91A8
:10E1B0000F91FF90EF90DF90CF90BF90AF900895B8
:10E1C000FC01848195810895089580E090E0089590
:10E1D000009789F0FC0120852F70253061F40E94A2
:10E1E00048B9009741F0FC0120852F70243019F4C4
:10E1F00081859285089580E090E00895DF92EF9206
:10E20000FF920F931F93CF93DF9300D000D0CDB731
:10E21000DEB761E777E18EE49EE00E9460B102E93B
:10E220001BE0D12C80E1E82EF12CF80180818031B7
:10E2300030F464EF76E08EE49EE00E949DB2F80137
:10E240008081F5E090E0A0E0B0E089839A83AB8321
:10E25000BC83FE82ED82BE016F5F7F4F8EE49EE045
:10E26000DF1639F00E94938D6FE677E10E9460B16E
:10E2700004C00E94938D0E9487B2D3940F5F1F4FFA
:10E2800086E0D812D2CF26960FB6F894DEBF0FBE26
:10E29000CDBFDF91CF911F910F91FF90EF90DF9055
:10E2A00008954F925F926F927F928F929F92AF925A
:10E2B000BF92CF92DF92EF92FF920F931F93CF9373
:10E2C000DF9300D000D0CDB7DEB75C017E836D83D5
:10E2D0007A0149016115710509F45AC141155105C9
:10E2E00009F456C1FB011082FC016081662311F024
:10E2F00030FD54C1CD80DE8091FE4DC1F50182819B
:10E30000E82FE295EF708E2F90E0FC013197EC3012
:10E31000F10508F040C18827E15EFE4F8F4F0C9455
:10E32000FBD6F501248130E0D8010E9412D72FEFEF
:10E3300030E040E050E00E94A6D65F934F933F93B9
:10E340002F938BE598E00BC0F50187818F93868131
:10E350008F9385818F9384818F938EE598E09F932F
:10E360008F93FF92EF92DF92CF920E94C6DA02C1A2
:10E37000F50187818F9386818F9385818F93848127
:10E380008F9382E698E0EBCFF50184809580A6809C
:10E39000B780C501B4012AE030E040E050E00E94BF
:10E3A000A6D697FF07C090958095709561957F4F91
:10E3B0008F4F9F4F9F938F937F936F93C501B401AE
:10E3C0002AE030E040E050E00E94A6D65F934F93F1
:10E3D0003F932F9386E698E0C5C0C5010E946494E0
:10E3E000F501248185809680B78097FF18C030E0C2
:10E3F000D8010E9412D72FEF30E040E050E00E9499
:10E40000A6D65F934F933F932F931F928F92B0FAAC
:10E41000BB24B0F8BF929F9280E798E0A3C09F937F
:10E420008F9330E0D8010E9412D72FEF30E040E008
:10E4300050E00E94A6D65F934F933F932F931F9275
:10E440008F92B0FABB24B0F8BF929F928DE698E00D
:10E450009F938F93FF92EF92DF92CF920E94C6DA42
:10E4600089C0F50185811F928F9396818781817084
:10E470008F939F9383E798E072CFF5018480958016
:10E48000A680B78020E030E0A901C501B4010E9458
:10E490003AD52401350187FF04C077FA709477F8E4
:10E4A0007094C301B2010E940CD869837A838B8374
:10E4B0009C8329813A81B901330F880B990B0E9403
:10E4C00041D59B01AC01C301B2010E942DD720E0D0
:10E4D00030E048EC52E40E94A0D50E9497D80E94F8
:10E4E0000CD8162F072F20E030E0A901C501B40198
:10E4F0000E943AD587FF09C00F931F933A813F933B
:10E5000089818F9389E798E02ACF0F931F93FA812F
:10E51000FF9329812F938AE798E021CFF501848129
:10E520001F928F9385811F928F9386811F928F9365
:10E5300080E798E09F938F93FF92EF92DF92CF92C4
:10E540000E94C6DA17C0F50187811F928F938481DC
:10E550001F928F9385811F928F9386811F928F9335
:10E560008DE698E09F938F93FF92EF92DF92CF9288
:10E570000E94C6DA0FB6F894DEBF0FBECDBF0BC047
:10E58000F50164817581A701C6010E94ACDA03C060
:10E5900080E090E027C08D819E8124C0F9E06F9FCC
:10E5A000B0011124605F704F8D819E810E9436CE34
:10E5B000A70164EC79E08D819E810E948EDAED8165
:10E5C000FE8101900020E9F731972D813E81E21B09
:10E5D000F30B6901CE0EDF1EEE1AFF0A31E0E31ADB
:10E5E000F1088ACE26960FB6F894DEBF0FBECDBFD7
:10E5F000DF91CF911F910F91FF90EF90DF90CF901F
:10E60000BF90AF909F908F907F906F905F904F9052
:10E610000895EF92FF920F931F93CF93DF93CDB79F
:10E62000DEB7A0970FB6F894DEBF0FBECDBF7C015A
:10E630000FEF10E020E033E040E250E0BE016F5FFA
:10E640007F4F0E945171F7016281062F0F70162FC4
:10E6500012951F70BE016F5F7F4F8BEF9EE00E948F
:10E660009DB26CEF76E18BEF9EE00E9460B14AE0D4
:10E6700050E0612F8BEF9EE00E94EFB165EF76E1F5
:10E680008BEF9EE00E9460B14AE050E0602F8BEF7C
:10E690009EE00E94EFB18BEF9EE00E9487B2A096B1
:10E6A0000FB6F894DEBF0FBECDBFDF91CF911F91A3
:10E6B0000F91FF90EF900895EF92FF920F931F93A9
:10E6C000CF93DF936115710551F0E42EEB018C01BE
:10E6D000CB010E94438AF82E811103C03DC0F12C6A
:10E6E0003BC0EC81FD813097B1F080858F70825006
:10E6F000823088F4D80114964D915D916D917C9192
:10E7000017974187528763877487EC81FD818085E5
:10E71000807F82608087EC81FD81309769F0808501
:10E72000982F9F708EEF890F823030F4D8011296A7
:10E730008C91807F892B8087EE2029F0F801608101
:10E74000CE010E94F48B6EEE76E18BEF9EE00E948C
:10E7500060B1C8010E9409738F2DDF91CF911F9185
:10E760000F91FF90EF900895AF92BF92CF92DF92FA
:10E77000EF92FF920F931F93CF93DF936115710573
:10E7800051F0A42E7B01EC01CB010E94438AB82EEC
:10E79000811103C074C0B12C72C0F701C480D58050
:10E7A000F6010085C114D10409F441C0802F8F7097
:10E7B0009EEF980F923038F4102F159515951595FA
:10E7C000159589F434C0853091F560E0C6010E944A
:10E7D00048B9009761F1FC011085159515951595BF
:10E7E000159529F104C0823071F4F60107C060E08C
:10E7F000C6010E9448B9009731F0FC0181859285DD
:10E80000A385B48503C080E090E0DC018C839D8308
:10E81000AE83BF831295107F8A818F70182B1A8365
:10E82000AA2069F1C7010E941F8C888328C0029525
:10E83000007F0595059505950595023099F0033003
:10E8400009F0A9CFF60161857285838594850E94C0
:10E8500041D52A812F7020672A836C837D838E8324
:10E860009F830DC0F60141855285638574858A8139
:10E870008F70806A8A834C835D836E837F838B2D48
:10E88000DF91CF911F910F91FF90EF90DF90CF908C
:10E89000BF90AF900895CF93DF93CDB7DEB72897A1
:10E8A0000FB6F894DEBF0FBECDBFFC016F70828142
:10E8B000807F682B628388E0DE01119601900D92C3
:10E8C0008A95E1F729813A814B815C816D817E8156
:10E8D0008F81988528960FB6F894DEBF0FBECDBF06
:10E8E000DF91CF910895CF93DF93CDB7DEB728970F
:10E8F0000FB6F894DEBF0FBECDBFFC01608398E079
:10E90000DE01119601900D929A95E1F729813A81E5
:10E910004B815C816D817E818F81988528960FB6B1
:10E92000F894DEBF0FBECDBFDF91CF9108950F9356
:10E930001F93CF93DF93CDB7DEB728970FB6F89428
:10E94000DEBF0FBECDBF8C0177FD06C065367105F9
:10E950002CF064E670E002C060E070E0F8018281B3
:10E96000982F92959F709150923018F08F7080611F
:10E9700082832FEF30E0DB010E9412D724E630E0E3
:10E9800040E050E00E94A6D6F801248388E0DE0132
:10E99000119601900D928A95E1F729813A814B8178
:10E9A0005C816D817E818F81988528960FB6F89461
:10E9B000DEBF0FBECDBFDF91CF911F910F910895A4
:10E9C000CF92DF92EF92FF920F931F93CF93DF933B
:10E9D000CDB7DEB760970FB6F894DEBF0FBECDBFE0
:10E9E000FC01028102950F70202F30E0862F90E00D
:10E9F0002817390711F488E04FC0162F6F0162EE17
:10EA000076E18BEF9EE00E9460B14AE050E0602F1B
:10EA10008BEF9EE00E94EFB16FED76E18BEF9EE011
:10EA20000E9460B14AE050E0612F8BEF9EE00E94AF
:10EA3000EFB16DED76E18BEF9EE00E9460B1F601E3
:10EA4000008119861A861B861C861D861E861F86D7
:10EA5000188A1295107F6B856F70162B1B8709879C
:10EA6000EE24EA94FE2C1181228133814481558168
:10EA700066817781CE0109960E949695F6012083E2
:10EA80003183428353836483758386839783C6016E
:10EA90000E94097388E0F601DE01119601900D9243
:10EAA0008A95E1F729813A814B815C816D817E8174
:10EAB0008F81988560960FB6F894DEBF0FBECDBFEC
:10EAC000DF91CF911F910F91FF90EF90DF90CF904A
:10EAD0000895CF92DF92EF92FF92FC01362F928140
:10EAE00092959F70963009F47AC020F4915092303C
:10EAF00070F1A5C09730B9F19A50923008F09FC0DC
:10EB000084819581A681B781662399F0B7FD9DC068
:10EB10008F3F9105A105B10529F024F08FEF90E01A
:10EB2000A0E0B0E02FEF30E0A901481B590BCA016B
:10EB30008EC0B7FD87C08F3F9105A105B10509F0D3
:10EB40000CF485C08FEF90E0A0E0B0E080C064815D
:10EB5000332331F02FEF30E0C901861B910977C0D4
:10EB6000862F90E074C0C480D580E680F78066234D
:10EB7000E9F020E030E0A901C701B6010E943AD5D2
:10EB800087FD63C020E030E04FE753E4C701B601E2
:10EB90000E9442D818160CF455C0A701960160E0F7
:10EBA00070E08FE793E40E942DD715C020E030E09D
:10EBB000A901C701B6010E943AD587FD43C020E0F4
:10EBC00030E04FE753E4C701B6010E9442D818165F
:10EBD000E4F1C701B6010E940CD8CB0138C06481B2
:10EBE0007581868197813323B1F0673F5FEF7507A9
:10EBF0008507950754F161152AE072078105910593
:10EC00000CF526EF3FEF4FEF5FEF0E94A6D6C9014C
:10EC100081509F4F1CC0673F4FEF740784079407D4
:10EC20008CF061155AE075078105910574F42AE0AE
:10EC300030E040E050E00E94A6D6C90108C08FEF46
:10EC40009FEF05C080E090E002C08FEF90E0FF9062
:10EC5000EF90DF90CF900895FC014281E42FE29580
:10EC6000EF704E2F50E0FA013197EB30F10570F55F
:10EC7000DC018827E55DFE4F8F4F0C94FBD6149680
:10EC80006D917D918D919C9117970EC014966D9109
:10EC90007D918D919C9117972AE030E040E050E003
:10ECA0000E94A6D6CA01B9010E9441D508951496C2
:10ECB0006C9170E080E090E00E943FD5089514963A
:10ECC0006D917D918D919C911797089560E070E012
:10ECD000CB010895CF93DF93EC018A81E82FE29571
:10ECE000EF708E2F90E0FC013197EB30F10520F5AD
:10ECF0008827EA5CFE4F8F4F0C94FBD66C817D8198
:10ED00008E819F811CC06C8170E080E090E017C014
:10ED10006C817D818E819F810E940CD810C06C8196
:10ED20007D818E819F812AE030E040E050E00E94AA
:10ED3000A6D6CA01B90103C060E070E0CB01DF9143
:10ED4000CF910895FC019281892F807E803241F01D
:10ED5000907F81E0903431F0903521F080E008958B
:10ED600081E008950895AF92BF92CF92DF92EF9223
:10ED7000FF920F931F93CF93DF93CDB7DEB7C154AC
:10ED8000D1090FB6F894DEBF0FBECDBF5C016B0199
:10ED90008A016CE677E18BEF9EE00E9460B1B501DD
:10EDA0008BEF9EE00E949DB269E677E18BEF9EE0DB
:10EDB0000E9460B1C114D10409F4A1C00C0D1D1D45
:10EDC000F80110820E94C33F6A3F71055CF46CE554
:10EDD00077E186E59EE00E9460B186E59EE00E94B4
:10EDE00087B28DC07601E016F10641F0F70161911E
:10EDF0007F018BEF9EE00E9459B1F5CF8BEF9EE033
:10EE00000E9487B280919410909195109E012F5F7F
:10EE10003F4F790120E030E0059719F443E050E0DE
:10EE200019C042E050E061E4C7010E94D23EF70100
:10EE300001900020E9F731978F010E191F09A801F1
:10EE4000B701C5010E949EDA0097A9F020E030E0EA
:10EE500041E050E061E4C7010E94D23EF701019019
:10EE60000020E9F731978F010E191F09A801B7019A
:10EE7000C5010E949EDA892B39F061E577E18BEFBD
:10EE80009EE00E9460B13BC00A0D1B1D62E878E065
:10EE9000C8010E947EDA892B69F4F60101900020F6
:10EEA000E9F73197EC19FD09329720F0C6010E946D
:10EEB0008BA225C06FE270E0C8010E9473DA5C018A
:10EEC000009741F0FC01108281818432C1F0FFEF94
:10EED000AF1ABF0AF8018081843289F0B801C701F6
:10EEE0000E940D8DC7010E94438A882329F0A50145
:10EEF000B601C7010E946D42C7010E942C8CCF5BF6
:10EF0000DF4F0FB6F894DEBF0FBECDBFDF91CF91BC
:10EF10001F910F91FF90EF90DF90CF90BF90AF9037
:10EF20000895CF92DF92EF92FF920F931F93CF93AA
:10EF3000DF93CDB7DEB767970FB6F894DEBF0FBE8D
:10EF4000CDBF8091241090912510892B09F4CFC05A
:10EF50006CE377E18BEF9EE00E9460B18BEF9EE067
:10EF60000E9487B28091D70A8823E9F00E9400A30B
:10EF700080919A10882341F0809198109091991077
:10EF8000892B11F00E94EC2E0E94289E80919410F3
:10EF900090919510059711F00E94D6330E944C92E3
:10EFA0000E94E932DFCF66E277E18BEF9EE00E94BC
:10EFB00060B18BEF9EE00E9487B2E0919610F091D5
:10EFC0009710068117818091961090919710892B48
:10EFD00071F10115110559F1D80118968C918F70B6
:10EFE000853009F5C8010E94C9B98823E1F0D8012C
:10EFF0006D917C91CE0101960E940D8DCE010196FE
:10F000000E94438A882359F08A859B85009739F0AE
:10F01000DC01ED91FC910284F385E02D1995CE0180
:10F0200001960E942C8CF80102811381CCCF1092A2
:10F03000C50A1092C40A6EE177E18BEF9EE00E9450
:10F0400060B18BEF9EE00E9487B20E94C33F6B01CC
:10F050007C0166E077E18BEF9EE00E9460B12AE0E0
:10F0600030E0B701A6018BEF9EE00E94E2B18091F3
:10F070002410909125100E94EB47109225101092B9
:10F0800024101092C30A1092C20A10929710109284
:10F0900096101092D50A1092D40A1092D00F1092A6
:10F0A000CF0F1092CE0F1092CD0F10929910109298
:10F0B000981010922810109227100E94C33F6B01E5
:10F0C0007C0161E077E18BEF9EE00E9460B12AE075
:10F0D00030E0B701A6018BEF9EE00E94E2B18BEF1A
:10F0E0009EE00E9487B21092CC0F1092400A679661
:10F0F0000FB6F894DEBF0FBECDBFDF91CF911F9149
:10F100000F91FF90EF90DF90CF9008950895CF93E7
:10F11000DF931F92CDB7DEB76983DC01ED91FC91DF
:10F120000280F381E02D41E050E0BE016F5F7F4F30
:10F1300019950F90DF91CF910895FC01818D928DEB
:10F140000895FC018489958908952AEE33E0FC0135
:10F1500031832083FB014089518962897389FC01D5
:10F1600042835383648375830895DC01ED91FC91A0
:10F17000048CF58DE02D199480E00895FC019485B0
:10F18000FB018485981303C081E0943009F480E08A
:10F19000089521E0FC018485843009F420E0822F69
:10F1A000089508958F929F92AF92BF92DF92EF924F
:10F1B000FF920F931F93CF93DF931F921F92CDB7B0
:10F1C000DEB77C014B018A01FC01A688B788D08C90
:10F1D000CE0101960E941DC689819A810E94B96B59
:10F1E0008D2D0E9423AE8017910720F48D2D0E9453
:10F1F00023AE8C019801A401B5018D2D0E94BEADF6
:10F200000E94B86BF70186899789800F911F978BB1
:10F21000868BC8010F900F90DF91CF911F910F91B6
:10F22000FF90EF90DF90BF90AF909F908F900895E8
:10F23000CF93DF93FC0124852430D1F0EC010E94B0
:10F2400022C6843181F0882371F0883161F08C31DD
:10F2500061F4E881F9810084F185E02DCE011995F2
:10F2600021E0892B19F420E001C021E0822F01C0A8
:10F2700080E0DF91CF9108958EBD00000DB407FEB0
:10F28000FDCF8EB50895DF92EF92FF920F931F93FB
:10F29000CF93DF931F921F92CDB7DEB7D82ECE014A
:10F2A00001960E941DC689819A810E94B96BE12C4A
:10F2B000F12C8D2D0E94DAB78C01892B21F08D2D38
:10F2C0000E94DAB77C010E151F0599F70E94B86BF2
:10F2D000C8010F900F90DF91CF911F910F91FF9078
:10F2E000EF90DF900895FC011382128288EE93E084
:10F2F000A0E0B0E084839583A683B7838CE494E098
:10F30000918380838AEE93E097878687108A118A9B
:10F31000128A138A84E0808F0895AF92BF92CF92B1
:10F32000DF92EF92FF920F931F93CF93DF93CDB7AE
:10F33000DEB7AF970FB6F894DEBF0FBECDBF7C012E
:10F340005B016A010AEE13E01A8309831B821C82A7
:10F350001D821E82CE0109960E9473791BA70AA7FF
:10F360001CA61DA61EA61FA68091DC0C9091DD0C8C
:10F37000A091DE0CB091DF0C8EA39FA3A8A7B9A724
:10F380008B839C83AD83BE8318861F82AE01465D4E
:10F390005F4FB501CE0101960E9451A781309105C2
:10F3A000B1F4D701ED91FC910488F589E02D1DA3FE
:10F3B0000CA38CA59DA5AEA5BFA58EA39FA3A8A7B2
:10F3C000B9A7A601BE016C5D7F4FC7011995AF9625
:10F3D0000FB6F894DEBF0FBECDBFDF91CF911F9166
:10F3E0000F91FF90EF90DF90CF90BF90AF90089576
:10F3F0009B0190E00496982F8827642F820F931F1B
:10F400000C94BFB71F93CF93DF931F921F92CDB77A
:10F41000DEB7182FCE0101960E941DC689819A8100
:10F420000E94B96B60E170E0812F0E940DC64FEF22
:10F4300062E070E0812F0E94F8790E94B86B0F9013
:10F440000F90DF91CF911F910895DF92EF92FF927D
:10F450000F931F93CF93DF931F921F92CDB7DEB709
:10F46000182FD62E7A01022F0E94027ACE01019621
:10F470000E941DC689819A810E94B96B4D2D402B37
:10F4800060E070E0812F0E94F879E114F10459F4F2
:10F49000E0902210F09023108FEFE81AF80AF09213
:10F4A0002310E09222104F2D64E070E0812F0E9423
:10F4B000F8794E2D65E070E0812F0E94F87961E0C7
:10F4C00070E0812F0E940DC60E94B86B81E00F9002
:10F4D0000F90DF91CF911F910F91FF90EF90DF90F0
:10F4E0000895CF93DF93FC01808D843029F0EF01E4
:10F4F0000E94027A84E0888FDF91CF910895CF92A5
:10F50000DF92EF92FF920F931F93CF93DF931F929F
:10F510001F92CDB7DEB7FC01F484F4E0FF1699F139
:10F520008C01CE0101960E941DC689819A810E949C
:10F53000B96B68E070E08F2D0E940DC60E94B86B19
:10F540000E9445A76B017C01C8010E9422C6882346
:10F55000B9F062E370E080E090E00E940BA70E94A7
:10F5600045A7DC01CB018C199D09AE09BF09883E76
:10F570009340A105B10540F3F80184850E94027A09
:10F5800084E0F80184870F900F90DF91CF911F9155
:10F590000F91FF90EF90DF90CF900895CF93DF937E
:10F5A00090E00496982F8827EC01C60FD71F0E9481
:10F5B0005AB78FE00E943C798D2F0E943C798C2FA6
:10F5C0000E943C7980E00E943C79C82F0E9454B789
:10F5D0008C2FDF91CF910895CF92DF92FF920F93FE
:10F5E0001F93CF93DF931F921F92CDB7DEB7F82EF4
:10F5F0006B01CE0101960E941DC689819A810E94ED
:10F60000B96B68E270E08F2D0E94CE7A082F10E06F
:10F6100069E270E08F2D0E94CE7A702F6627682BEA
:10F6200021E030E0A6018F2D0E9476AD0E94B86BDC
:10F6300081E090E00F900F90DF91CF911F910F919B
:10F64000FF90DF90CF900895CF93DF931F92CDB7B7
:10F65000DEB7FC01218D328D232B49F0BE016F5F97
:10F660007F4F808D0E94EC7A898190E002C08FEFFD
:10F670009FEF0F90DF91CF9108958F929F92BF924D
:10F68000CF92DF92EF92FF920F931F93CF93DF936E
:10F690001F921F92CDB7DEB7B82E6B017A01CE0153
:10F6A00001960E941DC689819A810E94B96B812CA6
:10F6B000912C8B2D0E94DAB78C01892B21F08B2D98
:10F6C0000E94DAB74C010815190599F701151105C3
:10F6D00099F463E070E08B2D0E94CE7A8431D9F1E9
:10F6E0008823C9F101E010E08C3111F400E010E052
:10F6F0001195019511092FC0E016F1060CF4870150
:10F700001016110644F568E270E08B2D0E94CE7A47
:10F71000E82EF12C69E270E08B2D0E94CE7AFE2C4F
:10F72000EE24E82A9801A601B7018B2D0E9476AD40
:10F73000E00EF11E4F2D68E270E08B2D0E94F879EB
:10F740004E2D69E270E08B2D0E94F87960E470E044
:10F750008B2D0E940DC60E94B86BC8010F900F90B0
:10F76000DF91CF911F910F91FF90EF90DF90CF909D
:10F77000BF909F908F900895CF93DF93FC01218DD0
:10F78000328D2115310519F48FEF9FEF11C0EC0177
:10F790004217530708F0A901888D0E943D7B181677
:10F7A000190694F7298D3A8D281B390B3A8F298F2A
:10F7B000DF91CF9108950F931F93CF93DF931F9203
:10F7C000CDB7DEB7FC01218D328D232B61F08C018A
:10F7D00041E050E0BE016F5F7F4F808D0E943D7B16
:10F7E000181619061CF08FEF9FEF08C0F801818DE5
:10F7F000928D0197928F818F898190E00F90DF9198
:10F80000CF911F910F9108950F931F93CF93DF9383
:10F81000CDB7DEB728970FB6F894DEBF0FBECDBFC9
:10F820008C01D80159968D919C915A97892B41F062
:10F83000ED91FC910284F385E02DC8011995F1CF7B
:10F84000F801808D0E9443791816190654F548E096
:10F8500050E0BE016F5F7F4FD80158968C910E9497
:10F860003D7B18161906FCF4D801509684E0FE0181
:10F87000319601900D928A95E1F78D8190E0982F55
:10F8800088272E81820F911DF801958B848B8F81A3
:10F8900090E0982F88272885820F911D928F818F65
:10F8A00002C080E090E028960FB6F894DEBF0FBE4D
:10F8B000CDBFDF91CF911F910F9108951F93CF93EB
:10F8C000DF931F921F92CDB7DEB7182FCE0101969E
:10F8D0000E941DC689819A810E94B96B63E070E025
:10F8E000812F0E94CE7A182F0E94B86B812F0F9023
:10F8F0000F90DF91CF911F910895EF92FF921F9388
:10F90000CF93DF93FC01208D243011F080E01CC0E8
:10F910007B01EC0110E0812F0E945E7C811102C00E
:10F92000188F05C08831E1F31F5F1430A1F7888D6F
:10F93000843061F3FD86EC861A8E198E20E0A701D3
:10F9400062E00E94257A81E0DF91CF911F91FF90C4
:10F95000EF9008951F93CF93DF931F921F92CDB71F
:10F96000DEB7FC01108DCE0101960E941DC6898173
:10F970009A810E94B96B60E270E0812F0E940DC6EF
:10F9800062E070E0812F0E94CE7A84FD1DC062E0AB
:10F9900070E0812F0E94CE7A83FF0BC048E162E0C5
:10F9A00070E0812F0E94F8790E94B86B80E090E0AF
:10F9B00015C00E94B86BCE0101960E941DC68981B8
:10F9C0009A810E94B96BDCCF40E162E070E0812F48
:10F9D0000E94F8790E94B86B81E090E00F900F9040
:10F9E000DF91CF911F910895CF93DF93C82FD62F2A
:10F9F000472F60E170E00E94F8794D2F61E170E0DF
:10FA00008C2FDF91CF910C94F87990E0982F882774
:10FA100044E050E0845F9B4F0C9490B7BF92CF922C
:10FA2000DF92EF92FF920F931F93CF93DF9300D05B
:10FA300000D0CDB7DEB7FC01208D243009F04CC0DA
:10FA40006A017B018C01B12C63E070E08B2D0E9478
:10FA5000CE7A811103C0F801B08E06C08831D9F387
:10FA6000B394F4E0BF12F0CFF801808D8430A1F19F
:10FA700096E0E2E4F4E0DE01119601900D929A9591
:10FA8000E1F7F70193819F779C8394819D83958112
:10FA90009E83B7016E5F7F4F0E94057DB601F8011E
:10FAA000808D0E94F47CF801808D90E0982F88274B
:10FAB00046E050E0BE016F5F7F4F8A5F9B4F0E9420
:10FAC00090B7F801128E118E20E8A60162E0808DB9
:10FAD0000E94257A81E001C080E026960FB6F89456
:10FAE000DEBF0FBECDBFDF91CF911F910F91FF9071
:10FAF000EF90DF90CF90BF900895DF92EF92FF924A
:10FB00000F931F93CF93DF931F921F92CDB7DEB752
:10FB1000FB01DC0157961C921E92569722812111FF
:10FB200009C02381211106C02481211103C0258130
:10FB30002223F1F041155105D9F07A018F01FC0122
:10FB4000D08CCE0101960E941DC689819A810E94A7
:10FB5000B96BB8016E5F7F4F8D2D0E94057DB70197
:10FB60008D2D0E94F47C0E94B86B81E090E002C071
:10FB700080E090E00F900F90DF91CF911F910F9157
:10FB8000FF90EF90DF900895A8950895E5E0F1E0EB
:10FB900080818F7980830895E5E0F1E0808180663F
:10FBA00080830895CF92DF92EF92FF920F931F937D
:10FBB000CF93DF936C01EB0109900020E9F72197C7
:10FBC000C61BD70BC032D10514F0CFE1D0E08B01BA
:10FBD000E12CF12CEC16FD0664F4F80161918F0123
:10FBE000C7018C0D9D1D0E9466D6FFEFEF1AFF0A1C
:10FBF000F1CF60E0C6018C0F9D1FDF91CF911F9167
:10FC00000F91FF90EF90DF90CF900C9466D6CF933A
:10FC1000DF931F92CDB7DEB71982892B21F0FB014C
:10FC20006281738103C0BE016F5F7F4F86E390E006
:10FC30000E94D27D6BE178E18EE49EE00E9460B18B
:10FC40000F90DF91CF910895CF93DF93C0E0D0E084
:10FC500060E0CE010E9466D62196CD34D105C1F771
:10FC60006CE486E490E00E9466D668E487E490E065
:10FC70000E9466D663E488E490E00E9466D666E45B
:10FC800089E490E00E9466D66BE078E18EE49EE025
:10FC9000DF91CF910C9460B1EF92FF920F931F937D
:10FCA000CF93DF931F92CDB7DEB78B01CE010196C4
:10FCB0009F938F9387E99BE09F938F9386E99BE0C7
:10FCC0009F938F9385E99BE09F938F9384E99BE0BB
:10FCD0009F938F9383E99BE09F938F9382E99BE0AF
:10FCE0009F938F938BE898E09F938F93FB01838181
:10FCF0008F9382818F930E9432DB0FB6F894DEBF20
:10FD00000FBECDBF06977CF4F801028113816DE22E
:10FD100078E186E59EE00E9460B1B80186E59EE04C
:10FD20000E949DB219C00E94FE7082E9E82E8BE00D
:10FD3000F82E00E010E0F70161917F01C8010E94F8
:10FD400066D60F5F1F4F06301105A9F76FE378E104
:10FD50008EE49EE00E9460B10F90DF91CF911F91E1
:10FD60000F91FF90EF900895EF92FF920F931F93E2
:10FD7000CF93DF93CDB7DEB72C970FB6F894DEBFE5
:10FD80000FBECDBF8C017B018AEE93E09A838983FD
:10FD90001B821C821D821E8298878F8319861A8679
:10FDA0001B861C86053011055CF0BE01695F7F4F24
:10FDB000F701808591850E945C4D892B09F052C026
:10FDC000BE016F5F7F4F82E190E00E943D4D0430A5
:10FDD00011050CF44FC0BE01695F7F4FF7018681AA
:10FDE00097810E945C4D892B09F444C0BE01695F74
:10FDF0007F4F8EE090E00E943D4DBE01695F7F4FD6
:10FE0000F701848195810E945C4D892BF1F1BE013F
:10FE1000695F7F4F8AE090E00E943D4DBE01695FBF
:10FE20007F4FF701828193810E945C4D892BC1F144
:10FE3000BE01695F7F4F86E090E00E943D4D64EF18
:10FE400077E18EE49EE00E9460B12C960FB6F894A4
:10FE5000DEBF0FBECDBFDF91CF911F910F91FF90FD
:10FE6000EF900895BE01695F7F4F82E190E00E94AC
:10FE70003D4DB1CFBE016F5F7F4F8EE090E00E949D
:10FE80003D4D033011050CF0B8CFBE016F5F7F4FC1
:10FE90008AE090E00E943D4D023011050CF0BECF8B
:10FEA000BE016F5F7F4F86E090E00E943D4D0130C4
:10FEB000110529F6BE016F5F7F4F86E090E00E943A
:10FEC0003D4D6BEF77E18EE49EE00E9460B1B7CFCD
:10FED000CF93DF93CDB7DEB72C970FB6F894DEBF84
:10FEE0000FBECDBF1C821B821E821D828FEF9FEF33
:10FEF00098878F8384E794E09A8389838CE490E0E9
:10FF00009A8789871C861B866AED77E18EE49EE0DE
:10FF10000E9460B16091241070912510CE0101966D
:10FF20000E945CA36FEFCE0101960E948FB46AEC31
:10FF300077E18EE49EE00E9460B12C960FB6F894B3
:10FF4000DEBF0FBECDBFDF91CF910895CF93DF937A
:10FF5000CDB7DEB769970FB6F894DEBF0FBECDBF41
:10FF60008FE290E09A838983FE01339687E1DF0177
:10FF70001D928A95E9F765EB77E18EE49EE00E9499
:10FF800060B1AE014E5F5F4F66E082E99BE00E9488
:10FF900032401E866FE978E0CE0101960E9468DA51
:10FFA000BE016F5F7F4F8BEF9EE00E949DB2CE013E
:10FFB00001960E94F14A1E8667EA78E0CE0101961A
:10FFC0000E9468DABE016F5F7F4F8BEF9EE00E9458
:10FFD0009DB261EB78E0CE0101960E9430426996B5
:10FFE0000FB6F894DEBF0FBECDBFDF91CF9108955D
:10FFF0008091D60A8F5F8093D60AA8950E94E93235
:020000021000EC
:100000008091D60A81508093D60A089567EE7AE1EE
:100010008EE49EE00E9460B164ED7AE18EE49EE0A1
:100020000E9460B166EC7AE18EE49EE00E9460B1CD
:100030006EEB7AE18EE49EE00E9460B18EE49EE079
:100040000E9487B26EEA7AE18EE49EE00E9460B17F
:1000500061EA7AE18EE49EE00E9460B161E97AE1B2
:100060008EE49EE00E9460B165E87AE18EE49EE055
:100070000E9460B16EE67AE18EE49EE00E9460B17B
:100080006CE57AE18EE49EE00E9460B167E47AE17B
:100090008EE49EE00E9460B168E37AE18EE49EE027
:1000A0000E9460B169E27AE18EE49EE00E9460B154
:1000B00061E27AE18EE49EE00E9460B160E17AE163
:1000C0008EE49EE00E9460B165E07AE18EE49EE0FD
:1000D0000E9460B16BEF79E18EE49EE00E9460B116
:1000E00063EF79E18EE49EE00E9460B167EE79E112
:1000F0008EE49EE00E9460B16DEC79E18EE49EE0BA
:100100000E9460B16EEA79E18EE49EE00E9460B1E7
:1001100069E979E18EE49EE00E9460B16CE879E1E2
:100120008EE49EE00E9460B16EE779E18EE49EE08D
:100130000E9460B162E779E18EE49EE00E9460B1C6
:100140006AE679E18EE49EE00E9460B16FE579E1B4
:100150008EE49EE00E9460B162E579E18EE49EE06B
:100160000E9460B16AE479E18EE49EE00E9460B191
:100170006FE379E18EE49EE00E9460B18EE49EE040
:100180000C9487B2AF92BF92CF92DF92EF92FF9220
:100190000F931F93CF93DF936C017B018A010E9421
:1001A0005ED681508E3FA0F45701C0E0D0E00150F0
:1001B0001109C017D1077CF4C6018C0F9D1F0E9446
:1001C0005ED6F50181935F01882329F02196F1CF56
:1001D00080E090E005C0CE0DDF1D188281E090E048
:1001E000DF91CF911F910F91FF90EF90DF90CF9013
:1001F000BF90AF900895882319F068E478E102C0B9
:100200006AE478E18EE49EE00C9460B1CF93DF93D2
:10021000CDB7DEB72C970FB6F894DEBF0FBECDBFBB
:100220006AE977E18EE49EE00E9460B18EE49EE090
:100230000E9487B28CE490E00E945ED68B37D1F5A5
:100240001C821B821E821D828FEF9FEF98878F83F7
:1002500084E794E09A8389838CE490E09A87898785
:100260001C861B860E949177CE0101960E94ECC5E8
:100270009093251080932410892B49F46DE777E142
:1002800086E59EE00E9460B186E59EE01BC066E7C1
:1002900077E18EE49EE00E9460B18EE49EE00E94D1
:1002A00087B20E94E15783E09FE00E947F7A81E05D
:1002B00090E00CC069E877E18EE49EE00E9460B1B6
:1002C0008EE49EE00E9487B280E090E02C960FB60C
:1002D000F894DEBF0FBECDBFDF91CF910895AF92EE
:1002E000BF92CF92DF92EF92FF920F931F93CF9323
:1002F000DF93CDB7DEB7C058D1090FB6F894DEBF93
:100300000FBECDBF8E010F5B1F4FD8011D921C92F7
:10031000FE01ED5BFF4F2EE1DF011D922A95E9F70B
:100320000297CCF0FB01628173814FE150E0C8017C
:100330000E94ACDAB80186E190E00E94D27DB8015B
:100340008EE49EE00E949DB268E379E18EE49EE037
:100350000E9460B11BC040E250E0B80186E190E02D
:100360000E94C280892BB1F440E250E06CE279E156
:10037000C8010E9436CE6EE079E18EE49EE00E94D4
:1003800060B1B8018EE49EE00E949DB28EE49EE0D2
:100390000E9487B28091970B1F928F938091960B4A
:1003A0001F928F938091950B1F928F938091940B46
:1003B0001F928F938091930B1F928F938091920B3A
:1003C0001F928F9383EB98E09F938F931F9280E40B
:1003D0008F93CE0101966C019F938F930E94C6DA92
:1003E0006AEF78E18EE49EE00E9460B1B8018EE48D
:1003F0009EE00E949DB2B6018EE49EE00E949DB2F6
:100400008EE49EE00E9487B27E0191E6E90EF11C27
:10041000D70113961C921E92129788EE93E0A0E0EB
:10042000B0E0F70184839583A683B78384E0848753
:1004300084EC93E09183808316870587108A178662
:1004400080E590E0928B818B158A6AE175EB8BE9F0
:1004500096EB0E949ACE8C010FB6F894DEBF0FBEC9
:10046000CDBF892BE1F183E090E00E9408CBD80159
:100470001D969C938E931C97FC01F182E082128260
:10048000C7010E941879882319F0C7010E947F7A5A
:10049000D7011F966D917C9150975196AD90BC906D
:1004A00052976115710569F0CE0189589F4F0E94DE
:1004B0009FB2A501BE0169587F4FC7010E94476CDA
:1004C00007C0F70165857685A501C7010E94757093
:1004D000181619060CF478C0C8010E9474B600E022
:1004E00010E0F701E388F4880115110509F463C0F1
:1004F000F8ECEF16F10409F04CC06EEE78E18EE4F2
:100500009EE00E9460B1EB961FAE1EAEEB97ED969B
:100510001FAE1EAEED978FEF9FEFEF969FAF8EAFA2
:10052000EF978AE894E0E9969FAF8EAFE997C158BC
:10053000DF4F19830883CF57D040F8940E949177FA
:10054000CE0189589F4F0E94ECC59093251080934F
:1005500024107894C8010E9474B680912410909160
:100560002510892B29F467ED78E186E59EE027C008
:100570006CEC78E18EE49EE00E9460B10E94E1574D
:1005800065EC78E18EE49EE00E9460B184E090E04A
:10059000BBC06DEA78E186E59EE00E9460B14AE06A
:1005A00050E0B70186E59EE00E9480B286E59EE0BD
:1005B0000E9487B206C06AE978E18BEF9EE00E9454
:1005C00060B18EE090E0A0C0D7011D96BC901D9751
:1005D0001E96AC90DF92CF9286E998E19F938F931D
:1005E0001F930F930E9423CFDF92CF9281E998E16E
:1005F0009F938F931F930F930E9423CFD8011C9634
:10060000ED91FC911D9781E08283DF92CF928EE87D
:1006100098E19F938F931F930F930E9423CFD8014C
:100620001C96ED91FC911D971282AF92BF9288E5C6
:1006300098E19F938F931F930F930E9423CF83E999
:1006400098E19F938F931F930F930E9423CFF701FD
:10065000148A138AD8011C96ED91FC911D97A080F5
:10066000B1800FB6F894DEBF0FBECDBF83E3C82EB6
:10067000D12CD501ED91FC910084F185E02DC501CF
:10068000199541975CF4B1E0CB1AD10839F064E1D7
:1006900070E080E090E00E940BA7EBCF6E01F7E7DF
:1006A000CF0ED11CDF92CF928CE498E19F938F9371
:1006B0001F930F930E9440CF0F900F900F900F90B9
:1006C0000F900F90019709F00CCFF6018081918176
:1006D000D70154969C938E935397D12C80E08A3007
:1006E00039F4BAE0DB1609F4FCCE9AE0D92E03C047
:1006F0008D3009F0D82EC8010E94E5CE8F3F79F7E2
:10070000C8010E9474B6EDCEC058DF4F0FB6F89402
:10071000DEBF0FBECDBFDF91CF911F910F91FF9034
:10072000EF90DF90CF90BF90AF9008950E946F81BF
:10073000909395108093941083E09FE00C947F7ABF
:10074000089584E090E00895DC011496ED91FC9109
:100750001597309729F08081082E000C990B089589
:1007600080E090E008950895DC011296ED91FC91EF
:100770001397309779F016968D919C911797833047
:10078000910549F0049719F421E030E006C0208576
:1007900030E003C0089522E030E0C901089580915F
:1007A0002B1090912C1008950C94A0CB0C94A0CBFE
:1007B0000C94A0CB66E17BE18BEF9EE00E9460B1E0
:1007C0008BEF9EE00E9487B210922C1010922B109B
:1007D00081E090E008950E949C9C69E07BE18BEFB2
:1007E0009EE00E9460B18BEF9EE00E9487B281E0A4
:1007F00090E090932C1080932B1008958F929F92ED
:10080000AF92BF92CF92DF92EF92FF920F931F931E
:10081000CF93DF93CDB7DEB728970FB6F894DEBF3E
:100820000FBECDBF09831A83122F2B833C834D83C8
:100830005E836F837887B7011F70C12ED12CDC01D6
:100840001496ED90FC9015976115710569F0FB0108
:100850008081882349F0D7011F968D919C915097F4
:100860000E948F56892B51F5D7011F96ED91FC916F
:100870005097E680F780812E912CA12CB12CE114A9
:10088000F104E1F06FE078E0C7010E948F56FC01AF
:1008900090859F70923049F481859285A385B485B7
:1008A00088159905AA05BB0549F062EE78E0C701F5
:1008B0000E948F56F701E280F380E1CFF980FF209C
:1008C000A1F1C114D10419F0113089F503C0CC2471
:1008D000C394D12C8FEF8F0D823020F16AE77CE139
:1008E0008BEF9EE00E9460B14AE050E06F2D8BEFED
:1008F0009EE00E94EFB18BEF9EE00E9487B26AE615
:100900007CE18BEF9EE00E9460B14AE050E0B601CE
:100910008BEF9EE00E9480B28BEF9EE00E9487B238
:1009200080E001C081E090E014C01130B9F21130D4
:1009300068F467E87CE18BEF9EE00E9460B12B8158
:10094000207F81E090E029F480E003C01230B9F309
:10095000D6CF28960FB6F894DEBF0FBECDBFDF917D
:10096000CF911F910F91FF90EF90DF90CF90BF90AC
:10097000AF909F908F9008954F925F926F927F9269
:100980008F929F92AF92BF92CF92DF92EF92FF929F
:100990000F931F93CF93DF93EC01EC81FD8183854F
:1009A0009485892B21F485859685892B89F1809101
:1009B000291090912A10892B59F5E881F981048436
:1009C000F585E02DCE0119954C0181E08816910442
:1009D000F9F4EC81FD8145805680612C712C0E94D8
:1009E00045A79B01AC01EC81FD8167817085818504
:1009F0009285AA24AA94BA2C6501830172010E94EF
:100A00001C3E81111AC004C010922A1010922910A5
:100A1000EC81FD8185819681DF91CF911F910F91AE
:100A2000FF90EF90DF90CF90BF90AF909F908F900E
:100A30007F906F905F904F900895EA81FB810190C5
:100A4000F081E02D0081118164E67CE18BEF9EE076
:100A50000E9460B1B8018BEF9EE00E949DB28BEFC7
:100A60009EE00E9487B290922A1080922910EC8119
:100A7000FD8141815281052E000C660B770B23818D
:100A80008AE99BE00E94FCBCEC81FD81038114811A
:100A9000618172814AE050E08BEF9EE00E9480B25B
:100AA00060E67CE18BEF9EE00E9460B1A80160E00F
:100AB00070E02AE08BEF9EE00E9499B18BEF9EE000
:100AC0000E9487B260E070E08A819B810E940A8B5D
:100AD0008093310D8AE99BE09093300D80932F0D28
:100AE00010923C0E10923E0E10923D0EEC81FD8154
:100AF0006385748542E050E0CE010E94A2A4EC819F
:100B0000FD816585768543E050E0CE010E94A2A478
:100B10000C811D8180E00E94063EF801678370878A
:100B200081879287EA81FB810190F081E02D00812D
:100B3000118167E57CE18BEF9EE00E9460B1B80116
:100B40008BEF9EE00E949DB28BEF9EE00E9487B2E9
:100B50000E9445A72B013C010E9445A79B01AC01C7
:100B6000AA24AA94BA2C650112E3E12EF12C00E02C
:100B700010E0C301B2010E941C3E811145CF0E94CA
:100B8000C933EACFCF93DF93EC0169EE78E08EE5CD
:100B90009EE00E9428468C819D810E94A0CB60E04F
:100BA00070E08A819B810E944F8A1D821C8281E0B5
:100BB00090E0DF91CF9108958F929F92AF92BF9274
:100BC000CF92DF92EF92FF920F931F93CF93DF9319
:100BD000EC010E949C9C8C819D81892B59F481E1C0
:100BE00090E00E9408CBBC018A819B810E944F8AC1
:100BF0009D838C830C811D810115110559F466E1DB
:100C00007CE186E59EE00E9460B186E59EE00E9460
:100C100087B2B7C180E00E94063ED80117966D9357
:100C20007D938D939C931A970C811D81CA80DB80E4
:100C30000115110509F42CC1C114D10409F428C10E
:100C4000F601E280F380E114F10409F421C1D70137
:100C500018968C918F70853009F01AC1C7010E94D7
:100C6000C9B9823008F414C161E0C7010E9448B9D3
:100C7000FC0190859F70943029F4C184D284C11402
:100C8000D10439F46DEB7BE186E59EE00E9460B112
:100C900066C1B60180912710909128100E948F564E
:100CA0007C01009761F461EA7BE186E59EE00E94A9
:100CB00060B1B60186E59EE00E949DB250C168EF2A
:100CC00078E00E948F56009709F445C0FC0120850A
:100CD0002F70243009F03FC0A184B284B5018BEF9E
:100CE0009EE00E949DB26DE97BE18BEF9EE00E9449
:100CF00060B185E5882E8BE1982EC12CD12CA114F2
:100D0000B104E9F0B401C5010E94FFCD892B69F45B
:100D100086E08C9DF0018D9DF00D1124E75AF44E74
:100D200025913491922F832F12C0FFEFCF1ADF0A43
:100D300086E0880E911CACE0CA16D10401F768E386
:100D40007BE18BEF9EE00E9460B196E080E0F801CD
:100D50009383848307C086E090E0D80114969C9327
:100D60008E9313976FEF78E0C7010E948F56EC8146
:100D7000FD810097A9F0DC0118962C9118972F702F
:100D8000223071F419964D915D916D917C911C9773
:100D9000411551056105710519F05283418304C065
:100DA00080E895E29283818341815281052E000C77
:100DB000660B770B23818AE99BE00E94FCBC64E010
:100DC00079E0C7010E948F566C010C811D8100974C
:100DD00079F1FC0180858F70863051F569E079E00A
:100DE000C6010E948F56D8011C969C938E931B9728
:100DF0006EE079E0C6010E948F56F80196878587DC
:100E000062E179E0C6010E948F56009749F0DC014B
:100E100019968D919C911A97F8019683858311C03C
:100E200088EE93E0D80116969C938E93159709C08F
:100E3000F8011486138688EE93E0968385831686E0
:100E4000158668E179E0C7010E948F56D801509657
:100E50009C938E931F97EA81FB810190F081E02D96
:100E60000081118160E07CE18EE49EE00E9460B12F
:100E7000B8018EE49EE00E949DB28EE49EE00E9446
:100E800087B2EC81FD8181E0808381E090E07BC0CE
:100E9000F601A280B380C5010E94C9B9E82ED50130
:100EA00018968C918F70FF24F394853009F4F12CFF
:100EB00067ED7BE186E59EE00E9460B161E070E055
:100EC000012B11F460E070E04AE050E086E59EE01E
:100ED0000E9480B265ED7BE186E59EE00E9460B1F4
:100EE00061E070E0CD2811F460E070E04AE050E08D
:100EF00086E59EE00E9480B263ED7BE186E59EE0A0
:100F00000E9460B161E070E0AB2811F460E070E035
:100F10004AE050E086E59EE00E9480B261ED7BE110
:100F200086E59EE00E9460B16F2D70E04AE050E0DF
:100F300086E59EE00E9480B26FEC7BE186E59EE054
:100F40000E9460B161E070E0B1E0BE1510F460E0B5
:100F500070E04AE050E086E59EE00E9480B286E5BF
:100F60009EE00E9487B26CEE7BE186E59EE00E94E7
:100F700060B186E59EE00E9487B2EC81FD8182E04F
:100F8000808380E090E0DF91CF911F910F91FF90DF
:100F9000EF90DF90CF90BF90AF909F908F9008958B
:100FA000AF92BF92CF92DF92EF92FF920F931F9377
:100FB000CF93DF93CDB7DEB768970FB6F894DEBF57
:100FC0000FBECDBF098B1A8B2B8B3C8B4D8B5E8B51
:100FD0006F8B788FDC0112962D913C911397232B08
:100FE00009F482C0CC2009F47FC06C01ED91FC9122
:100FF000028CF38DE02D19955C016DE27BE18BEFA6
:101000009EE00E9460B1CE0141960E940973A11436
:10101000B10451F460E0CE0141960E946975682FD9
:10102000F601848195815DC0F1E0AF16B10431F025
:1010300082E0A816B10421F081E003C085E001C080
:1010400084E019861A861B861C861D861E861F86CE
:10105000188A8295807F9B859F70892B8B87198644
:10106000EE24EA94FE2C09891A892B893C894D8942
:101070005E896F89788DCE0109960E94969563E20C
:101080007BE18BEF9EE00E9460B1CE0109960E9449
:101090000973A1E0AA16B10429F0B2E0AB16B104BD
:1010A00051F025C0B88863E070E0C6010E94DE9E62
:1010B0006B2D0E94F76D6F85F601848195810E94EA
:1010C000F76DBE8461E070E0C6010E94DE9E6B2D6C
:1010D0000E94F76DBD8462E070E0C6010E94DE9E52
:1010E0006B2D0E94F76D03C080E090E002C081E0AC
:1010F00090E068960FB6F894DEBF0FBECDBFDF91CB
:10110000CF911F910F91FF90EF90DF90CF90BF9004
:10111000AF9008950F931F93CF93DF93EC011D863B
:101120000A811B8160E070E0C8010E940A8B87FD84
:1011300002C08C8304C081958C8381E08D878C8173
:101140008150853410F080E28C8361E070E0C8014A
:101150000E940A8B87FD02C08D8304C081958D8318
:1011600081E08D878D818150853410F081E28D83FF
:1011700062E070E0C8010E940A8B863410F48E830E
:1011800001C01E8263E070E0C8010E940A8B9C01CE
:10119000215031092115344018F49A87898702C0FB
:1011A0001A86198664E070E0C8010E940A8B8130BB
:1011B00024E0920710F080E094E09C878B8765E044
:1011C00070E0C8010E940A8B1816190614F080E11D
:1011D00097E298878F83DF91CF911F910F910895A8
:1011E000CF93DF93EC010E949C9CCE010E948A88E1
:1011F0006CE179E08EE59EE00E94284661E08C81FA
:101200000E94C2A561E08D810E94C2A56D858C817E
:101210000E9493A56D858D810E9493A560E08E81CB
:101220000E94C2A540E050E0BA018A819B810E94E1
:10123000918A60E070E18A819B810E946B8B60E003
:1012400070E28A819B810E946B8B81E090E0909399
:10125000AD0A8093AC0A8093000281E090E0DF91B8
:10126000CF910895CF936130710541F164F4672BFC
:1012700091F59093330D8093320D5093350D40933B
:10128000340D81E024C06230710571F06330710566
:1012900011F59093330D8093320D55275093350DF2
:1012A0004093340D84E013C09093330D8093320D3E
:1012B0005093350D4093340D83E009C09093330D66
:1012C0008093320D5093350D4093340D82E00E948F
:1012D00045BAC82F06C06FE37CE18BEF9EE00E9409
:1012E00060B1CC2389F06AE27CE186E59EE00E9451
:1012F00060B14AE050E06C2F86E59EE00E94EFB1BD
:1013000086E59EE00E9487B281E0C11180E0CF9126
:10131000089587E090E008958AE090E0089581E0E4
:1013200090E0089588E090E00895CF93DF930097D0
:1013300009F46AC0FC012081222309F465C0EC0194
:1013400062E275E10E94FFCD892B09F442C066E09C
:1013500075E1CE010E94FFCD892BF1F162EC7CE1B9
:10136000CE010E94FFCD892BD1F16EEB7CE1CE0145
:101370000E94FFCD892BB1F16AEB7CE1CE010E9486
:10138000FFCD892B91F166EB7CE1CE010E94FFCD70
:10139000892B71F162EB7CE1CE010E94FFCD892B9C
:1013A00051F16EEA7CE1CE010E94FFCD892B31F133
:1013B00069EA7CE1CE010E94FFCD892B11F165EA3B
:1013C0007CE1CE010E94FFCD892BF1F48CE090E00E
:1013D0001DC082E090E01AC081E090E017C088E074
:1013E00090E014C085E090E011C086E090E00EC06F
:1013F00087E090E00BC089E090E008C08AE090E0D0
:1014000005C08BE090E002C080E090E0DF91CF91DA
:1014100008950C94A0CB0C94A0CB0F931F93CF9363
:10142000DF938C01FC01C081D1816FE270E0CE01BD
:101430000E94BBDA0097C1F0FC011192CF010E941B
:101440009589EC016DEE7CE18BEF9EE00E9460B12E
:101450004AE050E0BE018BEF9EE00E9480B28BEF2D
:101460009EE00E9487B209C0CE010E949589EC01DE
:10147000892B19F0F80111821082CE01DF91CF91F2
:101480001F910F910895DC01ED91FC91309729F0A7
:1014900090859F7081E0953009F080E00895EF928B
:1014A000FF920F931F93CF93DF93EC017B018E810B
:1014B0009F81892B01F5888199810E94C9B9082FE4
:1014C00010E005301105BCF40E9468B6FC01892BC0
:1014D00041F08085807F8260808711861286138626
:1014E0001486FF83EE83BF01888199810E94E9B948
:1014F0000F5F1F4FE6CFEE81FF81309751F080855F
:101500008F70823021F4E682F782F70102C0E0E0BA
:10151000F0E0CF01DF91CF911F910F91FF90EF90FD
:101520000895CF92DF92EF92FF920F931F93CF9384
:10153000DF93EC016A017B018E819F81892B01F58C
:10154000888199810E94C9B9082F10E005301105E2
:10155000BCF40E9468B6FC01892B41F08085807F35
:10156000826080871186128613861486FF83EE833D
:10157000BF01888199810E94E9B90F5F1F4FE6CFB3
:10158000EE81FF81309711F180858F708230F1F408
:10159000C186D286E386F48661EE7CE18BEF9EE025
:1015A0000E9460B12AE030E0B701A6018BEF9EE017
:1015B0000E9438B28BEF9EE0DF91CF911F910F9187
:1015C000FF90EF90DF90CF900C9487B2DF91CF9196
:1015D0001F910F91FF90EF90DF90CF900895FC0145
:1015E00086819781009791F0FC0120852F70223031
:1015F00041F0253059F460E00E9448B9009731F07D
:10160000FC016185728583859485089560E070E0B2
:10161000CB0108950F931F93CF93DF93FC01C281F9
:10162000D381209799F088858F70823029F4672BB9
:1016300069F489859A8514C0853041F48B01CE0107
:101640000E94C9B990E0081719071CF080E090E0EB
:1016500007C0602FCE010E9448B9FC0181859285A8
:10166000DF91CF911F910F9108950F931F93CF9307
:10167000DF93EC018B017B836A8381EC92E0998399
:10168000888360E070E0C8010E940A8B97FF03C066
:101690009195819591099D838C83D8011296ED9146
:1016A000FC911397309771F090859F70923039F0CC
:1016B000953041F4CF010E94C9B990E005C081E0A6
:1016C00090E002C080E090E09F838E83DF91CF9115
:1016D0001F910F9108950F931F93CF93DF93EB0109
:1016E00063E0FC01808191810E9448B9009741F13B
:1016F000AE01409550954F6F60E070E0FC010185B0
:101700001285238534854023512362237323418727
:1017100052876387748768ED7CE18BEF9EE00E94BF
:1017200060B14AE050E0BE018BEF9EE00E9480B2C3
:101730008BEF9EE0DF91CF911F910F910C9487B2B8
:10174000DF91CF911F910F9108950F931F93CF9326
:10175000DF93EB0163E0FC01808191810E9448B935
:10176000009731F1AE01442760E070E0FC01018593
:10177000128523853485402B512B622B732B418797
:101780005287638774876FEC7CE18BEF9EE00E9449
:1017900060B14AE050E0BE018BEF9EE00E9480B253
:1017A0008BEF9EE0DF91CF911F910F910C9487B248
:1017B000DF91CF911F910F910895CF93DF93EB01AC
:1017C00063E0FC01808191810E9448B9009739F063
:1017D000FC018185928588278C239D2302C080E0AF
:1017E00090E0DF91CF910895CF93C62F63E0FC0185
:1017F000808191810E9448B90097F9F0FC014185F0
:101800005285638574854427662777274C2B41874B
:1018100052876387748767EC7CE18BEF9EE00E94C0
:1018200060B14AE050E06C2F8BEF9EE00E94EFB178
:101830008BEF9EE0CF910C9487B2CF91089563E037
:10184000FC01808191810E9448B9009719F0FC0148
:10185000818508958FEF0895DC0119968D919C91F3
:101860001A97009739F0DC01ED91FC910280F38129
:10187000E02D19940895FF920F931F93CF93DF9358
:10188000EC010E94438A882309F4C1C088819981B0
:101890000E94C9B9082F10E004301105ACF40E9471
:1018A00068B6FC01892B41F08085807F826080874B
:1018B0001186128613861486BF01888199810E9441
:1018C000E9B90F5F1F4FE8CF0881198160E0C801B7
:1018D0000E9448B9DC011996FC90F88661E0C801C5
:1018E0000E9448B99B838A8362E0C8010E9448B97C
:1018F0009D838C8364E0C8010E9448B98C019F835A
:101900008E838F2D90E08F30910508F080C0FC0110
:101910008827EF5BFE4F8F4F0C94FBD68AE090E058
:101920000E9408CB8C01BE010E94358B80E495E0BB
:10193000F801918380833EC088E090E00E9408CB4C
:101940008C01BE010E94358B82EC94E0D8018D930E
:101950009C9330C08DE090E00E9408CB8C01BE01CA
:101960000E94358B85EE92E0F80191838083C80157
:101970000E94F5C11FC084E090E00E9408CBDC010A
:101980001396DC93CE93129720EA34E02D933C9388
:101990009A8789873CC08EE090E00E9408CB8C013A
:1019A000FC01D383C28385E692E091838083C801E2
:1019B0000E948A881A8709872AC086E090E00E94E0
:1019C00008CBFC01D383C28386EE94E009C086E095
:1019D00090E00E9408CBFC01D383C2838EE195E0A6
:1019E000918380830115110571F0D80118968C91AF
:1019F00018978F70823029F416960D911C911797C5
:101A000002C000E010E015830483FA87E987DF91C4
:101A1000CF911F910F91FF9008958F929F92AF9257
:101A2000BF92CF92DF92EF92FF920F931F93CF93CB
:101A3000DF93CDB7DEB767970FB6F894DEBF0FBE62
:101A4000CDBF8C017B014C018BE0880E911C9F8ADD
:101A50008E8AF801128611861386168A158A672BDC
:101A600009F448C0A0909610B0909710A114B1044A
:101A700009F440C06FE270E0C7010E9473DA6C01A4
:101A8000892B81F1F701DE01119680E090E0BD0124
:101A90002191222341F02F3231F08431910519F048
:101AA0002D930196F5CFFB01E80FF91F1082C501B8
:101AB0000E948F56F80191838083B6016F5F7F4F3C
:101AC0004AE050E0C4010E94ACDACE0146960E9482
:101AD0000D8AF801968B858B8E899F89892B69F4F5
:101AE00013860BC0B701C5010E948F56F801918380
:101AF000808303C0F80111821082C8010E943B8CD0
:101B000067960FB6F894DEBF0FBECDBFDF91CF91C1
:101B10001F910F91FF90EF90DF90CF90BF90AF900B
:101B20009F908F900895CF93DF93EC01FB01248168
:101B3000358140815181628173810E9438B2CE012A
:101B4000DF91CF910895089508956F927F928F92BB
:101B50009F92AF92BF92CF92DF92EF92FF920F933C
:101B60001F93CF93DF93CDB7DEB7C854D1090FB61B
:101B7000F894DEBF0FBECDBF3C014B01FC01E080FD
:101B8000F18063EE75E0C7010E948F565C0168EE3C
:101B900075E0C7010E948F566C01A114B10419F4BD
:101BA000892B09F4F9C065E876E0C7010E948F56D9
:101BB0008C0160E876E0C7010E948F567C01F3013A
:101BC00073806AE97CE18BEF9EE00E9460B14AE09D
:101BD00050E0672D8BEF9EE00E94EFB168E97CE159
:101BE0008BEF9EE00E9460B14AE050E0B4018BEFC1
:101BF0009EE00E9480B28BEF9EE00E9487B2C114EB
:101C0000D104E1F1F60180858F708430B9F56185EA
